:020000040000FA
:1000000000020400000000002E9E00002E9E000052
:100010002E9E00002E9E00002E9E00002E9E0000B0
:100020002E9E00002E9E00002E9E00002E9E0000A0
:100030002E9E00002E9E00002E9E00002E9E000090
:100040002E9E00002E9E00002E9E00002E9E000080
:100050002E9E0000647100008A7100002E9E000038
:100060002E9E00002E9E00002E9E00002E9E000060
:100070002E9E00002E9E00002E9E00002E9E000050
:100080002E9E00002E9E00002E9E00002E9E000040
:100090002E9E00002E9E00002E9E00002E9E000030
:1000A0002E9E00002E9E00002E9E00002E9E000020
:1000B0002E9E00002E9E00002E9E00002E9E000010
:1000C0002E9E00002E9E00002E9E00002E9E000000
:1000D0002E9E00002E9E00002E9E00002E9E0000F0
:1000E0002E9E00002E9E00002E9E00002E9E0000E0
:1000F0002E9E00002E9E00002E9E00002E9E0000D0
:100100002E9E00002E9E00002E9E00002E9E0000BF
:100110002E9E00002E9E00002E9E00002E9E0000AF
:100120002E9E00002E9E00002E9E00002E9E00009F
:100130002E9E00002E9E00002E9E00002E9E00008F
:100140002E9E00002E9E00002E9E00002E9E00007F
:100150002E9E00002E9E00002E9E00002E9E00006F
:100160002E9E00002E9E00002E9E00002E9E00005F
:100170002E9E00002E9E00002E9E00002E9E00004F
:100180002E9E00002E9E00002E9E00002E9E00003F
:100190002E9E00002E9E00002E9E00002E9E00002F
:1001A0002E9E00002E9E00002E9E00002E9E00001F
:1001B0002E9E00002E9E00002E9E00002E9E00000F
:1001C0002E9E00002E9E00002E9E00002E9E0000FF
:1001D0002E9E00002E9E00002E9E00002E9E0000EF
:1001E0002E9E00002E9E00002E9E00002E9E0000DF
:1001F0002E9E00002E9E00002E9E00002E9E0000CF
:10020000FFFFFF00FFFFFF002E9E00002E9E00005C
:100210002E9E00002E9E00002E9E00002E9E0000AE
:100220002E9E00002E9E00002E9E00002E9E00009E
:100230002E9E00002E9E00002E9E00002E9E00008E
:100240002E9E00002E9E00002E9E00002E9E00007E
:100250002E9E0000647100008A7100002E9E000036
:100260002E9E00002E9E00002E9E00002E9E00005E
:100270002E9E00002E9E00002E9E00002E9E00004E
:100280002E9E00002E9E00002E9E00002E9E00003E
:100290002E9E00002E9E00002E9E00002E9E00002E
:1002A0002E9E00002E9E00002E9E00002E9E00001E
:1002B0002E9E00002E9E00002E9E00002E9E00000E
:1002C0002E9E00002E9E00002E9E00002E9E0000FE
:1002D0002E9E00002E9E00002E9E00002E9E0000EE
:1002E0002E9E00002E9E00002E9E00002E9E0000DE
:1002F0002E9E00002E9E00002E9E00002E9E0000CE
:100300002E9E00002E9E00002E9E00002E9E0000BD
:100310002E9E00002E9E00002E9E00002E9E0000AD
:100320002E9E00002E9E00002E9E00002E9E00009D
:100330002E9E00002E9E00002E9E00002E9E00008D
:100340002E9E00002E9E00002E9E00002E9E00007D
:100350002E9E00002E9E00002E9E00002E9E00006D
:100360002E9E00002E9E00002E9E00002E9E00005D
:100370002E9E00002E9E00002E9E00002E9E00004D
:100380002E9E00002E9E00002E9E00002E9E00003D
:100390002E9E00002E9E00002E9E00002E9E00002D
:1003A0002E9E00002E9E00002E9E00002E9E00001D
:1003B0002E9E00002E9E00002E9E00002E9E00000D
:1003C0002E9E00002E9E00002E9E00002E9E0000FD
:1003D0002E9E00002E9E00002E9E00002E9E0000ED
:1003E0002E9E00002E9E00002E9E00002E9E0000DD
:1003F0002E9E00002E9E00002E9E00002E9E0000CD
:10040000CF272200007F22000001880000000000AA
:100410000C00070060FA280001002000110007000E
:10042000000020000000E000020032000000020096
:1004300000000000B49D0200000000000040DA004F
:100440000000FE004440A900E02E20000000E00073
:100450000300320000002000A00188004440A800F2
:100460000000060091018800800078000000EB0089
:1004700015003700E280400032A0B4009101BA00BC
:10048000E280400032A0B4009102BA00E280400055
:1004900032A0B4000002EB00472BDE00F507B200EB
:1004A000602CE10004003A000059EB008301E900F0
:1004B000FDFF3E00040037006128E100010032002A
:1004C0000082EB00040007001101BA000200E00006
:1004D000E8FF3A00000006003159BA008301E90044
:1004E0000C0032002159BA008301E90008003200F3
:1004F0000400E00003003A00E280400032A0B400B3
:10050000F5FF370011D9BA008301E900FAFF3A007C
:100510008100E800E180400032A0B4000000060045
:1005200000000000000000000000000000000000CB
:1005300000000000000000000000000000000000BB
:1005400000000000000000000000000000000000AB
:10055000000000000000000000000000000000009B
:1007E0000000000000000000889FBE008A9FBE003D
:1007F000010578000100E0000400350008003C001D
:100800000000E0002000320005003700600010000A
:10081000E080180002003B0001F02C001A003700B5
:100820000004BE006011B8006B0920000982CF00EF
:10083000020039000882CF000441B0006942520032
:100840000E00320008003B008281710061016400EB
:100850008904D1000884D3008B05E8000442E80035
:10086000F9FF3A00050037000804440089844C0071
:100870008B05E9000442E900FBFF3A002C01070068
:100880000AF0A70001F0A0004F05BE004F04BE0013
:1008900000000600F4FF2F004B0137001400200079
:1008A00049013700889FBE008A9FBE008C1F7800D8
:1008B000600107006701330003866C006450E100AB
:1008C0002E0032006420E100330032006150E1006C
:1008D0002F0032006120E100310032008585550093
:1008E000EB07B000090020000804200005003700D5
:1008F0000804440089844C000A00310006034300C8
:1009000087834B000001530081815B00F8FF3300B7
:100910000203BE000800A0000804440089844C00C3
:10092000F6FF3900C639DD00830173000100320093
:10093000130020008904D1000884D3000998A30083
:10094000050032000800A7000300A0008904D100C0
:100950000884D3008B05E8008904D1000884D30003
:100960000001EB000281D200F100070001F0A100BC
:100970000CF0A70001F0A0003F0137006420E10067
:10098000410132000801BE000200BE00F7FF37003F
:100990006120E1003C0132006000B800F3FF370045
:1009A0000000200001F82700F0FF370003F0A2004C
:1009B000889FBE008A9FBE008C1F78001D01070023
:1009C000240133006450E1004F0032006420E10054
:1009D0005200320003826C0007003B000905D00082
:1009E0000306D000820F54000C065D00020039009F
:1009F00002003200890178000306780085825500E4
:100A000004003D000003FD008103FD008502EA00B3
:100A10008B854200840F720002003B0060001000D2
:100A2000E08018006011B8000005EB007A28E100B2
:100A30000A00390006007800C75DDD00F707B20044
:100A4000878075002D003700828171000A017800CF
:100A5000610560008180D1000080D3008502E9003B
:100A6000F9FF3B00060440008784480002003B0079
:100A700060041400E0841C000988A3000700320011
:100A80008A81710082817100610164008904D10052
:100A90000884D3008B05E800170037000978A3000D
:100AA00013003A000B00E000130034008B05E9004E
:100AB0000804440089844C000A4474000978A300A7
:100AC0000D003A000B00E000070034008B05E90040
:100AD0000804440089844C0001003A000B00200007
:100AE0000978A300F7FF32000001EB000200370095
:100AF000828171000A0178008D0007000CF0A700C8
:100B000001F0A000DC0037006420E10002003A00A0
:100B1000838F6C00DC0033000801BE000200BE00C1
:100B2000D5003700889FBE008A9FBE008C1F7800CA
:100B3000C0000700C700330003866C006450E1006A
:100B4000240032006420E100270032006150E100FF
:100B5000220032006120E100210032008B8542003A
:100B6000EB07B1000134B800003AB80008044200B5
:100B700089844A00013AB8000030B80088804000FB
:100B800009014A0004003300000040008180480051
:100B9000020149008B05E900C909DD0083017000ED
:100BA0000100320013002000C814DE004814DD00EC
:100BB0004709DE001200B200C808DE000884700099
:100BC0005B00070001F0A1000CF0A70001F0A000FD
:100BD000A90037006120E100AB0032000801BE002F
:100BE0000200BE00F7FF37006150E100FCFF3A0051
:100BF000A50037000001BE00A60007000470A70092
:100C000003F0A10003F8A30013003A006509B10046
:100C100010003200090035006928E10002003500AB
:100C2000010028000000050000004000818048000D
:100C30008502E900FCFF3A0000000600F88F420040
:100C4000050035008100D1000080D3008502E80056
:100C5000FCFF3A00000006008000EB0000000500E9
:100C60006022B800060220000000D0008180D2007F
:100C70000482D2008582D2000000A000020252004D
:100C800083825A00030031000202420083824A003C
:100C90000000A1000603E900F3FF3A00000006008F
:100CA000EFFF07000400BE00000006000001BE00C8
:100CB000780007000470A70003F0A1006509B100E7
:100CC000160032000D0035006828E10006003500EE
:100CD000F0FF2F00F1FF27000300E00013003B00AE
:100CE000010028000000050000004000818048004D
:100CF0008502E900FCFF3A0008003700F88F420047
:100D000002003C008000EB00000005008100D100E3
:100D10000080D3008502E800FCFF3A000300E000F9
:100D200002003B0060001000E08018000000060098
:100D300081002000618055000B003D000B00200069
:100D400061FE2F000100E1001D003400828171006E
:100D5000610164008904D1000884D3000000E80028
:100D6000FAFF3A0071002000610064000300700087
:100D7000020060000900320061044400E0844C007D
:100D80000988A500050032008B05E8006808E1002D
:100D900002003A008904D1000884D300F20F200039
:100DA0000258E10005003D00C75DDD00F907B20013
:100DB0008980750008007800000006000BF8270005
:100DC0008B00780000000500889FBE008A9FBE004F
:100DD000841F7800170007004F00780011003300CF
:100DE000F0FF2F00838F6C0006003B0004056500B8
:100DF0000A00A7000800370009F0A6001000200034
:100E000008003700820F5400838F5C000300390014
:100E10001000200001003E000000200009F0A700A3
:100E20000000EA004F05BE004F04BE000000E000D5
:100E3000000006000004BE00160007000003BE000C
:100E40000405BE000200BE0012000700844F7500BA
:100E5000000006000200BE006450E10005003600FC
:100E60006420E100020036000968A30001003A0096
:100E70000800BE000160A0004F0678004F05BE00CC
:100E80004F04BE0000000600F0FF2F00F1FF270016
:100E9000F9FF3700C70ADE00F107B200F50FB20014
:100EA00008003200E1CF4200020032000170A000D1
:100EB00024000500810F70000100320004080500C5
:100EC00044000500810F700002003A001400050084
:100ED0008502E9000000400081C04800FCFF3B00A3
:100EE0000170A00024000500005E0000BCE20000CC
:100EF000613F0000DD830000C29C00007E200000F6
:100F0000A3FD00001F4100009DC30000217F0000E1
:100F1000FCA20000401E00005F010000E3BD0000D5
:100F20003E60000082DC0000237D00009FC10000C5
:100F3000421C0000FEA00000E1BF00005D030000B5
:100F400080DE00003C620000BEE00000025C0000A9
:100F5000DF810000633D00007C220000C09E000095
:100F60001D430000A1FF000046180000FAA4000085
:100F7000277900009BC5000084DA00003866000075
:100F8000E5BB000059070000DB8500006739000061
:100F9000BAE400000658000019470000A5FB000055
:100FA00078260000C49A0000653B0000D987000045
:100FB000045A0000B8E60000A7F900001B45000035
:100FC000C69800007A240000F8A60000441A000029
:100FD00099C70000257B00003A64000086D8000015
:100FE0005B050000E7B900008CD20000306E000005
:100FF000EDB30000510F00004E100000F2AC0000F5
:101000002F71000093CD0000114F0000ADF30000E0
:10101000702E0000CC920000D38D00006F310000D4
:10102000B2EC00000E500000AFF10000134D0000C4
:10103000CE900000722C00006D330000D18F0000B4
:101040000C520000B0EE0000326C00008ED00000A8
:10105000530D0000EFB10000F0AE00004C12000094
:1010600091CF00002D730000CA9400007628000084
:10107000ABF500001749000008560000B4EA000074
:1010800069370000D58B000057090000EBB5000060
:10109000366800008AD4000095CB00002977000054
:1010A000F4AA000048160000E9B70000550B000044
:1010B00088D60000346A00002B75000097C9000034
:1010C0004A140000F6A80000742A0000C896000028
:1010D000154B0000A9F70000B6E800000A54000014
:1010E000D78900006B3500004C450000540000001B
:1010F0004946000000540000484500004E00000032
:10110000454C000053450000004700004F540000CC
:101110004F000000474F0000535500004200000000
:101120005245000054550000524E0000005200008D
:10113000454D000000500000524900004E54000090
:10114000004900004E5000005554000000460000C9
:101150004F520000005400004F0000004E450000B8
:1011600058540000005200004541000044000000B7
:10117000444100005441000000530000544100006D
:10118000525400000053000054410000525400002B
:1011900052000000535400004F5000000053000064
:1011A000544F00005052000000530000454E000014
:1011B000440000005245000043450000495600002D
:1011C00045000000434C00004B000000444100007B
:1011D0005400000042490000545200004541000004
:1011E000440000004144000043000000415500005D
:1011F00058000000505300005500000050550000FA
:101200004C4C0000555000000041000055580000B3
:10121000504900004E0000004652000045510000B9
:1012200000440000555400005900000044450000EF
:101230004C410000590000004D41000043520000A5
:101240004F000000454E0000440000000052000026
:10125000554E0000004C00004953000054000000AF
:101260004558000049540000004400004542000079
:1012700055470000004E00004557000000000000E8
:101280003E200000000800002008000000000000D0
:10129000203D00002000000056520000454700009D
:1012A000207400006F6F0000206C00006F7700005A
:1012B0002C200000697300002074000068650000A5
:1012C000726500002061000020730000686F00005C
:1012D000727400003F0000002E2000003C0000005F
:1012E0003E0000002E200000000D00000A28000033
:1012F000002900003E20000000420000757300003D
:101300002050000069720000617400006520000038
:10131000763100006100000046690000726D000037
:10132000776100007265000020760000352E000015
:1013300035200000287200003436000034290000F7
:10134000002000002800000041330000004200009F
:101350003400000042350000004200003800000068
:10136000554E00004B000000290000004909000014
:10137000004F00000900000048090000004C000078
:1013800009000000456E0000746500007220000036
:101390007261000077200000766100006C7500002B
:1013A00065200000666F00007220000042520000BD
:1013B00047000000306200000030000030300000C4
:1013C0002C000000303000000030000031320000FE
:1013D0003334000035360000373800003941000052
:1013E0004243000044450000463000007800000001
:1013F000436F0000756C0000646E000027740000ED
:10140000206B000065650000702000007570000012
:1014100000000000535000004931000000000000AF
:1014200000290000002000005700000020520000AA
:101430000049000032430000310000003A20000063
:10144000000000002E000000315700003031000085
:101450000000000008080000080800000800000064
:1014600000000000204800007A000000000000009A
:1014700000410000525400003100000042420000D0
:10148000494F000031000000524100005731000078
:1014900000000000314100004C530000000000003B
:1014A0004F43000044310000000000000000000035
:1014B0000000000029000000000000000000000003
:1014C000000000001A00FA000000EB00100F980066
:1014D0000000EB00506988000000EB0040698800C4
:1014E0000000EB00A04088000000EB00606988006D
:1014F0000000EB00100798000000EB004007980088
:10150000140037000000EB00200798000B003700A4
:101510004E009000AE0090004500DD0081004000CC
:10152000E0D22000808040000040EB00804878003E
:101530002E0090000000E800200798002E00900088
:10154000FF0F5000F2FF34004E0090000000E80052
:10155000400798004E009000E40F5000E9FF34006F
:101560000000EB00706E8800A1408000E0022000C7
:101570000088B9006102200080804000E0932000D4
:1015800000804000B06C020000000000D1408000EC
:1015900000202000008060000000E0000400320015
:1015A00071002000C0592000C49902000000000012
:1015B00000942800B06C020000000000ED0037002D
:1015C000706E80000000E00063003200706E8000EA
:1015D0000000E900706E88000000EB002007980012
:1015E0001E00370042698000706E8000AE009000DF
:1015F0004500DD0081004000E0D220000080400076
:101600009040780080C2200000004100014878002E
:10161000706E8000AE0090004500DD00810040004B
:10162000E0D2200000804000104078000C710200E1
:1016300000000000406980000000E8004069880068
:101640002E0090000000E80020079800416980000B
:10165000F00F20000080600040698800706E8000FC
:10166000AE0090004500DD0081004000E0D2200087
:1016700000804000104078000004E000D9FF3A00EC
:101680000000EB00706E88003300370070B7200058
:1016900010407800624060000004E0002E0032003C
:1016A000A1408000E00220000088B900FA0040005C
:1016B000E09320000080400010007800000001004E
:1016C0000000E00024003200A1408000E002200081
:1016D0000088B9006102200080804000E093200073
:1016E00000804000B06C0200000000000094280060
:1016F000B06C020000000000516980004069800069
:10170000808F50001400320050698000200798003C
:101710000D003700AE00900080C220000080400025
:10172000104078000C71020000000000AE00900034
:10173000F00F200000806000200798002E0090002D
:101740000000E80020079800AE009000406980008B
:10175000808F5000EFFF3A00EE70020000000000A2
:101760000004E000C9FF3200FA700200000000002F
:10177000604798006E4090000080FB00200F9800AA
:101780002E089000E80F500011003200AE089000C3
:10179000E88F500007003C002E0990000200E00096
:1017A0003C003200AE099000E28F5100440032004C
:1017B0004B0037002E089000EA0F50001300320053
:1017C000AE089000ED8F500010003200440037004A
:1017D0004169800050698000808F500065003200B0
:1017E000406980000000E90040698800416980008C
:1017F000F00F2000008060004069880030942800CD
:10180000B06C0200000000005A00370010002000F9
:10181000100F9800406980008000E800F00F200061
:101820008080600050698000808F50000D00320081
:101830004169800080C22000808040000040EB00B1
:1018400080487800406980000000E8004069880016
:1018500041698000F00F200000806000406988002E
:101860000800370070C0B3000C71020000000000D7
:101870004169800080C22000808040000040EB0071
:101880008048780070942800DC6C020000000000A2
:10189000380037001E0090000000E8001007980094
:1018A0001E009000F40F500032003A002E77020024
:1018B000000000000000EB00100798002D0037002A
:1018C0001E009000E40F50002A00340096860200AB
:1018D000000000000000EB00100798002500370012
:1018E000406980008000E800F00F200080806000E8
:1018F00050698000808F5000160032006E409000CA
:10190000FF4F50001B0036006E4090000004E000C6
:10191000180035006E4090000C71020000000000BD
:10192000416980006E41900080C22000008040002C
:1019300002487800406980000000E80040698800A3
:1019400041698000F00F200000806000406988003D
:101950000800370070C0B3000C71020000000000E6
:101960004169800080C22000808040000040EB0080
:10197000804878001E0890000000E00010FF320050
:1019800040698000700798005069800060079800E7
:101990000000EB00100F98000000EB00000F980013
:1019A0000000EB0060698800D1408000002020002A
:1019B000008060000000E000A90432004E30020008
:1019C0000000000051002000305A20004E9A020012
:1019D0000000000010002000000F9800A004370055
:1019E0005169800080C220000080400010407800D3
:1019F000604798006E4090000080FB006101B900D4
:101A0000320F9800430F9800D007200001002000FB
:101A10003E099000CE099000800F5100818F59003F
:101A200061043E003E089000CE0890000060010076
:101A30005F0437005C0437005B0437005A0437004A
:101A4000590437005804370057043700560437004C
:101A5000550437005404370055043700520437004A
:101A600051043700520437004F0437004E0437004A
:101A70004D0437004C0437004B0437004A0437004C
:101A8000490437004804370047043700460437004C
:101A9000450437004404370043043700420437004C
:101AA00041043700400437003F0437003E0437004C
:101AB0003F0437001C04370093023700EE00370064
:101AC000FB003700AA0137009801370036043700C1
:101AD0006A02370034043700330437003404370017
:101AE00033043700C8033700E1033700AC03370085
:101AF0000D0337000C0337000B0337000A033700D0
:101B000009033700080337000703370006033700CF
:101B1000050337000403370023043700220437008D
:101B2000AB013700950037001F043700460037002F
:101B30000D013700FF0037001B0437006B00370032
:101B400077013700180437001704370016043700F0
:101B5000150437001404370013043700120437004B
:101B60006C003700100437000F0437000E043700F4
:101B70000D0437000C0437000B04370091013700C7
:101B80000904370008043700070437000C01370048
:101B9000050437000404370003043700BE02370091
:101BA0008C033700CE023700C0033700A303370091
:101BB000FD033700D20037002E0037004100370008
:101BC00049013700F8033700300037003200370092
:101BD000150037001F003700F3033700F20337000A
:101BE0005900370021003700EF033700230037008A
:101BF000ED033700EC0337002B0337006D0137008E
:101C0000E9033700E80337001E00370022013700E0
:101C1000E5033700E4033700E3033700A70237008A
:101C200073003700B70237009C0607000000E00091
:101C3000DF033A0050698000600798004069800027
:101C400070079800DA033700649A02000000000071
:101C5000D7033700F1070700A04080000000E00034
:101C6000D30332004F080700D103370003060700F3
:101C7000CF03370075090700CD0337004D09070072
:101C8000CB033700C1080700C90337007C7402008A
:101C900000000000C6033700A04080000000E00004
:101CA00005003A00D1012000305D20004E9A02006C
:101CB00000000000BE033700E072020000000000D8
:101CC000BB03370070B72000104078000000A1006F
:101CD00071B720008048780061012000805A200000
:101CE0004E9A020000000000B103370070B72000D8
:101CF000104078000000A00071B7200080487800F4
:101D000051012000E05B20004E9A0200000000001C
:101D1000A703370070B72000104078000020A00013
:101D200071B7200080487800C1012000B07E2000FB
:101D3000C49902000000000070942800DC6C0200CE
:101D4000000000009A03370070B7200010407800B0
:101D50000020A10071B7200080487800B101200068
:101D6000007D2000C499020000000000709428004B
:101D7000DC6C0200000000008D0337005069800019
:101D80000000E8005069880051698000F00F2000D1
:101D90000080600050698800A6050700BA030700AC
:101DA000200798002E009000AA6F0200000000009B
:101DB00080942800B06C0200000000002E0090000B
:101DC000486F02000000000080942800B06C020000
:101DD000000000002E009000106D020000000000C6
:101DE00070942800DC6C02000000000070033700D3
:101DF000506980000000E800506988005169800047
:101E0000F00F2000008060005069880089050700FD
:101E10009D030700200798002E0090008497020081
:101E2000000000000080FB00200798002E009000BA
:101E3000AA6F02000000000080942800B06C02002D
:101E4000000000002E009000486F0200000000001B
:101E500080942800B06C0200000000002E0090006A
:101E6000106D02000000000070942800DC6C02007D
:101E7000000000004E033700F49A0200000000004A
:101E80000000E0004A0332005100200030632000CF
:101E90004E9A02000000000023C2BF0061406000B3
:101EA0000004E000FCFF32000000FE0040033700A9
:101EB000F49A0200000000000000E0003C03320041
:101EC000A1002000806320004E9A02000000000064
:101ED0004006200022970200000000009E950200AC
:101EE0000000000023C2BF00614060000004E00069
:101EF000FCFF320081BF2A00014001002C033700A3
:101F0000060507000000E8004007980002003700BF
:101F1000BA750200000000004E0090000000E900C9
:101F2000400798004E0090000000E000F8FF3A00E3
:101F30001F033700F90407000000E800400798007D
:101F40000200370098750200000000004E0090006B
:101F50000000E900400798004E0090000000E000FB
:101F6000F8FF3A0012033700EC0407000000E80015
:101F7000400798000B00370061012000206420001A
:101F8000C499020000000000DC750200000000009F
:101F90009A6C02000000000070942800DC6C0200C3
:101FA000000000004E0090000000E900400798008B
:101FB0004E0090000000E000EFFF3A00FC02370006
:101FC000A04080000000E00005003A00D1012000A0
:101FD000305D20004E9A020000000000F40237003D
:101FE000C082A900C282A800C8A2A900CAA2A800F3
:101FF00021E3A8002000200022970200000000003A
:10200000A0C0B300E495020000000000800078004A
:10201000001B2000808F50000F00360090C0B300DE
:10202000E49502000000000080007800702B200082
:10203000808F5000080036001101200080652000CC
:10204000C49902000000000070942800DC6C0200BB
:10205000000000000E003700C082A900C282A90063
:10206000C8A2A900CAA2A900C0942800DC6C020082
:10207000000000002101200090662000C4990200A9
:102080000000000070942800DC6C020000000000DA
:1020900021E3A900C6023700A04080000000E00054
:1020A00005003A00D1012000305D20004E9A020068
:1020B00000000000BE023700C082A900C282A90051
:1020C000C8A2A900CAA2A900210120009066200090
:1020D000C49902000000000070942800DC6C02002B
:1020E00000000000B2023700F1002000A0392000FB
:1020F000C499020000000000FE95020000000000EC
:1021000011002000903A2000C49902000000000055
:1021100070942800DC6C020000000000A40237006C
:102120001096020000000000A10237007B040700A7
:10213000400798006100200070682000C4990200E8
:10214000000000004E009000EA6E02000000000057
:1021500021002000D06820004E9A020000000000FC
:102160004E0090004E9702000000000090023700E1
:102170006A04070040079800610020007068200092
:10218000C4990200000000004E009000EA6E0200B8
:10219000000000002100200090EC20004E9A020078
:1021A000000000004E009000229702000000000096
:1021B0007F023700D04080000090A000D04088000F
:1021C0007B02370010760200000000007802370022
:1021D000100020006069880010002000200798008F
:1021E00010003700516980002E0090008080400070
:1021F000F00F20008080600080C22000008040003E
:1022000090407800E0C3B30080CF500002003A0055
:102210000000EB00606988002E0090000000E800DC
:1022200020079800516980002E00900080804000B7
:10223000F00F20008080600080C2200000804000FD
:10224000104078000004E000E6FF3A00AE00900085
:1022500020022000808F5000020034001000200077
:1022600060698800606980000000E00050023A0068
:10227000506980000000E8005069880051698000C2
:10228000F00F200000806000506988007E02070087
:102290002007980051698000F00F200080806000C6
:1022A00080C220000080400090407800D0C3B3007E
:1022B00080CF500044003A002E0090000000E00063
:1022C0003E0034002E009000E50F50003B003C0023
:1022D000506980000000E800506988005169800062
:1022E000F00F200000806000506988002E009000F0
:1022F0000000E900200798000000EB00400798006C
:102300000B0037002E009000CE0090004500DD004D
:1023100081004000E0D22000808040000040EB00BF
:10232000804878004E0090000000E80040079800C8
:102330004E009000FF0F5000F2FF34000000EB0051
:102340004007980015003700AE0190004E02900043
:102350005169800080C22000008040001041780058
:102360004518DD0084004000E0D2200000804000DD
:10237000024878004E0090000000E80040079800F6
:10238000506980000000E8005069880051698000B1
:10239000F00F2000008060005069880051698000C3
:1023A00080C220000080400090407800E0C3B3006D
:1023B00080CF5000E4FF3A00FD01370010002000FC
:1023C00060698800FA0137002E0090000000E000EC
:1023D0001B003A000000EB00400798001400370093
:1023E0004E0090000040E800486F0200000000002E
:1023F000C0962800B06C0200000000004E00900063
:102400004500DD0080007800E0D220000080400020
:10241000B06C02000000000000972800DC6C020095
:10242000000000004E0090000000E8004007980007
:102430004E009000E40F5000E9FF3400DC0137004B
:102440002E0090000000E000090034002E009000F3
:10245000E50F500006003C0070942800DC6C020080
:1024600000000000AE009000716E8800D0013700BF
:102470001000200060698800CD013700506980009D
:102480000000E8005069880051698000F00F2000CA
:102490000080600050698800FB0107005007980029
:1024A000E403070051698000F00F20008080600085
:1024B00080C22000008040009040780090C2B300AD
:1024C00080CF50000D003A00A1408000E0022000C3
:1024D0000088B900FC004000E0932000008040002C
:1024E000900078005E0090000100010070942800C8
:1024F000DC6C020000000000AD013700100020007D
:1025000060698800AA013700100020006069880017
:10251000100020002007980010003700516980004B
:102520002E00900080804000F00F2000808060002E
:1025300080C22000008040009040780020C2B3009C
:1025400080CF500002003A000000EB006069880074
:102550002E0090000000E8002007980051698000DC
:102560002E00900080804000F00F200080806000EE
:1025700080C2200000804000104078000004E0008D
:10258000E6FF3A00606980000000E00088013A0040
:1025900071002000F0682000C499020000000000D3
:1025A00020C2B3000C7102000000000023003700BD
:1025B00051698000F00F20000080600050698800A1
:1025C0005169800080C220000080400010407800E7
:1025D0000C710200000000005169800080C22000E0
:1025E00000804000104078000000FB005007980079
:1025F00070B7200010407800644060000004E000E4
:10260000050032005E009000849702000000000088
:102610000080FB0050079800A1408000E0022000ED
:102620000088B900E8004000E093200000804000EE
:10263000900078005E009000010001005069800069
:102640000000E8005069880051698000F00F200008
:102650008080600080C220000080400090407800B0
:1026600020C2B30080CF5000D1FF3A0050698000F3
:10267000F10F2000010060005069880020C2B30003
:102680000C7102000000000070942800DC6C020055
:102690000000000046013700A1408000E002200059
:1026A0000088B90080007800E0932000008040009E
:1026B00010007800000001003D013700A1408000BB
:1026C000E00220000088B9008080E800E09320004C
:1026D0000080400010007800000001003401370045
:1026E000A1408000E00220000088B900E400400022
:1026F000E0932000008040001000780000000100FE
:102700002B013700A1408000E00220000088B900C2
:10271000E6004000E09320000080400010007800B8
:10272000000001002201370071002000F068200045
:10273000C4990200000000005301070050079800F0
:10274000506980000000E9005069880051698000EC
:10275000F00F20000080600050698800EF02070041
:102760000000E800400798000F030700000F780002
:102770001E00E000420032001E0078008040780019
:1027800080B72000014878003D0037005E009000CF
:102790009C9602000000000080B7200010407800E6
:1027A000E84F500007003200B0C3B3000C710200C4
:1027B0000000000080B7200010407800486F020041
:1027C0000000000070B720001040780064406000F6
:1027D0000004E000050032005E00900084970200D3
:1027E000000000000080FB0050079800A14080001E
:1027F000E00220000088B900E8004000E0932000DB
:1028000000804000900078005E0090000100010010
:102810002007980000C2B3000C7102000000000005
:10282000AE009000F00F2000808F500014003C009C
:102830006100200060692000C499020000000000CF
:1028400070B7200010407800644060000004E00091
:10285000050032002E009000849702000000000066
:102860000080FB00200798002E0090009C9602003C
:102870000000000000C2B3000C7102000000000064
:102880004E0090000000E900400798004E009000C4
:102890000000E000BDFF3A0070942800DC6C0200EC
:1028A00000000000C20037006100200060692000C5
:1028B000C499020000000000980207000000E80030
:1028C00040079800B8020700000F78001E00E000E3
:1028D000290032001E0078008040780080B7200078
:1028E0000148780024003700A1408000E002200069
:1028F0000088B900EA004000E0932000008040001A
:1029000010007800000001006047980070B72000B8
:1029100010407800644060000004E00004003200D1
:102920006E4090008497020000000000604798000D
:102930006E4090000080FB009C96020000000000AA
:1029400080B7200010407800E84F500007003200A8
:10295000B0C3B3000C7102000000000080B720007B
:1029600010407800486F02000000000000C2B30071
:102970000C710200000000004E0090000000E90011
:10298000400798004E0090000000E000D6FF3A009B
:1029900070942800DC6C0200000000008400370006
:1029A00081002000C06920004E9A02000000000053
:1029B000A1408000E00220000088B900EC00400047
:1029C000E09320000080400010007800000001002B
:1029D0007700370081002000406A20004E9A0200F4
:1029E00000000000A1408000E00220000088B90043
:1029F000EE004000E09320000080400010007800CE
:102A0000000001006A003700E1002000C06A2000D9
:102A10004E9A020000000000A1408000E002200069
:102A20000088B900F0004000E093200000804000E2
:102A300010007800000001005D003700E100200078
:102A4000A06B20004E9A020000000000A140800010
:102A5000E00220000088B900F2004000E09320006E
:102A60000080400010007800000001005000370096
:102A7000C1002000B0672000C499020000000000DF
:102A8000A1408000E00220000088B900F40040006E
:102A9000E09320000080400010007800000001005A
:102AA0009A6C020000000000410037001B02070082
:102AB00040079800D1002000806D2000C4990200DA
:102AC000000000004E0090009C96020000000000F4
:102AD0004E0090000000E800400798000800370012
:102AE000A1408000E00220000088B900F60040000C
:102AF000E0932000008040001000780000000100FA
:102B00004E0090000000E900400798004E00900041
:102B10000000E000F2FF3A0070942800DC6C020034
:102B20000000000022003700FC0107000000E80060
:102B300040079800A1002000506E2000C4990200B8
:102B4000000000000D003700A1408000E0022000DE
:102B50000088B900F8004000E093200000804000A9
:102B600010007800000001009A6C020000000000D4
:102B700000C2B3000C710200000000004E00900083
:102B80000000E900400798004E0090000000E000BF
:102B9000EDFF3A0001012000806C20004E9A0200F7
:102BA000000000000200370010002000606988006B
:102BB000506980000000E800506988005169800079
:102BC000F00F20000080600050698800606980007C
:102BD0000000E0001C00320051012000F06E2000D7
:102BE000C499020000000000EE00900050698000CF
:102BF000808F5000070031005069800080407800CD
:102C00006E00900000C05000486F020000000000FD
:102C10000600370050698000804078006E00900008
:102C200000C05000486F0200000000000000EB00F0
:102C30006069880010002000000F98007094280040
:102C4000DC6C0200000000005169800040698000D7
:102C5000808F500002003A0010002000000F980002
:102C60000E0890000000E0005DFB32007E00900046
:102C7000506988007E009000406988000000EB00E9
:102C8000100F980038FA37000600FA000000EB0039
:102C9000100798000000EB00000F780051698000D9
:102CA0001E00900080804000F00F200080806000B7
:102CB00080C22000008040009040780000C3B30034
:102CC00080CF500043003400516980001E00900006
:102CD00080804000F00F20008080600080C22000D3
:102CE000008040009040780090C3B30080CF500037
:102CF00038003C00516980001E0090008080400038
:102D0000F00F20008080600080C220000080400022
:102D1000104078008000FB0000FD2F00008F400075
:102D20001E0090000000E800100798001200370015
:102D30001E0078006A00B900000F78005169800019
:102D40001E00900080804000F00F20008080600016
:102D500080C2200000804000104078000000FB008E
:102D60009E00400000FD2F00008F40001E009000DC
:102D70000000E80010079800516980001E009000D4
:102D800080804000F00F20008080600080C2200022
:102D90000080400090407800F0C2B30080CF500027
:102DA00051013400516980001E0090008080400075
:102DB000F00F20008080600080C220000080400072
:102DC0009040780090C3B30080CF5000D8FF34000B
:102DD00045013700516980001E009000808040004E
:102DE000F00F20008080600080C220000080400042
:102DF0009040780000C3B30080CF500035013A0006
:102E00001E0090000000E800100798005169800043
:102E10001E00900080804000F00F20008080600045
:102E200080C22000008040009040780020C6B3009F
:102E300080CF50000B003200516980001E009000CE
:102E400080804000F00F20008080600080C2200061
:102E5000008040009040780020C4B30080CF500034
:102E60002D003A001E0090000000E80010079800B6
:102E7000120037001E00780000004000000F7800AC
:102E8000516980001E00900080804000F00F2000FB
:102E90008080600080C220000080400010407800E8
:102EA0000000FB009E00400000FD2F00008F40004E
:102EB0001E0090000000E800100798005169800093
:102EC0001E00900080804000F00F20008080600095
:102ED00080C22000008040009040780010C3B30002
:102EE00080CF5000E3FF3200516980001E00900047
:102EF00080804000F00F20008080600080C22000B1
:102F0000008040009040780000C3B30080CF5000A4
:102F1000D8FF3200F4003700516980001E00900095
:102F200080804000F00F20008080600080C2200080
:102F3000008040009040780080C7B30080CF5000F0
:102F40000B003200516980001E009000808040001C
:102F5000F00F20008080600080C2200000804000D0
:102F60009040780080C5B30080CF50008E003A00BA
:102F70001E0090000000E80010079800470037008E
:102F80001E0078004400DD00000F780051698000C9
:102F90001E00900080804000F00F200080806000C4
:102FA00080C220000080400090407800F0C2B30052
:102FB00080CF500018003400516980001E0090003E
:102FC00080804000F00F20008080600080C22000E0
:102FD000008040009040780090C3B30080CF500044
:102FE0000D003C00516980001E0090008080400070
:102FF000F00F20008080600080C220000080400030
:10300000104078000000FB009E00400000FD2F00F3
:10301000008F40001E003700516980001E009000A4
:1030200080804000F00F2000008160005169800026
:103030001E00900080804000F00F20008080600023
:1030400080C22000008040009040780000C2B300A1
:1030500080C0700080C2200000004100014878005C
:10306000516980001E00900080804000F00F200019
:103070008080600080C22000008040001040780006
:103080000000FB009E00400090FA2F00008F4000DF
:103090001E0090000000E8001007980051698000B1
:1030A0001E00900080804000F00F200080806000B3
:1030B00080C220000080400090407800F0C2B30041
:1030C00080CF50000B003400516980001E0090003A
:1030D00080804000F00F20008080600080C22000CF
:1030E000008040009040780090C3B30080CF500033
:1030F000A3FF3400516980001E00900080804000D2
:10310000F00F20008080600080C22000008040001E
:103110009040780000C4B30080CF50000B00340012
:10312000516980001E00900080804000F00F200058
:103130008080600080C220000080400090407800C5
:1031400060C4B30080CF50008DFF3400516980000F
:103150001E00900080804000F00F20008080600002
:1031600080C22000008040009040780000C6B3007C
:1031700080CF50005C003400516980001E00900038
:1031800080804000F00F20008080600080C220001E
:10319000008040009040780060C6B30080CF5000AF
:1031A00077FF340050003700516980001E00900006
:1031B00080804000F00F20008080600080C22000EE
:1031C0000080400090407800F0C2B30080CF5000F3
:1031D00045003400516980001E009000808040004E
:1031E000F00F20008080600080C22000008040003E
:1031F0009040780090C3B30080CF50003A003C006C
:10320000516980001E00900080804000F00F200077
:103210008080600080C22000008040001040780064
:103220008000FB0000FD2F00008F400012003700DF
:103230001E0078006A00B900000F78005169800014
:103240001E00900080804000F00F20008080600011
:1032500080C2200000804000104078000000FB0089
:103260009E00400000FD2F00008F40001E009000D7
:103270000000E80010079800516980001E009000CF
:1032800080804000F00F20008080600080C220001D
:103290000080400090407800F0C2B30080CF500022
:1032A00011003400516980001E00900080804000B1
:1032B000F00F20008080600080C22000008040006D
:1032C0009040780090C3B30080CF5000D8FF340006
:1032D0000500370010002000606988000000EB0046
:1032E000200798000A003700516980001E009000F6
:1032F000008040005069880051698000F00F200074
:1033000000806000506988001E0078002007980047
:103310002E0090000080FA00000006000400FA0071
:10332000506980008000E800F00F2000808060007D
:1033300080C220000080400090407800A0C3B3000D
:1033400080CF500013003A00506980000080E800F0
:103350005069880051698000F00F200000806000F3
:103360005069880048FE0700000F7800506980000F
:103370000000E9005069880051698000F00F2000CA
:1033800000806000506988001E00780010079800D7
:103390000200370010002000100798001E00900067
:1033A0000080FA00000006000400FA005069800066
:1033B0008000E800F00F20008080600080C22000C4
:1033C0000080400090407800B0C3B30080CF500030
:1033D00013003A00506980000080E80050698800BE
:1033E00051698000F00F2000008060005069880063
:1033F00025FE0700000F7800506980000000E900FA
:103400005069880051698000F00F20000080600042
:10341000506988001E0078001007980002003700ED
:103420000000EB00100798001E0090000080FA00DA
:10343000000006000000FA00070037005069800015
:103440000000E8005069880051698000F00F2000FA
:1034500000806000506988005169800080C22000AF
:10346000008040009040780000C2B30080CF500040
:10347000F2FF32000080FA00000006000400FA00AB
:103480000000EB00000F7800506980000000E800A9
:103490005069880051698000F00F200000806000B2
:1034A00050698800E3FF0700F7FD0700000F780070
:1034B0001E00E0004D003A000000EB0010079800ED
:1034C000130037001E0090000040E800486F020023
:1034D0000000000020972800B06C020000000000EF
:1034E0009E009000E00220000088B90061022000E8
:1034F00080804000E093200000804000DC6C0200EF
:10350000000000001E0090000000E8001007980076
:103510001E009000E80F5000EAFF34007101200007
:10352000407020004E9A0200000000000000EB00F6
:103530006069880013002000920020001100200024
:1035400010002000F6000700000FE900E0FF2F0048
:103550009E0F1000030032000080EB009E0F100051
:1035600005003A00E1002000B07120004E9A0200F0
:103570000000000042003700A1408000E00220006F
:103580000088B9000102200080804000E093200004
:103590000080400010007800000001009E950200AD
:1035A000000000001E007800A0408800A1408000BC
:1035B000E00220000088B900FE004000E0932000F7
:1035C0000080400010007800000001001E00E000B4
:1035D00001003200CA82A80051002000305A2000A9
:1035E0004E9A020000000000250037001E0FE9007F
:1035F000800020009E0F10001D003C00A1408000B4
:10360000E00220000088B900010220008080400014
:10361000E0932000008040001000780000000100CE
:103620009E950200000000001E007800A040880067
:10363000A1408000E00220000088B900FE004000A8
:10364000E09320000080400010007800000001009E
:103650001E00E00001003200CA82A80051002000D4
:10366000305A20004E9A020000000000040037008B
:1036700051012000907220004E9A020000000000CC
:10368000406980008000E900F00F200000806000A9
:10369000506988000080FA00000006002600FA0049
:1036A0001000200020079800506980000000E90009
:1036B000100798009E009000F00F2000008060002E
:1036C00010079800430037009E00900080C2200041
:1036D00000804000104078000004E00036003A000E
:1036E0001E0090008000E800F00F20008080600045
:1036F00080C2200000804000104078000004E000FC
:103700002D0032002E009000486F020000000000E3
:1037100020972800B06C020000000000100020007C
:10372000000F78000A0037001E0090009E00400045
:10373000F00F20008080600080C2200000804000E8
:10374000104078000C710200000000001E0FE8001D
:103750001E0090009E004000F00F2000808060005E
:1037600080C2200000804000104078000004E0008B
:10377000EDFF3A00AE0190001E0090008000E800CE
:10378000F00F200000816000E60047000380410048
:1037900002B078002E0090000000E800200798009A
:1037A0002E009000EF0F50000E00320070942800A1
:1037B000DC6C0200000000001E0090000000E90028
:1037C000100798009E009000F00F2000008060001D
:1037D000100798009E00900050698000808F500074
:1037E000B9FF3A0071002000E07320004E9A0200F9
:1037F00000000000130020002E01900011002000A6
:103800000000EB0046000700100798001E00900023
:10381000E10F400003003A0010002000201798003C
:103820003C0037000000EB0020079800160037002E
:10383000416980002E00900080804000F00F200041
:10384000008160001E009000E6004700000040007C
:10385000E08078002E00900080804000F00F200073
:103860008080600080C2200000804000904078008E
:1038700080C2200000004100014878002E00900026
:103880000000E800200798001E009000E6004700B6
:1038900000004000E08078002E0090008080400012
:1038A000F00F20008080600080C220000080400077
:1038B000104078000004E000DDFF3A00406980001D
:1038C0008000E900F00F200000806000506988004F
:1038D000516980002E009000008040008080E80048
:1038E000F00F20000080600040698800406980007F
:1038F0008000E900F00F20008080600080C220007E
:10390000808040000040EB00804878000000EB0021
:10391000201798002E1090000080FA00000006008A
:103920001E00FA00100F9800210F9800320F980027
:10393000430F98000000EB00400798000000EB00E8
:10394000200798000000EB00100798000000EB0033
:10395000000F780050972800B06C020000000000B3
:103960001E089000486F0200000000009097280099
:10397000B06C02000000000067003700FA7002001F
:1039800000000000204F98002E4890000000FB002F
:10399000600F98006E089000ED0F50002900320073
:1039A000EE089000ED8F500007003C006E0990007B
:1039B000E80F51000D0032006E089000EA0F500031
:1039C0002000320035003700D0022000EE089000C1
:1039D000808F50001E003200800720006E0990008A
:1039E000800F5100270032002C0037004E0090005D
:1039F0000000E000070032004E0090000000E900E7
:103A00004007980030942800B06C020000000000CD
:103A1000410037001E00E000060032000000EB000D
:103A2000000F780030942800B06C02000000000005
:103A30003900370070C0B3000C71020000000000B4
:103A400035003700100020002007980032003700B2
:103A50004E0090000000E00006003A00D0C2B30023
:103A60000C7102000000000010002000000F780020
:103A70002900370070C0B3000C7102000000000084
:103A8000250037004E0890000000E00003003200DF
:103A90000080EB00500F98005D003700AE489000AA
:103AA000F0C2B30080CF500018003400AE48900040
:103AB00090C3B30080CF500014003C004E00900033
:103AC000E30F50000600340070C0B3000C71020018
:103AD0000000000040002000400798000E00370062
:103AE0002E4890000C71020000000000CE009000F3
:103AF0006B0047002E499000827078004E009000C5
:103B00000000E800400798000300370070C0B300D1
:103B10000C710200000000002E0090000000E00088
:103B200096FF320070942800DC6C02000000000058
:103B30004E0090000000E00003003A001E089000D4
:103B4000500F9800320037000000EB00100798007B
:103B50004E0090000000E90040079800CE00900061
:103B600031079800110037001E0090006A00B9006C
:103B700010079800BE0090004E009000808050001A
:103B80006B004700614078008000FB001E00900041
:103B90008080400000FD2F0000804000100798004A
:103BA0004E0090000000E900400798004E00900091
:103BB0000000E000ECFF3D009E0090002E08900009
:103BC000808F50000D0035009E0090003E08900050
:103BD000808F500009003C001E00E000040032000D
:103BE0001E0090000000EA00500F98000800370007
:103BF0001E019000520F980005003700B10120000F
:103C0000E0EA20004E9A02000000000049FF370061
:103C10005E0890000080FA00000006000400FA0030
:103C2000D0972800DC6C020000000000C09828003B
:103C3000B06C020000000000D10020007080200065
:103C4000C499020000000000A1BF2A000000EB00A0
:103C50002472020000000000000F78001E007800AF
:103C60004800DE00486F020000000000E0C2B30020
:103C70000C710200000000001E007800486F020076
:103C80000000000070942800DC6C020000000000BE
:103C90006100200000762000C499020000000000AE
:103CA000B04080000270020000000000710020009F
:103CB00070EA2000C499020000000000C0408000AB
:103CC0000270020000000000109A2800B06C020090
:103CD00000000000C040800010079800200423006E
:103CE0009E009000808F50001600320020042300B8
:103CF0009E009000808F500005003E0030002300A1
:103D00009E009000808F50000A003200190037009A
:103D1000300423009E009000808F50000D00320080
:103D2000600423009E009000808F50000D00320040
:103D300010003700409A2800B06C0200000000001C
:103D40000F003700709A2800B06C020000000000DD
:103D50000B003700A09A2800B06C020000000000A1
:103D600007003700D09A2800B06C02000000000065
:103D700003003700009B2800B06C02000000000028
:103D8000409B2800DC6C020000000000E1012000E4
:103D9000607620004E9A0200000000000080FA00C9
:103DA000000006000000FA005100200020922000D0
:103DB000C499020000000000C1BF2A000000EB000F
:103DC00024720200000000000270020000000000E7
:103DD0006100200070922000C499020000000000E1
:103DE000E1BF2A000000EB00247202000000000086
:103DF000027002000000000070942800DC6C0200D9
:103E000000000000C1002000407820004E9A02000F
:103E1000000000005D000700CAC2BF000042B200FF
:103E20000004E00005003200110120008065200040
:103E3000C4990200000000000400370021012000A6
:103E400090662000C499020000000000C0C2B300C8
:103E50000C7102000000000000C2B3000C710200EF
:103E60000000000070B7200010407800684060003B
:103E70000004E0000500320021022000007920004B
:103E80004E9A02000000000004003700E10120000B
:103E9000207B20004E9A02000000000070B7200036
:103EA00010407800644060000004E00005003A0023
:103EB000B1012000007D2000C49902000000000034
:103EC00004003700C1012000B07E2000C499020028
:103ED00000000000C0C2B3000C710200000000002E
:103EE00000C2B3000C71020000000000B10120000C
:103EF000C0202100C49902000000000080B720000B
:103F000010407800486F0200000000007094280004
:103F1000DC6C02000000000070B720001040780048
:103F2000614060000004E000050032005101200003
:103F3000E05B20004E9A0200000000000400370001
:103F400061012000805A20004E9A0200000000000B
:103F5000A1408000E00220000088B900410220005A
:103F600080804000E0932000008040001000780036
:103F700000000100C1002000407820004E9A02009D
:103F8000000000000080FA00000006000000FA00B7
:103F9000A1002000A00521004E9A020000000000B0
:103FA00061042000200B21004E9A02000000000056
:103FB000A101200040062100C49902000000000079
:103FC000A1408000E00220000088B900210220000A
:103FD00080804000E09320000080400010007800C6
:103FE00000000100A1002000E0072100C4990200A8
:103FF00000000000004020005000070000102000DA
:104000004E000700002020004C00070000042000A4
:104010004A000700000820004800070070942800AC
:10402000DC6C02000000000041002000800F210035
:10403000C49902000000000021E3A800A0C0B30062
:10404000E4950200000000004C7002000000000037
:1040500011002000903A2000C499020000000000E6
:1040600090C0B3000C7102000000000090C0B300CB
:10407000E4950200000000004C7002000000000007
:1040800011002000903A2000C499020000000000B6
:1040900090C0B3000C71020000000000C0C0B3006B
:1040A000E4950200000000004C70020000000000D7
:1040B00011002000903A2000C49902000000000086
:1040C00090C0B3000C71020000000000B0C0B3004B
:1040D000E4950200000000004C70020000000000A7
:1040E00011002000903A2000C49902000000000056
:1040F00090C0B3000C7102000000000021E3A90091
:10410000004020001C000700001020001A000700DB
:1041100000202000180007000004200016000700FF
:10412000000820001400070070942800DC6C0200D6
:10413000000000000080FA00000006000200FA0003
:10414000000F7800401680001E0060000000E000B4
:1041500004003200609B2800B06C020000000000E8
:1041600003003700909B2800B06C020000000000A4
:104170000080FA00000006000200FA00000F78003C
:10418000501680001E0060000000E00004003200B5
:10419000C09B2800B06C0200000000000300370044
:1041A000F09B2800B06C0200000000000080FA00C4
:1041B000000006000200FA00506980000000E800DC
:1041C0005069880051698000F00F20000080600075
:1041D0005069880097FC0700ABFA0700000F7800D1
:1041E0001E00E00006003400400020009E0F10007A
:1041F00003003C001E00E900904088000D003700DD
:104200000000EB006069880021022000408120004E
:104210004E9A0200000000008001EB0042002000E6
:104220001100200010002000BDFD07000000E90083
:104230009040880021012000608320004E9A0200F7
:10424000000000000080FA00000006000200FA00F2
:10425000506980000000E8005069880051698000C2
:10426000F00F2000008060005069880071FC07009A
:1042700085FA0700104798001E4090000004E000F7
:10428000090032001E409000EA4F500006003E0038
:104290001E4090000040E90080407800008120002E
:1042A000014878000F0037000000EB0060698800CB
:1042B000D1082000308720004E9A02000000000044
:1042C0008001EB00A20020001100200090002000DF
:1042D00093FD07000040E900804078000081200045
:1042E000014878000081200010407800E94F50001C
:1042F00010003A004FFC070063FA0700004F7800F7
:104300001E04E0000B003A000000EB00606988002A
:10431000209C2800DC6C0200000000008001EB0003
:10432000F2FF27008000EB00200220007CFD070048
:10433000004F780041012000009020004E9A0200BA
:104340000000000011012000B01F21004E9A020061
:104350000000000023C2BF00614060000004E000D4
:10436000FCFF32000081200010407800E94F50002F
:1043700003003A001E4078002A710200000000008D
:104380006E9602000000000000003700EE70020090
:10439000000000000004E000FCFF3200FA700200A0
:1043A000000000008040780000C2B30080CF5000C1
:1043B00001003200F5FF37000080FA00000006001F
:1043C0000000FA006173800040E720000080400098
:1043D0009040780030C8B30080CF50000E003A0003
:1043E000607380000000E8006073880003003700FD
:1043F000607380000000E8006073880061738000D3
:1044000040E72000008040009040780000CEB300DC
:1044100080CF5000F6FF36000080FA000000060052
:104420000A00FA00300798000000EB00200798000F
:10443000AE00900040E720000080400090407800EF
:1044400000CEB30080CF500003003E000080EB00A0
:104450004007980023003700AE00900040E720009E
:1044600000804000104078008080FB0000F22F00A8
:1044700000804000100798002E0090008000E800A7
:1044800040E7200000804000104078000080FB00E2
:104490004801DD002E0090008080E80040E7200009
:1044A00000804000104078000080FB00000F4100B9
:1044B0009E0078003E009000808F500003003A007C
:1044C0002E00900040079800060037009E009000E4
:1044D0002E009000008040006300400020079800FC
:1044E000D3FF37004E0090000080FA000000060065
:1044F0000600FA00881F78000000EB00000F78002B
:104500006173800040E72000008040009040780008
:1045100080C2B30080CF500010003A00607380006A
:104520000000E800607388001D010700000F78009C
:104530006173800040E720000080400090407800D8
:1045400090C2B30080CF5000AA003A006073800090
:104550000000E80060738800A600370061738000E7
:1045600040E72000008040009040780000C4B30085
:1045700080CF5000160036006173800040E72000B5
:104580000080400090407800A0C5B30080CF50006C
:104590000F003E006273800040E7200000004100F1
:1045A000104078008080FB00F0FB2F00008040006E
:1045B00080004000C0E02000008040001000780033
:1045C000200798000200E800607388008B00370025
:1045D0006173800040E72000008040009040780038
:1045E00000C8B30080CF50007400360061738000B3
:1045F00040E7200000804000104078000080FB0071
:10460000100798000100E80060738800700920001E
:104610009E009000808F5000410032007009200001
:104620009E009000808F50000D003C00400920004B
:104630009E009000808F500016003200600920001C
:104640009E009000808F50002B0032003009200027
:104650009E009000808F5000180032004600370006
:10466000900920009E009000808F50001E003200B4
:10467000900920009E009000808F50003900350086
:10468000A00920009E009000808F50002E00320074
:1046900039003700A1408000E00220000088B90006
:1046A000EA004000E0932000008040001000780005
:1046B00000000100000F78004E003700A14080008C
:1046C000E00220000088B900E8004000E0932000EC
:1046D00000804000100478008200070008000100FC
:1046E000000F780043003700DC7502000000000076
:1046F000000F78003F003700A1408000E00220005A
:104700000088B900F4004000E093200000804000E1
:104710001000780000000100000F7800350037001D
:10472000A1408000E00220000088B900F8004000AD
:10473000E09320000080400010007800000001009D
:10474000000F78002B003700CAC2BF000080FB00BA
:104750004500DE00614060000080FB00000F780033
:1047600024003700C0C0B300E49502000000000040
:10477000000F78001F0037000000EB00000F7800EA
:104780001C0037001E0078006A00B900000F780096
:104790006173800040E720000080400010407800F6
:1047A0000080FB009E00400000FD2F00008F4000B5
:1047B000607380000000E80060738800617380000F
:1047C00040E720000080400090407800F0C2B30035
:1047D00080CF5000070036006173800040E7200062
:1047E000008040009040780090C3B30080CF50001C
:1047F000E4FF36001E007800200798002E0090008D
:104800004F0478000080FA00000006000600FA005D
:1048100037FF0700000F7800000037006173800049
:1048200040E720000080400090407800A0C2B30024
:1048300080CF50000A0032006173800040E7200002
:104840000080400090407800F0C2B30080CF50005C
:10485000030032001E007800200798001E00370079
:104860006173800040E72000008040001040780025
:104870000080FB00100798000100E80060738800CA
:10488000A00220009E009000808F500005003200A2
:10489000F00220009E009000808F50000700320040
:1048A000DEFF370012FF0700800078001E0078004E
:1048B0000180B900000F7800D8FF37000CFF070017
:1048C000000178001E007800110009000200D800E5
:1048D000000F7800D1FF37002E0090000080FA0012
:1048E000000006000600FA00C8FF0700000F78006D
:1048F000000037006173800040E720000080400026
:1049000090407800D0C2B30080CF50000A0032003F
:104910006173800040E720000080400090407800F4
:10492000B0C2B30080CF5000030032001E007800F8
:1049300020079800170037006173800040E72000CF
:1049400000804000104078000080FB0010079800B5
:104950000100E80060738800B00220009E00900013
:10496000808F500008003200D00220009E0090008E
:10497000808F500001003200DEFF3700A3FF0700E8
:104980001E0F1000DBFF3700A0FF07001E0F4000C6
:10499000D8FF37002E0090000080FA0000000600CB
:1049A0000C00FA006273800040E720000000410024
:1049B000104078008080FB00F0FB2F00008040005A
:1049C00080004000C0E0200000804000900078009F
:1049D000210798000200E800607388000000EB00E7
:1049E000000F78000B0037009E0178006273800092
:1049F00040E720000000410010407800804078002F
:104A000066004700817178000200E800607388004A
:104A10001E0FE8006173800040E720000080400026
:104A20009040780000C4B30080CF500007003600EB
:104A30006173800040E720000080400090407800D3
:104A4000A0C5B30080CF50000E0036006173800017
:104A500040E720000080400090407800F0C2B300A2
:104A600080CF5000E0FF36006173800040E72000F7
:104A7000008040009040780090C3B30080CF500089
:104A8000D9FF3E0097FF0700100798006600470017
:104A9000104078000000FB0050079800C003200081
:104AA000DE009000808F500032003200C0032000F2
:104AB000DE009000808F500005003C0010022000B6
:104AC000DE009000808F5000410032004E00370021
:104AD000D0032000DE009000808F500005003200DF
:104AE000E0032000DE009000808F50000A003200BA
:104AF000450037000000EB0040079800AE00900032
:104B00001E009000808F500041003A0011002000EC
:104B1000410798003E003700660047009040900033
:104B2000D0C3B30080CF500009003A000000EB0072
:104B300040079800AE0090001E009000808F50004B
:104B40003300350011002000410798003000370085
:104B50000000EB0040079800AE0090001E0090009F
:104B6000808F50002A003400110020004107980077
:104B7000270037006600470090409000D0C3B30084
:104B800080CF500009003A000000EB004007980079
:104B9000AE0090001E009000808F50001C003C0072
:104BA0001100200041079800190037000000EB00B9
:104BB00040079800AE0090001E009000808F5000CB
:104BC00013003D001100200041079800100037003D
:104BD0006600470090409000D0C3B30080CF5000E3
:104BE00009003A000000EB0040079800AE0090007A
:104BF0001E009000808F5000050032001100200040
:104C000041079800020037000000EB0040079800C1
:104C10004E0090000080FA00000006001C00FA0020
:104C2000881F78000000EB00607388000000EB0034
:104C3000300798000000EB00200798000000EB0010
:104C4000100798000000EB00707388000000EB0074
:104C5000807388000000EB00907388000000EB0078
:104C600050079800D04080000080A000D04088000D
:104C70000000EB0040079800090037004E0090004C
:104C800080004000C0E02000808040000000EB0079
:104C9000800878004E0090000000E800400798006F
:104CA0004E009000F90F5000F4FF34003304370039
:104CB0001E0090000000E00021003A0061738000B7
:104CC00040E720000080400090407800F0CDB30025
:104CD00080CF500003003E002000200030079800E5
:104CE000290437006173800040E720000080400005
:104CF000104078008080FB0000F22F000080400010
:104D000060079800607380008000E80040E72000A2
:104D100000804000104078000080FB004801DD006A
:104D2000607380008080E80040E720000080400041
:104D3000104078000080FB000000710050079800D0
:104D40000000EB001007980060738000E300400053
:104D500040E7200000804000104078000080FB0009
:104D60006101B90000F82F00F1FF2F00020140009F
:104D700083814800420F9800530F980010022000D2
:104D8000010020004E099000DE099000800F5100C4
:104D9000818F5900ED033E004E089000DE08900020
:104DA000006001002100370035003700E7033700BD
:104DB000E60337007100370081003700A300370099
:104DC000B7003700BE0037003B01370088013700CD
:104DD000DE033700EE013700350237009902370055
:104DE000A0023700AE023700BC023700CA0237000B
:104DF000D8023700D50337007A0337005E03370047
:104E0000D2033700D1033700E2023700F002370047
:104E1000A1033700AC033700000337001403370049
:104E200034033700B4033700C503370010002000F7
:104E3000200798006073800066004000607388005F
:104E4000607380008080E90040E72000008040001F
:104E5000104078008080FB00F0FB2F0000844000B1
:104E6000A0FE07000001780088004400C0E0200098
:104E7000008040000208780051FD0700B5033700AC
:104E8000100020002007980060738000640040003C
:104E900060738800C2FE07000000E0001C003200C2
:104EA00061738000310F980040E720003E099000B8
:104EB00000004100904078008041EB00435798008B
:104EC00020C8B30080CF500002003A0010C0B300E9
:104ED00040579800BE0890000100E8006073880009
:104EE0004E5190000204E0009A03320010002000AE
:104EF00010079800607380006300500060738800A2
:104F000094033700607380000000E800607388003D
:104F10006173800040E720000080400090407800EE
:104F200030C8B30080CF50000700320061738000AA
:104F300040E72000008040009040780000CEB300A1
:104F400080CF5000EFFF36006173800040E7200003
:104F5000008040009040780030C8B30080CF5000FF
:104F60007C033A0010002000100798006073800056
:104F70000080E9006073880076033700100020008D
:104F80002007980060738000640040006073880010
:104F900054FE070022FD0700000F78008081EB001F
:104FA0009E8F1100030032001E007800607388009D
:104FB0006803370060002000300798006503370061
:104FC00010002000200798006073800064004000FB
:104FD0006073880080738000E90F500018003C0067
:104FE00082738000617380006E009000008040003A
:104FF0008001E9008200410000E4200000804000C0
:1050000003087800807380000000E8008073880047
:1050100034FE070002FD0700000F78008080EB00DF
:105020009E8F1000030032001E017800627388001A
:105030004803370060002000300798004503370020
:1050400070002000300798004203370000892800D4
:10505000B06C020000000000100020002007980043
:10506000807380000000E0000A003200807380003E
:105070000000E90080738800807380008000400099
:1050800000E4200000804000100078006073880079
:105090003003370080002000300798002D033700D0
:1050A0001000200020079800617380006E009000BF
:1050B00000804000630040006073880025033700D3
:1050C00010002000200798006073800064004000FA
:1050D00060738800570037006173800040E720004C
:1050E000008040009040780020C2B30080CF500084
:1050F0001F003A00607380000000E80060738800C1
:1051000010003700D04080000080A100D04088000F
:105110006173800040E7200000804000104078006C
:10512000004178000100E8006073880002407800C8
:105130000C71020000000000D04080000080A00040
:10514000D04088006173800040E72000008040006C
:105150009040780020C2B30080CF5000E9FF3A00B1
:10516000607380000000E800607388003100370041
:105170006173800040E7200000804000904078008C
:1051800000C4B30080CF5000070036006173800078
:1051900040E720000080400090407800A0C5B300A8
:1051A00080CF50000D0036006173800040E7200082
:1051B00000804000104078000004E00013003D0033
:1051C0006173800040E7200000804000904078003C
:1051D000F0CDB30080CF50000C003E00C1FD0700B1
:1051E000000F7800D04080000080A100D0408800EF
:1051F0001E007800EA6E020000000000D04080002F
:105200000080A000D04088000A0037006173800051
:1052100040E720000080400090407800B0C3B30019
:1052200080CF500003003A00607380000000E80067
:10523000607388006173800040E7200000804000B8
:1052400090407800F0CDB30080CF500007003E00C2
:105250006173800040E720000080400090407800AB
:1052600030C8B30080CF50009BFF3A0060738000CD
:105270008000E90040E72000008040009040780076
:10528000B0C3B30080CF500009003200D04080008E
:105290000080A100D040880060922800DC6C0200F1
:1052A00000000000D04080000080A000D0408800B6
:1052B00043FC0700A70237001000200020079800D9
:1052C000D04080000080A100D04088006073800042
:1052D00064004000607388006173800040E7200034
:1052E000008040009040780020C2B30080CF500082
:1052F00018003A00607380000000E80060738800C6
:105300000A0037006173800040E720000080400001
:1053100010407800004178000100E80060738800C8
:10532000024078000C7102000000000061738000F0
:1053300040E72000008040009040780020C2B30089
:1053400080CF5000EFFF3A00607380000000E8005B
:10535000607388006173800040E720000080400097
:1053600090407800C0C2B30080CF500004003A00E3
:10537000607380000000E80060738800020037005E
:1053800030002000300798006173800040E7200063
:1053900000804000104078008080FB00F0FB2F0070
:1053A000008440008001EB00F2FF27008000EB004A
:1053B0000000EB00901C02000000000000017800DB
:1053C00088004400C0E0200000804000020878000F
:1053D000607380000000E80060738800F8FB07003D
:1053E000D04080000080A000D040880059023700E3
:1053F00010002000200798006073800064004000C7
:105400006073880070738000E30F500004003C005C
:10541000707380000000E80070738800020037009D
:105420004000200030079800727380006373800092
:1054300040E7200000804100104078008080FB00A1
:1054400000FC2F00008240006610B9008080E80058
:1054500040E5200000804000040878000300E800D8
:10546000607388006173800040E720000080400086
:1054700090407800D0C3B30080CF500011003A00B4
:10548000607380000000E800607388007073800023
:105490006600B9008080E80040E520000080400000
:1054A000100078000004E9000EFD070000017800FC
:1054B00088004400C0E0200000804000020878001E
:1054C000020037003000200030079800637380002E
:1054D000130F980040E720009E08900000804000D5
:1054E000904078000041EB0002579800B0C8B3002C
:1054F00080CF500002003A0013C0B3000357980059
:105500009E0890000100E800607388000E51900032
:105510000204E0000900320078738000F1FC07000B
:10552000000178006640B900E400400040E520003A
:1055300000804000020878000200370030002000A0
:10554000300798006173800040E720000080400031
:1055500090407800F0CDB30080CF500008003600B6
:1055600070738000627380006600B900800078006C
:1055700040E520000080400002087800020037006B
:1055800030002000300798008DFB0700F101370044
:105590001000200020079800607380006400400025
:1055A000607388006273800040E7200000004100C3
:1055B000104078008080FB0000FC2F00008F40002E
:1055C0000200E80060738800500020003007980057
:1055D0000000EB00400798002F0037004E009000BD
:1055E0006600B9008080E80040E5200000804000AF
:1055F000100078009E0F500024003A001E00E900C1
:1056000080004000C0E020000080400010017800D1
:105610004E0090006600B900E400400040E5200024
:105620000080400010007800800F510012003D0003
:105630009E00E90001814000C0E020000000410020
:10564000100078000001E80081804000C0E02000E8
:1056500000804000020878004E0090006600B9000B
:105660008000780040E520000080400010007800B5
:105670006073880003003700707380000000E90049
:10568000707388000000EB00300798004E00900017
:105690000000E80040079800717380004E00900001
:1056A000810F5000CDFF340045FB0700A9013700F2
:1056B0001000200020079800607380006400400004
:1056C00060738800907380000000E00027003A00BB
:1056D0000000EB00400798000A003700CE00900061
:1056E00040E7200000804000104078008080FB00F0
:1056F0004E0090008080400030F22F00008040007B
:10570000400798004E009000E300400040E7200072
:105710000080400090407800E0C8B30080CF500087
:1057200006003200CE00900040E7200000804000DC
:10573000104078000004E000E8FF3A00CE0090003E
:1057400040E7200000804000104078000004E000A6
:10575000040032004E009000640040009073880006
:10576000020037009000200030079800637380002B
:10577000030F780090738000607388009E007800AB
:1057800040E7200000804000104078008080FB004F
:10579000F0FB2F000084400055FB0700000178005B
:1057A00088004400C0E0200000804000020878002B
:1057B00060738000907388001E00E80060738800AA
:1057C0009173800040E72000008040009040780006
:1057D000C0C2B30080CF500003003A009073800035
:1057E0000000E800907388009173800040E720007B
:1057F000008040009040780000CEB30080CF500081
:105800000E00360090738000E300400040E7200067
:105810000080400090407800E0C8B30080CF500086
:10582000030032000000EB00907388000300370093
:10583000907380006400400090738800E0FA0700D5
:105840004401370010002000200798006173800099
:105850006E0090000080400063004000607388008C
:105860003C01370010002000200798006073800082
:105870006400400060738800A1408000E0022000C6
:105880000088B90080007800E0932000008040008C
:105890001000780000000100C9FA07002D01370050
:1058A0001000200020079800607380006400400012
:1058B00060738800A1408000E00220000088B900E9
:1058C0008080E800E0932000008040001000780015
:1058D00000000100BAFA07001E0137001000200086
:1058E00020079800607380006400400060738800A7
:1058F000A1408000E00220000088B900E4004000E0
:10590000E0932000008040001000780000000100BB
:10591000ABFA07000F0137001000200020079800A5
:10592000607380006400400060738800A1408000C4
:10593000E00220000088B900E6004000E09320006B
:105940000080400010007800000001009CFA070071
:1059500000013700100020002007980060738000CD
:105960006400400060738800A1408000E0022000D5
:105970000088B900E8004000E0932000008040006B
:1059800010047800D7FB0700080001008CFA07001C
:10599000F00037001000200020079800607380009E
:1059A0006400400060738800CEFB07000000E00048
:1059B000030032009875020000000000020037006A
:1059C000BA750200000000007DFA0700E100370010
:1059D00010002000200798006073800064004000E1
:1059E00060738800BFFB07000000E0000500320084
:1059F000C082A900C282A800C8A2A900CAA2A800A9
:105A000004003700C082A900C282A900C8A2A90070
:105A1000CAA2A9006AFA0700CE00370010002000D1
:105A20002007980060738000640040006073880065
:105A3000ACFB07000000E0000600320070B7200059
:105A4000104078000000A00071B720008048780066
:105A50000500370070B72000104078000000A0005B
:105A600071B720008048780055FA0700B900370068
:105A70001000200020079800607380006400400040
:105A80006073880097FB0700206188002061800018
:105A90000000E00002003D000000EB0020618800F3
:105AA0002161800000FA2000808F50000200340045
:105AB00000FA20002061880030618000E10F500072
:105AC00002003C002000200030618800316180002D
:105AD00030062000808F5000020034003006200085
:105AE000306188003E7202000000000034FA0700B6
:105AF0009800370010002000200798006073800095
:105B0000640040006073880076FB07003061880005
:105B1000206180000000E00002003D000000EB007A
:105B2000206188002161800000FA2000808F5000F1
:105B30000200340000FA20002061880030618000FB
:105B4000E10F500002003C0020002000306188007E
:105B50003161800030062000808F50000200340048
:105B600030062000306188003E7202000000000014
:105B700013FA070077003700100020002007980074
:105B800060738000640040006073880055FB07006C
:105B90000000E00009003200A1408000E002200087
:105BA0000088B900F0004000E09320000080400031
:105BB000100078000000010008003700A1408000BC
:105BC000E00220000088B900F2004000E0932000CD
:105BD000008040001000780000000100F8F9070084
:105BE0005C003700100020002007980060738000E0
:105BF00064004000607388003AFB0700700798005B
:105C00007E009000E10F500010003200FE00900076
:105C1000E28F5000160032007E0190000200E0008A
:105C2000010032001A003700A1408000E00220008D
:105C30000088B900EE004000E093200000804000A2
:105C4000100078000000010011003700A140800022
:105C5000E00220000088B900EC004000E093200042
:105C600000804000100078000000010008003700AC
:105C7000A1408000E00220000088B900F60040004A
:105C8000E093200000804000100078000000010038
:105C9000CBF907002F0037001000200020079800E4
:105CA000607380006400400060738800617380004E
:105CB0006E009000008040000000E90060738800E2
:105CC000BFF90700230037001000200020079800CC
:105CD00060738000640040006073880001FB07006F
:105CE000000F78001E0078002297020000000000DC
:105CF000B3F90700170037001000200020079800B4
:105D0000607380006400400060738800F5FA07004B
:105D1000000F7800A1408000E00220000088B90058
:105D2000FC004000E09320000080400090007800DC
:105D30001E00780001000100A1F9070005003700EE
:105D400010002000300798000200370030002000CB
:105D5000300798002E0090000000E00005003A0097
:105D6000617380006E00900000804000630040007E
:105D7000607388000000EB00200798003E00900050
:105D80000000E000CAFB3200D04080000080A1008B
:105D9000D04088003E009000E10F50001800320013
:105DA00061002000A03A2000C49902000000000019
:105DB0003E009000EA6E020000000000810020001A
:105DC000003B2000C4990200000000005E0090002B
:105DD000EA6E020000000000B1002000803B2000BD
:105DE000C49902000000000060738000EA6E0200A7
:105DF0000000000060922800DC6C0200000000003F
:105E00004F0478000080FA00000006000200FA004B
:105E1000000F780000C2B3000C7102000000000007
:105E20001E007800B06C02000000000000C2B30049
:105E30000C710200000000000080FA000000060063
:105E40000400FA000000EB00607388003F00370098
:105E50006173800040E7200000804000904078009F
:105E6000214798002E4090000004E0000400350017
:105E70002E4090000C71020000000000300037003E
:105E8000AE40900000CEB30080CF50001C00360022
:105E900060922800DC6C020000000000607380004B
:105EA0008000E80040E720000080400010407800BB
:105EB0000080FB004801DD00607380008080E80006
:105EC00040E7200000804000104078000080FB0088
:105ED00000004100000F7800607380000080E8003F
:105EE000607388001E007800EA6E02000000000067
:105EF00000C2B3000C710200000000001000370067
:105F000000C2B3000C710200000000002E4090009F
:105F10008080FB0000F82F000080400080004000DF
:105F200020B320000080400010007800B06C020018
:105F30000000000000C2B3000C710200000000006D
:105F4000607380000000E800607388006173800067
:105F500040E7200000804000104078000004E0008E
:105F6000BBFF3A0060922800DC6C020000000000D9
:105F7000607380000000E900EA6E0200000000008B
:105F800071002000303C20004E9A0200000000000A
:105F90000080FA00000006000600FA0010079800D2
:105FA00050698000000F7800170037001E00900035
:105FB000104178005169800080C2200000804000BC
:105FC00010407800804F5100050032001E0078001C
:105FD000506988000000EB0020079800100037008F
:105FE000506980000000E800506988005169800015
:105FF000F00F200000806000506988001E009000B3
:106000000000E800100798001E0090001040780083
:106010000004E000E5FF3A0010002000200798008F
:106020002E0090000080FA00000006000400FA0034
:106030000000EB00000F7800100037001E00780011
:106040008000400020B32000008040001000780055
:10605000D1FF07000000E000070032001E007800BA
:106060008040780000C8B30000C040000080FB0002
:1060700010079800060037001E0FE80000022000FD
:106080009E0F1000EDFF34000000EB001007980099
:106090001E0090000080FA00000006003200FA00A6
:1060A00050698000600798001F003700EE009000E4
:1060B00080C22000008040009040780000C6B300FD
:1060C00080CF500011003400EE00900080C220000C
:1060D0000080400090407800A0C7B30080CF5000FF
:1060E0000A003C006E019000EE00900080C220008B
:1060F0000080400090407800F0CDB30080C0600088
:1061000080C2200000004100014878006E0090002D
:106110000000E80060079800EE009000F00F2000FB
:106120000080600060079800EE00900040698000E9
:10613000808F5000DDFF3A000000EB006007980000
:106140005169800080C220000080400090407800AB
:10615000F0C2B30080CF50001F01340051698000AD
:1061600080C22000008040009040780090C3B300BF
:1061700080CF500018013C000000EB006007980041
:10618000070037006E019000EE0047000040EB0072
:1061900000F178006E0090000000E80060079800B1
:1061A000EE00900020022000808F5000F5FF3400A8
:1061B0004416020000000000400798004E009000C6
:1061C0004880DE00804078006E0047001140980053
:1061D0004E0090008040780000C0EB0080C060005E
:1061E0006E004700214098004E0090008CF8070098
:1061F000300798003E009000E10F40002B00320075
:10620000BE00900040E72000008040001040780071
:106210008080FB0030F22F000080400010079800C3
:106220003E009000600798000D0037006E0190005E
:10623000EE0090001E0090008080400040E72000AB
:10624000008040009040780040E7200000004100BE
:10625000014878006E0090000000E8006007980098
:10626000014020001E009000808050006E009000D1
:10627000808F5000EDFF3C0008003700EE009000DA
:1062800040E72000808040000040EB00804878001C
:106290006E0090000000E80060079800EE0090009B
:1062A000F03F2000808F5000F4FF340030002000C9
:1062B000600798000000EB00000F78001A1A020037
:1062C000000000003E0037001E00E00002003A001F
:1062D0001A1A0200000000001E00E00004003A004C
:1062E00052FF07000080FB004007980002003700C3
:1062F0000000EB00400798004E0090000000E00016
:106300000C0032006E0190004E009000804078003A
:106310006E00470001717800CE00900070082000E8
:10632000808F50001A003A0010002000000F780003
:10633000170037005169800080C2200000804000B3
:106340009040780020C2B30080CF500001003A0096
:106350001E00A2006E0190005169800080C22000E2
:106360000080400010407800804078006E004700B8
:1063700001717800506980000000E80050698800D1
:1063800051698000F00F2000008060005069880093
:106390006E0090000000E80060079800EE0090009A
:1063A00030022000808F5000050034009100200052
:1063B000A03C20004E9A020000000000E5003700DB
:1063C0005169800040698000808F5000BEFF3A0014
:1063D0006E009000E30F5000DE0032006E0090006F
:1063E000E40F5000DB0032006E0090008040780027
:1063F000C0CDB30000C04000804078006E00470070
:10640000014878000000EB00600798000000EB00F6
:10641000200798000000EB00300798003D0037008F
:10642000EE00900040E7200000804000904078009F
:1064300000CEB30080CF500025003600EE00900063
:1064400040E7200000804000104078008080FB0082
:1064500000F22F0000804000100798006E009000AE
:106460008000E80040E72000008040009040780075
:106470006E0047001040900080CF50000E003E009C
:106480006E0090008080E80040E72000008040001F
:10649000904078006E0047002040900080CF500070
:1064A00005003100EE0090001E00900000804000CA
:1064B00063004000300798009E0090006E0090003E
:1064C0000080400063004000600798000200370031
:1064D0006E009000200798006E0090008000E80099
:1064E00040E7200000804000104078000080FB0062
:1064F0004801DD006E0090008080E80040E7200049
:1065000000804000104078000080FB000000410047
:10651000400798002E0090000000E000C0FF32000D
:106520006E004700104078008080FB0030F22F00A2
:1065300000804000400798002E00900060079800FF
:106540000D003700EE0090004E00900000814000EA
:10655000EE00900040E7200000804000904078006E
:1065600040E7200000004100014878006E009000E4
:106570000000E90060079800EE0090003E009000E7
:10658000808F5000EFFF3D000000EB006007980097
:106590000C003700BE0090006E00900000814000AB
:1065A000EE0090006E004700E140780040E72000D8
:1065B00000004100014878006E0090000000E800F3
:1065C00060079800EE0090004E009000808F500011
:1065D000F0FF35005F003700709228006EFE070064
:1065E0000000E000050032008CF9070060922800EE
:1065F000DC6C02000000000056003700B09228005A
:1066000065FE07000000E000020032000CFE0700FB
:1066100050003700009328005FFE07000000E000F4
:1066200004003200D04080000090A100D0408800DB
:10663000480037005093280057FE07000000E00094
:10664000200032000000EB006007980018003700BF
:106650000000EB00500798000F003700EE0090009C
:106660005E0090008080400040E7200000804000F5
:10667000104078000080FB00AA6F020000000000BC
:1066800000C2B3000C710200000000005E00900028
:106690000000E800500798005E009000EF0F5000E7
:1066A000EEFF34006E00900070004000600798001C
:1066B000EE009000F03F2000808F5000E4FF340097
:1066C00024003700B093280033FE07000000E000EC
:1066D0001C0032000000EB00600798000800370043
:1066E000EE00900040E72000808040000040EB007A
:1066F000804878006E0090000000E8006007980075
:10670000EE009000F03F2000808F5000F4FF340036
:1067100011CEB30040E720000148780080C0EB00B4
:1067200050E720000148780080C0EB0060E72000BF
:106730000148780011CAB30070E7200001487800D2
:1067400004003700C1002000303D20004E9A0200B6
:10675000000000000080FA000000060057524900C7
:1067600054452000424954003A2020002A6E65001A
:1067700078742000636C6F00636B2000285E290032
:10678000207769006C6C20007573650020746800C8
:106790006973200076616C007565310057495200BD
:1067A000452072006F757400696E650073202800C3
:1067B000432920003230300030204D0069636800EA
:1067C00061656C00205065006172630065204700C0
:1067D0004E55200047504C004E6F200064657600F7
:1067E000696365002C2074007279200028414C00F8
:1067F00041524D002920530045415200434820009A
:106800006D616300726F20006669720073744100ED
:106810004444520045535300204D410043524F0021
:10682000202030002E4D610063726F00206D6500E6
:106830006E754D00616372006F20200020202000E3
:10684000315749005245200061646400726573004D
:10685000730D0A00202020002A31570049524500BC
:1068600020524F004D2043004F4D4D00414E4400FB
:10687000204D410043524F00733A0D000A2035006D
:10688000312E52004541440020524F004D20280037
:1068900030783300332920002A666F00722073009D
:1068A000696E67006C652000646576006963650049
:1068B00020627500730D0A00203835002E4D41000E
:1068C0005443480020524F004D20280030783500B6
:1068D000352920002A666F006C6C6F0077656400B4
:1068E00020627900203634006269740020616400FF
:1068F0006472650073730D000A20320030342E007C
:10690000534B4900502052004F4D20002830780052
:1069100043432900202A66006F6C6C006F77650086
:1069200064206200792063006F6D6D00616E640009
:106930000D0A2000323336002E414C0041524D00EA
:10694000205345004152430048202800307845003C
:1069500043290D000A20320034302E0053454100F7
:106960005243480020524F004D2028003078460006
:10697000302941004C4152004D2053004541520006
:106980004348200028307800454329005345410002
:1069900052434800202830007846300029446500E2
:1069A00076696300652049004473200061726500C8
:1069B0002061760061696C0061626C006520620094
:1069C00079204D00414352004F2C20007365650033
:1069D00020283000292E52004541440020524F000B
:1069E0004D2028003078330033293A00204D4100F3
:1069F0005443480020524F004D2028003078350085
:106A0000352953004B49500020524F004D2028009B
:106A100030784300432955006E6B6E006F776E002F
:106A2000206D610063726F002C2074007279200069
:106A30003F206F007220280030292000666F72000E
:106A4000206865006C704200555320005245530089
:106A500045542000576172006E696E00673A20004D
:106A60002A5368006F727400206F7200206E6F00EE
:106A7000207075006C6C2D00757020002A4E6F0020
:106A800020646500766963006520640065746500B4
:106A90006374650064204400533138005332300081
:106AA0002048690067682000507265007320440028
:106AB0006967200054686500726D440053313800E6
:106AC00042323000205072006F6720005265730020
:106AD0002044690067205400686572006D445300CB
:106AE0003138320032204500636F6E002044690067
:106AF00067205400686572006D44530032343000E2
:106B000034204500636F6E0072616D00207469006F
:106B10006D652000436869007044530032343300CF
:106B2000312031004B204500455052004F4D55005B
:106B30006E6B6E006F776E0020646500766963008F
:106B4000655057004D20640069736100626C6500F8
:106B500064314B00487A2D00342C300030304B002B
:106B6000487A200050574D004672650071756500E7
:106B70006E63790020696E00204B48007A20500037
:106B80007265730063616C00653A500052323A00DE
:106B9000447574007920630079636C006520690096
:106BA0006E202500205057004D206100637469005D
:106BB0007665450052524F00523A200050574D0022
:106BC0002061630074697600652C200067207400E2
:106BD0006F20640069736100626C65004155580064
:106BE0002046720065717500656E6300793A200079
:106BF0004155580020494E00505554002F48490037
:106C00002D5A410055582000484947004841550039
:106C100058204C004F5756004F4C54004D455400DF
:106C2000455220004D4F440045564F004C54410002
:106C30004745200050524F0042453A00205645003B
:106C400072726F007228290020406C00696E650026
:106C50003A20400070676D007370610063653A0010
:106C600020627900746573002E546F006F206C00F1
:106C70006F6E6700215379006E74610078206500A3
:106C800072726F00724E6F002045450050524F00E7
:106C90004D457200617369006E6764006F6E650038
:106CA00053617600696E670020746F0020736C007A
:106CB0006F742000496E7600616C69006420730077
:106CC0006C6F74004C6F610064696E006720660031
:106CD000726F6D0020736C006F742000455252007B
:106CE0004F523A0020636F006D6D61006E642000AA
:106CF00068617300206E6F00206566006665630042
:106D0000742068006572650041434B004E414300AA
:106D10004B4932004320530054415200542042005A
:106D2000495449003243200053544F005020420040
:106D300049544900324320006D6F6400653A0D00EC
:106D40000A2031002E2053006F66740077617200B4
:106D5000650D0A0020322E00204861007264770021
:106D6000617265005365740020737000656564008E
:106D70003A0D0A0020312E00207E35004B487A0063
:106D80000D0A2000322E20007E3530004B487A005C
:106D90000D0A2000332E20007E313000304B480099
:106DA0007A0D0A0020342E00207E340030304B0053
:106DB000487A570041524E00494E47003A20480059
:106DC00041524400574152004520490032432000BF
:106DD0006973200062726F006B656E00206F6E0039
:106DE0002074680069732000504943002120280066
:106DF000524556002041330029536500742073002A
:106E000070656500643A0D000A2031002E203100C3
:106E100030304B00487A0D000A2032002E2034001A
:106E200030304B00487A0D000A2033002E2031000C
:106E30004D487A004932430020286D006F642000DD
:106E400073706400293D2800202030002E4D610021
:106E500063726F00206D65006E750D000A203100B1
:106E60002E376200697420006164640072657300EB
:106E7000732073006561720063680D000A203200A0
:106E80002E493200432073006E6966006665720009
:106E90005365610072636800696E670020493200C3
:106EA0004320610064647200657373002073700096
:106EB000616365002E2046006F756E0064206400DB
:106EC0006576690063657300206174003A536E0053
:106ED00069666600657228004241530049432900F3
:106EE00052656100647961002F412F0040206300EA
:106EF0006F6E7400726F6C00732041005558200053
:106F000070696E00612F41002F402000636F6E009A
:106F100074726F006C7320004353200070696E0020
:106F2000436F6D006D616E0064206E006F74200011
:106F300075736500642069006E20740068697300D1
:106F4000206D6F0064655000756C6C002D757000CD
:106F50002072650073697300746F720073204F00B4
:106F600046465000756C6C002D75700020726500EF
:106F700073697300746F720073204F004E53650085
:106F80006C662D0074657300742069006E204800E3
:106F9000695A20006D6F640065206F006E6C790087
:106FA00052455300455442004F4F54004C4F41004E
:106FB000444552004155580020494E005055540058
:106FC0002F4849002D5A2C002052450041443A00D8
:106FD00020506F00776572002073750070706C0030
:106FE00069657300204F4E00506F77006572200076
:106FF00073757000706C6900657320004F46460021
:10700000444154004120530054415400453A20006B
:1070100044454C00415920007573570052495400B3
:10702000453A200052454100443A2000434C4F006D
:10703000434B2C00203143004C4F43004B2C20008D
:1070400030444100544120004F55540050555400E5
:107050002C2031004441540041204F005554500031
:1070600055542C00203020002A7069006E206900E1
:1070700073206E006F77200048695A00434C4F0020
:10708000434B2000544943004B533A0020524500E3
:1070900041442000424954003A205300796E740064
:1070A00061782000657272006F72200061742000A8
:1070B00063686100722078002E2065007869740092
:1070C0002877690074686F00757420006368610038
:1070D0006E676500296E6F00206D6F00646520008B
:1070E000636861006E6765004E6F6E0065786900C9
:1070F000737465006E74200070726F00746F6300AB
:107100006F6C2100782E200065786900740D0A00EC
:10711000496E7600616C690064206300686F6900E5
:1071200063652C002074720079206100676169003A
:107130006E444500564944003A68740074703A0041
:107140002F2F6400616E670065726F0075737000A9
:10715000726F74006F747900706573002E636F0036
:107160006D2A2D002D2D2D002D2D2D002D2D2D00C6
:107170002A4F7000656E200064726100696E200005
:107180006F7574007075740073202800483D4800C6
:10719000692D5A002C204C003D474E0044294E00DA
:1071A0006F726D00616C20006F75740070757400F3
:1071B00073202800483D33002E3376002C204C00ED
:1071C0003D474E0044294D00534220007365740032
:1071D0003A204D004F53540020736900672062002D
:1071E000697420006669720073744C005342200079
:1071F000736574003A204C004541530054207300DD
:107200006967200062697400206669007273740007
:1072100020426F006F746C006F6164006572200023
:10722000762031002E20480045580D000A203200FB
:107230002E20440045430D000A2033002E2042003A
:10724000494E0D000A2034002E20520041574400C0
:10725000697370006C61790020666F00726D610067
:1072600074207300657456006F6C7400616765006C
:10727000206D6F006E6974006F7273003A203500E4
:10728000563A2000207C2000332E3300563A20004E
:10729000207C2000565055004C4C5500503A2000A0
:1072A0005365740020736500726961006C20700082
:1072B0006F72740020737000656564003A202800C6
:1072C00062707300290D0A0020312E002033300037
:1072D000300D0A0020322E002031320030300D00F7
:1072E0000A2033002E203200343030000D0A2000F6
:1072F000342E200034383000300D0A0020352E00A6
:107300002039360030300D000A2036002E203100A2
:1073100039323000300D0A0020372E00203338007B
:10732000343030000D0A2000382E2000353736006A
:1073300030300D000A2039002E2031003135320066
:1073400030300D000A3130002E204200524720001C
:1073500072617700207661006C75650041646A0097
:107360007573740020796F00757220007465720067
:107370006D696E00616C410072652000796F750067
:107380002073750072653F002043460047313A0084
:107390002043460047323A00285C2D002F5F5C00F6
:1073A0002D2928005C5F2F002D295300656C650096
:1073B000637420006F757400707574002074790018
:1073C00070653A000D0A2000312E20004F706500D4
:1073D0006E206400726169006E202800483D4800FC
:1073E000692D5A002C204C003D474E0044290D00C9
:1073F0000A2032002E204E006F726D00616C20005A
:1074000028483D00332E3300562C20004C3D4700C9
:107410004E44290052325700202873007064200027
:1074200068697A00293D2800202030002E4D610037
:1074300063726F00206D65006E750D000A203100CB
:107440002E4953004F37380031362D00332041008C
:1074500054520D000A2032002E4953004F37380095
:1074600031362D00332070006172730065206F008B
:107470006E6C790049534F002037380031362D00AB
:1074800033204100545220002852450053455400F7
:10749000206F6E0020435300290D0A00524553000F
:1074A0004554200048494700482C2000434C4F00D9
:1074B000434B2000544943004B2C200052455300BD
:1074C000455420004C4F570049534F002037380097
:1074D00031362D003320720065706C007920280051
:1074E000757365007320630075727200656E7400B9
:1074F000204C53004220730065747400696E67006D
:10750000293A200050726F00746F63006F6C3A006C
:1075100020736500726961006C3320007769720026
:1075200065322000776972006552460055756E001D
:107530006B6E6F00776E5200656164002074790095
:1075400070653A0020746F0020656E0064766100FB
:1075500072696100626C6500206C65006E67740082
:107560006844610074612000756E690074733A00AC
:10757000206E6F0020696E006469630061746900A9
:107580006F6E44006174610020756E0069742000A4
:107590006C656E006774680020286200697473006F
:1075A000293A200043532000454E4100424C4500FB
:1075B0004443530020444900534142004C45440099
:1075C00052335700202873007064200063736C00EE
:1075D000206869007A293D00282029000D0A44000E
:1075E000697363006F6E6E006563740020616E00E6
:1075F0007920640065766900636573000D0A4300B5
:107600006F6E6E0065637400202856007075200050
:10761000746F20002B355600292061006E64200015
:1076200028414400432074006F202B00332E330088
:107630005629430074726C00415558004D4F440068
:1076400045204C0045445000554C4C0055502000FE
:10765000485055004C4C55005020480056524500AB
:1076600047414400432061006E6420007375700040
:10767000706C790035565600505533002E33560045
:107680004144430042757300206869006768420006
:107690007573200048692D005A2030004275730030
:1076A000204869002D5A2000314D4F0044452000EC
:1076B000616E640020565200454720004C4544004E
:1076C00073207300686F75006C6420006265200091
:1076D0006F6E2100466F75006E6420002065720099
:1076E000726F7200732E4D004F534900434C4B0094
:1076F0004D4953004F435300204F4B00204641005B
:10770000494C5300657420007370650065643A004D
:107710000D0A2000312E200033304B00487A0D0036
:107720000A2032002E20310032354B00487A0D00FD
:107730000A2033002E20320035304B00487A0D00ED
:107740000A2034002E2031004D487A00436C6F002F
:10775000636B2000706F6C006172690074793A008D
:107760000D0A2000312E200049646C0065206C0059
:107770006F7720002A646500666175006C740D00E7
:107780000A2032002E204900646C650020686900E0
:1077900067684F007574700075742000636C6F002B
:1077A000636B200065646700653A0D000A203100B4
:1077B0002E204900646C650020746F002061630016
:1077C00074697600650D0A0020322E0020416300A6
:1077D00074697600652074006F206900646C650030
:1077E000202A640065666100756C7400496E700043
:1077F0007574200073616D00706C65002070680006
:10780000617365003A0D0A0020312E00204D690099
:1078100064646C0065202A006465660061756C0014
:10782000740D0A0020322E0020456E006453500073
:10783000492028007370640020636B00702073007F
:107840006B652000736D7000206373006C2068000E
:10785000697A29003D28200020302E004D61630008
:10786000726F20006D656E00750D0A0020312E00CC
:10787000536E690066662000435320006C6F7700EA
:107880000D0A2000322E53006E69660066206100EA
:107890006C6C20007472610066666900632D700074
:1078A000202D6600202A4200797465007320640050
:1078B000726F7000706564002A464100494C4500B3
:1078C000442C20004E4F20004441540041446100AC
:1078D0007461200062697400732061006E6420008E
:1078E00070617200697479003A0D0A0020312E002F
:1078F00020382C00204E4F004E4520002A646500A1
:10790000666175006C7420000D0A2000322E200084
:10791000382C2000455645004E200D000A2033002B
:107920002E2038002C204F00444420000D0A200057
:10793000342E2000392C20004E4F4E004553740049
:107940006F70200062697400733A0D000A203100E4
:107950002E203100202A640065666100756C740079
:107960000D0A2000322E2000325265006365690046
:1079700076652000706F6C006172690074793A005E
:107980000D0A2000312E200049646C006520310072
:10799000202A640065666100756C74000D0A200081
:1079A000322E200049646C006520300055415200A1
:1079B0005420280073706400206272006720640005
:1079C0006270200073622000727870002068690085
:1079D0007A293D0028202000302E4D00616372007E
:1079E0006F206D00656E75000D0A2000312E540069
:1079F00072616E007370610072656E0074206200C7
:107A00007269640067650D000A2032002E204C0068
:107A100069766500206D6F006E6974006F720D00ED
:107A20000A2033002E4272006964670065207700E7
:107A30006974680020666C006F772000636F6E00C9
:107A400074726F006C5541005254200062726900DC
:107A5000646765005265730065742000746F2000D0
:107A600065786900745261007720550041525400D6
:107A700020696E00707574005541520054204C000E
:107A8000495645002044490053504C0041592C00B0
:107A9000207D2000544F200053544F00504C49008B
:107AA0005645200044495300504C41005920530092
:107AB000544F500050454400574152004E494E002B
:107AC000473A200070696E0073206E006F742000CA
:107AD0006F7065006E206400726169006E2028007E
:107AE00048695A002920520045564900443A0D0081
:107AF0000A496E0076616C006964200063686F005B
:107B0000696365002C207400727920006167610050
:107B1000696E6D0073525300204C4F00572C2000AB
:107B2000434F4D004D414E0044204D004F44450011
:107B30005253200048494700482C2000444154003B
:107B400041204D004F44450041646400726573005C
:107B500073206F00662050004346380035373400EC
:107B60003F546800697320006D6F640065207200E7
:107B70006571750069726500732061006E20610097
:107B800064617000746572004C4344002074790095
:107B900070653A000D0A2000312E20004844340060
:107BA0003437380030202800757369006E67200074
:107BB0005043460038353700342049004F206500D7
:107BC000787061006E64650072294C0043442000A7
:107BD00028747900702061006464720029203D00DF
:107BE0002028200020302E004D616300726F20009D
:107BF0006D656E00750D0A0020312E004C43440067
:107C000020526500736574000D0A2000322E490071
:107C10006E697400204C4300440D0A0020332E008E
:107C2000436C6500617220004C4344000D0A200043
:107C3000342E4300757273006F722000706F7300F2
:107C4000697469006F6E200065783A002834290055
:107C500020300D000A2036002E577200697465002E
:107C600020746500737420006E756D00626572008B
:107C700073206500783A28003629200038300D003E
:107C80000A2037002E577200697465002074650061
:107C90007374200063686100726163007465720030
:107CA00073206500783A28003729200038304400D6
:107CB000697370006C617900206C69006E657300F7
:107CC0003A0D0A0020312E00203120000D0A20003C
:107CD000322E20004D756C00746970006C6549008F
:107CE0004E495400434C4500415243005552530005
:107CF0004F522000534554004E6F200041434B002B
:107D00002C206300686563006B2061006461700073
:107D100074657200434C4B00094D4F0053490900F4
:107D2000435309004D4953004F5069006E7374006E
:107D300061746500733A47004E440900332E3300E6
:107D4000560935002E3056000941440043095600BB
:107D5000505509004155580009500900500950007C
:107D60000949090049092D00094F570044092D0010
:107D7000092D2D000954780044092D00095278007E
:107D8000445343004C095300444109002D092D0080
:107D9000504743000950470044092D00092D310088
:107DA0002E28420052290900322E28005244290070
:107DB00009332E00284F5200290934002E2859007B
:107DC00057290900352E2800474E290009362E0074
:107DD00028424C00290937002E2850005529090057
:107DE000382E28004752290009392E002857540000
:107DF000290930002E2842006C6B2900474E4400B0
:107E000009474E004409410044430900352E300023
:107E1000560933002E3356000956500055094100CB
:107E200055580900657865006375740065203A004F
:107E300020205400494D45004F55540020302E005D
:107E4000204D610063726F00206D65006E750D003E
:107E50000A2031002E204C006976650020696E00F2
:107E600070757400206D6F006E6974006F72490048
:107E70006E70750074206D006F6E6900746F720013
:107E8000202A7300746172007462690074206500B6
:107E900072726F0072202A0070617200697479003A
:107EA00020657200726F7200202A7300746F700078
:107EB0006269740020657200726F7200204E4F007C
:107EC0004E452000554E4B004E4F57004E2045006A
:107ED00052524F005220610075746F0072616E0043
:107EE000676520002B4D48007A292B006B487A00EB
:107EF0002952610077207600616C7500652066006C
:107F00006F7220004252470020284D00494449002A
:107F10003D3132003729570041524E00494E47004B
:107F20003A2050006F73730069626C006520620034
:107F30007566660065726F0076657200666C6F002C
:107F400077416E0079206B0065792000746F200006
:107F500065786900745370006163650020746F0078
:107F600020636F006E7469006E7565004E756D005C
:107F700062657200206F66002062690074732000E1
:107F800072656100642F770072697400653A2000A1
:107F900043533A000D0A2000312E200043530D00B8
:107FA0000A2032002E202F00435320002A6465004F
:107FB000666175006C744700656E650072616C00E7
:107FC0000909090009095000726F74006F636F009E
:107FD0006C2069006E7465007261630074696F00E3
:107FE0006E2D2D002D2D2D002D2D2D002D2D2D0034
:107FF0002D2D2D002D2D2D002D2D2D002D2D2D0065
:108000002D2D2D002D2D2D002D2D2D002D2D2D0054
:108010002D2D2D002D2D2D002D2D2D002D2D2D0044
:108020002D2D2D002D2D2D002D2D2D002D2D2D0034
:108030002D2D2D002D2D2D002D2D2D002D2D2D0024
:108040002D2D2D002D3F0900546869007320680014
:10805000656C70000909090028302900094C690085
:10806000737420006375720072656E0074206D0079
:10807000616372006F733D00582F7C005809430004
:108080006F6E760065727400732058002F72650061
:108090007665720073652000580909002878290068
:1080A000094D610063726F0020787E0009536500FE
:1080B0006C66740065737400090909005B0953005C
:1080C00074617200742309005265730065740900BD
:1080D000090909005D095300746F700024094A0002
:1080E000756D700020746F0020626F006F746C00FB
:1080F0006F61640065720900097B090053746100B7
:1081000072742000776974006820720065616400F1
:10811000262F2500094465006C617900203120007C
:1081200075732F006D73090009097D0009537400F0
:108130006F7061002F412F004009410055585000D9
:10814000494E2000286C6F00772F4800492F5200BD
:1081500045414400290909002261620063220900A7
:1081600053656E0064207300747269006E6762006C
:1081700009536500742062006175640072617400C7
:10818000650909000931320033632F0043094100BA
:10819000555820006173730069676E006D656E004D
:1081A00074202800617578002F43530029090900C5
:1081B00030783100323364002F4409004D6561008E
:1081C000737572006520410044432000286F6E00E3
:1081D00063652F00434F4E00542E29000930620082
:1081E00031313000095365006E64200076616C0007
:1081F00075656600094D6500617375007265200044
:1082000066726500717565006E6379000909720018
:108210000952650061646700094765006E65720078
:10822000617465002066720065717500656E63009B
:10823000792F5000574D0900092F0900434C4B007E
:1082400020686900680943006F6D6D00616E64000D
:1082500068697300746F720079090900095C09008C
:10826000434C4B00206C6F00690956006572730027
:10827000696F6E00696E66006F2F73007461740021
:10828000757369006E666F0009095E0009434C0052
:108290004B20740069636B006C2F4C00094269002D
:1082A000746F72006465720020286D0073622F0085
:1082B0004C534200290909002D0944004154200073
:1082C00068696D0009436800616E670065206D0094
:1082D0006F646500090909005F09440041542000EA
:1082E0006C6F6F000953650074206F007574700027
:1082F000757420007479700065090900092E090061
:108300004441540020726500616470002F500900E0
:1083100050756C006C757000207265007369730095
:10832000746F7200732028006F6666002F4F4E0036
:108330002909210009426900742072006561640006
:10834000730953006372690070742000656E6700E2
:10835000696E6500090909003A09520065706500F7
:1083600061742000652E67002E2072003A313000C3
:1083700076095300686F770020766F006C74730085
:108380002F73740061746500730909003B09420092
:108390006974730020746F002072650061642F009F
:1083A0007772690074652000652E67002E2030000A
:1083B000783535003B3277002F5709005053550070
:1083C00020286F0066662F004F4E290009093C00E7
:1083D000783E2F003C783D00203E2F003C303E0090
:1083E0000955730065726D00616372006F2078003B
:1083F0002F617300736967006E2078002F6C69002D
:1084000073742000616C6C000000FA0080B92000D9
:10841000104078000030A00081B92000804878002A
:1084200080B9200010407800704060000004E00037
:1084300002003200CAC2A90001003700CAC2A80067
:1084400080B9200010407800704060000004E00017
:1084500003003200F0C2B3000C7102000000000003
:10846000A100200060AB20004E9A02000000000036
:108470000080FA00000006000000FA0080B9200029
:10848000104078000030A10081B9200080487800B9
:1084900080B9200010407800704060000004E000C7
:1084A00002003200CAC2A90001003700CAC2A800F7
:1084B00080B9200010407800704060000004E000A7
:1084C00003003200F0C2B3000C7102000000000093
:1084D000A100200060AB20004E9A020000000000C6
:1084E0000080FA00000006000000FA0080B92000B9
:1084F00010407800704060000004E000020032008C
:10850000CAC2A80001003700CAC2A90080B9200071
:1085100010407800704060000004E000030032006A
:10852000F0C2B3000C71020000000000B100200096
:1085300000AC20004E9A0200000000000080FA000B
:10854000000006000000FA0000C0EB002702070050
:108550000080FB000080FA00000006000600FA0020
:10856000100798001E00900020020700004F7800BE
:1085700080B9200010407800684060000004E000EE
:10858000030032001E80FB00200798000200370025
:1085900000102000200798002E0090000080FA00B4
:1085A000000006000000FA0001022000D0C92000EF
:1085B000C49902000000000060B72000104078005D
:1085C000486F02000000000000C2B3000C710200FE
:1085D0000000000080B92000104078006140600079
:1085E000486F02000000000000C2B3000C710200DE
:1085F0000000000080B92000104078000080FB00DF
:108600000000D10061406000486F020000000000DF
:1086100000C2B3000C7102000000000080B920000D
:10862000104078000080FB004200DE0061406000E6
:10863000486F02000000000000C2B3000C7102008D
:108640000000000080B92000104078000080FB008E
:108650004400DE0061406000486F0200000000003E
:1086600000C2B3000C7102000000000070B72000CF
:10867000104078000080FB004300DE006140600095
:10868000486F02000000000000C2B3000C7102003D
:108690000000000031002000F0AD2000C49902006D
:1086A000000000000080FA00000006000C00FA0044
:1086B0001A1A020000000000441602000000000028
:1086C000500798001A1A0200000000004416020029
:1086D00000000000400798001A1A02000000000085
:1086E0004416020000000000300798001A1A020029
:1086F000000000004416020000000000200798005F
:108700001A1A0200000000004416020000000000D7
:10871000000F78001A1A0200000000004416020040
:1087200000000000100798005E0090000000E000CC
:10873000090034005E009000E40F500006003C0089
:108740005E0090000040E9008040780060B72000A3
:1087500001487800020037000000EB005007980045
:108760004E0090000000E0000F0034004E0090002A
:10877000E20F50000C003C004E0090000040E90069
:10878000E140600080B920001040780061C16000C5
:10879000E1CFB300014060000240700081B92000C9
:1087A00080487800020037000000EB005007980076
:1087B0003E0090000000E000100034003E009000F9
:1087C000E20F50000D003C003E0090000040E90028
:1087D0006141600080B920009040780061406100F4
:1087E00000414000D0CFB30080C0600082C0700064
:1087F00080B9200001487800020037000000EB003B
:10880000500798002E0090000000E0001000340097
:108810002E009000E20F50000D003C002E00900052
:108820000040E9006141600080B92000904078007C
:10883000614061004201DD00B0CFB30080C0600044
:1088400082C0700080B92000014878000200370023
:108850000000EB00500798001E00E00010003400FC
:10886000200020009E0F10000D003C001E0078002C
:108870000040E9006141600080B92000904078002C
:10888000614061004401DD00F0CEB30080C06000B3
:1088900082C0700080B920000148780002003700D3
:1088A0000000EB00500798001E0090000000E00060
:1088B000100034001E009000E20F50000D003C003C
:1088C0001E0090000040EA006141600070B7200087
:1088D00090407800614061004301DD0070CFB3003B
:1088E00080C0600082C0700070B72000014878002E
:1088F000020037000000EB00500798005E00900077
:108900000000E00079003A000000EB006069880098
:1089100071032000D0BB20004E9A0200000000002E
:108920008001EB0042002000110020001000200018
:10893000901C0200000000000040E9008040780028
:1089400060B72000014878005103200040BF20009C
:108950004E9A0200000000008001EB00220020007F
:108960001100200010002000901C020000000000F8
:108970000040E900E140600080B92000104078002C
:1089800061C16000E1CFB3000140600002407000AF
:1089900081B92000804878003104200090C2200076
:1089A0004E9A0200000000008001EB00220020002F
:1089B0001100200020002000901C02000000000098
:1089C0000040E9006141600080B9200090407800DB
:1089D0006140610000414000D0CFB30080C0600022
:1089E00082C0700080B92000014878001103200087
:1089F000C0C620004E9A0200000000008001EB007B
:108A0000220020001100200010002000901C020015
:108A1000000000000040E9006141600080B92000D2
:108A200090407800614061004201DD00B0CFB300AA
:108A300080C0600082C0700080B9200001487800CA
:108A4000D1012000702221004E9A02000000000097
:108A50008001EB00220020001100200020002000F7
:108A6000901C0200000000000040E900614160002D
:108A700080B9200090407800614061004401DD0031
:108A8000F0CEB30080C0600082C0700080B92000CA
:108A900001487800F1042000B09320004E9A0200B3
:108AA000000000008001EB002200200011002000E7
:108AB00010002000901C0200000000000040EA00AE
:108AC0006141600070B72000904078006140610013
:108AD0004301DD0070CFB30080C0600082C0700031
:108AE00070B720000148780001003700ADFE070094
:108AF00080B92000104078000030A10081B920002A
:108B00008048780060B72000104078008080FB002B
:108B1000E081200000804000104078004B000700FA
:108B200080B92000104078000080FB004400DE0087
:108B300061406000614060004601DD00A12C200022
:108B400091407800F0CBB30000C06000024070009C
:108B5000CAE2B7000080FA00000006000000FA0038
:108B60008E0007000080FA00000006000400FA00F2
:108B7000000F78001E007800100798001E0090007B
:108B8000E10F50000C0032001E009000E10F500079
:108B9000040039001E009000E20F50001200320065
:108BA0001D00370041032000D0CB20004E9A020068
:108BB000000000001C003700710020005059200008
:108BC0004E9A020000000000F1002000C01E2100AB
:108BD0004E9A02000000000011C0B30010C0B300A4
:108BE000900007001000370071002000505920004D
:108BF0004E9A020000000000F1002000C01E21007B
:108C00004E9A02000000000011C0B3000040EB00CB
:108C1000840007000400370041022000C02020002B
:108C20004E9A0200000000000080FA0000000600DA
:108C30000000FA0001012000A00421004E9A020069
:108C4000000000000080FA00000006000200FA00A8
:108C5000004F780041E2A90070B720001040780072
:108C6000684060000004E00004003200CEE2A8008A
:108C7000CF02A800CEC2A80003003700CEE2A900B0
:108C8000CF02A900CEC2A900816A200091407800DD
:108C900000CEB30000C060007040B300A8E6B7008B
:108CA000916C20009140780000CEB30000C06000BD
:108CB0007040B300C9E6B700816C20009140780095
:108CC00000CEB30000C060000034A000C8E6B700CA
:108CD000CAC2A800C8C2A900C902A900C8E2A80067
:108CE000C922A9001E80FB001012880042A2A80021
:108CF00080B9200010407800614060006140600051
:108D00004601DD002124200091407800F0CBB30023
:108D100000C060000240700042E2B70080B920004D
:108D2000104078000080FB000000D100614060002E
:108D3000614160003124200091407800E0CFB30011
:108D400000C060000240700043E2B70080B920001C
:108D5000104078000080FB004200DE0061406000AF
:108D600061406000004140003124200091407800C3
:108D7000D0CFB30000C060000240700043E2B700F3
:108D80000000EB00201288000000EB0000128800B9
:108D900041E2A8000080FA00000006000000FA008E
:108DA00041E2A900A8C6BF00F041B300A8E6B700A1
:108DB000916C20009140780000CEB30000C06000AC
:108DC000C9E6B700816C20009140780000CEB30066
:108DD00000C06000C8E6B700CEE2A900CF02A9003B
:108DE000CEC2A9000080FA00000006000200FA00CE
:108DF000004F78001E80FB004012880085C0BF0035
:108E0000644060000004E000FCFF3200401280007B
:108E1000004F78008540A9001E80FB000080FA000A
:108E2000000006000400FA0020479800314798002F
:108E300010C0B300004F7800B471020000000000C1
:108E4000D6FF07007B0007002E4090000004E000E2
:108E500002003A0042E2A80062E2A8002E40900020
:108E6000E14F500003003E0041E2A80061E2A8008B
:108E7000000037001E04E00009003A00CAC2BF002B
:108E80000044B2000004E00005003200D0C5B30089
:108E9000C27102000000000010C0B300004F780053
:108EA00040C2BF000042B2000004E0002F003A00C0
:108EB00060C2BF000042B2000004E0002B003A0094
:108EC000401280001047980010C0B3009E4F100061
:108ED00005003A00B0C5B300C271020000000000F6
:108EE0000040EB00004F78003E4090000004E0009E
:108EF000050032001E4090000080FB00D46F02008D
:108F00000000000006003700C0C5B300C2710200B7
:108F1000000000001E409000C2710200000000002E
:108F200040138000104798003E4090000004E0008D
:108F30000B00320080C2B300C271020000000000CA
:108F40001E4090000080FB00D46F02000000000073
:108F500090C2B300C271020000000000030037009D
:108F60001E409000C27102000000000040C2BF001D
:108F70000044B2000004E00004003A0060C2BF00F8
:108F80000044B2000004E0000A003200CA82A900D6
:108F90003E4090000004E00003003200809F280063
:108FA000DC6C02000000000040C2A90060C2A90001
:108FB00013003700F27102000000000022C2BF005F
:108FC000614060000004E000AAFF3200311180001F
:108FD00020072000808F500003003A0041E2A900E2
:108FE00061E2A900A3FF37003E4090000004E000CA
:108FF0000300320090A02800DC6C0200000000009A
:109000008B00070081C6BF00F041B30081E6B700C6
:1090100060B72000104078008080FB00E0812000D5
:10902000008040001040780008FF07000080FA0030
:10903000000006000000FA00C8C2A800C902A8008B
:10904000C8E2A800C922A800A16A200091407800C7
:1090500000CEB30000C060006040B300AAE6B700D5
:10906000E16A20009140780000CEB30000C06000AB
:109070006040B300AEE6B700816A200091407800FE
:1090800000CEB30000C060009040B300A8E6B70077
:10909000916A20009140780000CEB30000C06000CB
:1090A0000034A000A9E6B700C16A20009140780012
:1090B00000CEB30000C060007040B300ACE6B70063
:1090C000D16A20009140780000CEB30000C060005B
:1090D0000034A000ADE6B70060B720001040780073
:1090E0008080FB00E081200000804000104078007C
:1090F0000080FB001012880080B92000104078002A
:1091000061406000614060004601DD0021242000D4
:1091100091407800F0CBB30000C0600002407000C6
:1091200042E2B70080B92000104078000080FB00C8
:109130000000D100614060006141600031242000E6
:1091400091407800E0CFB30000C0600002407000A2
:1091500043E2B7000000EB00201288000000EB00A3
:109160000012880060B72000104078008080FB006B
:10917000E081200000804000104078000080FB006B
:109180001013880080B92000104078006140600012
:10919000614060004601DD002126200091407800FA
:1091A000F0CBB30000C060000240700062E2B70084
:1091B00080B92000104078000080FB000000D10042
:1091C00061406000614160003126200091407800DC
:1091D000E0CFB30000C060000240700063E2B7005F
:1091E0000000EB00201388000000EB000013880053
:1091F0000000EB00401288000000EB0040138800E4
:109200004322A9006322A9004362A80042A2A90048
:109210006362A80062A2A90040C2A90060C2A900BE
:109220004402A8006402A8000080FA0000000600C2
:109230000000FA0041E2A9004362A90061E2A9002E
:109240006362A900AAC6BF00F041B300AAE6B70056
:10925000AEC6BF00F041B300AEE6B700A8C6BF007F
:10926000F041B300A8E6B700A9C6BF00F041B300C3
:10927000A9E6B700ACC6BF00F041B300ACE6B7004A
:10928000ADC6BF00F041B300ADE6B7000080FA0004
:10929000000006000000FA00A0A02800B06C020048
:1092A000000000000080FA00000006000A00FA003A
:1092B000881F780011C0B30060B720000148780013
:1092C00080B92000104078000000A10081B9200082
:1092D0008048780080B92000104078000010A0007D
:1092E00081B920008048780080B9200010407800C3
:1092F0000020A10081B920008048780070B72000CC
:10930000104078000030A00071B72000804878003D
:1093100060B72000104078008080FB002082200091
:10932000008040001040780048FE0700D9FF070089
:109330000000370022C2BF00614060000004E0006E
:10934000FCFF3200301180008040780060B92000BE
:109350000148780060B92000104078000080FB00D0
:109360004400DE008040780050B9200001487800B9
:1093700050B92000104078000080FB0040079800A2
:109380004E009000E40F5000FA0032004E009000B2
:10939000E40F500007003C004E0090000000E00089
:1093A0000B0032004E009000E10F5000CB00320065
:1093B0005C0137004E009000E60F5000F5003200CF
:1093C0004E009000E80F50000701320055013700B1
:1093D00060B92000104078000080FB003007980042
:1093E0003E009000E30F50002A0032003E00900043
:1093F000E30F50000A003C003E009000E10F5000D7
:109400001A0032003E009000E10F500019003C00AD
:109410003E0090000000E00012003200AB00370078
:109420003E009000ED0F5000220032003E00900000
:10943000ED0F500004003C003E009000E40F50008F
:1094400031003200A10037003E009000EE0F5000C6
:109450001F0032003E009000EF0F5000230032004A
:109460009A0037004DFE07003201370089FF0700E0
:10947000B0FF370060168000F1FB2F000100600094
:109480006016880010C0B3000C71020000000000DC
:10949000A8FF370060168000010420000100700062
:1094A0006016880010C0B3000C71020000000000BC
:1094B000A0FF37008040EB0020C0B30059FE07003A
:1094C00010C0B3000C7102000000000099FF3700CB
:1094D0008040EB000040EB0052FE070010C0B300DC
:1094E0000C7102000000000092FF37008040EB008A
:1094F00010C0B3004BFE070010C0B3000C71020097
:10950000000000008BFF370022C2BF0061406000F6
:109510000004E000FCFF32003011800010079800CA
:109520001E0090004800DD001007980022C2BF0016
:10953000614060000004E000FCFF32003011800058
:109540009E009000008070001007980022C2BF00AB
:10955000614060000004E000FCFF32003011800038
:10956000000F78001E0078004800DD00000F780032
:1095700022C2BF00614060000004E000FCFF320036
:10958000301180001E0F70009E009000F0FF200040
:10959000808F500003003E00F0FF20009E0F10005F
:1095A000040036000040EB000C71020000000000D7
:1095B00060FF37000000EB00200798000C00370028
:1095C00022C2BF00614060000004E000FCFF3200E6
:1095D000714080002E00900080804000301180009B
:1095E000804878002E0090000000E80020079800D6
:1095F000AE0090001E009000808F5000F0FF3900F8
:10960000CAC2A9000000EB0020079800080037003C
:10961000714080002E0090000080400010407800D3
:10962000F2FD07002E0090000000E80020079800DF
:10963000AE0090001E009000808F5000F4FF3900B3
:109640000000EB00200798000900370071408000FF
:109650002E0090000084400000C0EB00E3FD0700F6
:10966000004C78002E0090000000E80020079800D1
:109670002E0090009E0F5000F4FF3900CAC2A800CF
:1096800010C0B3000C710200000000000000EB00ED
:109690002007980009003700714080002E009000DC
:1096A00000804000104078000C71020000000000B3
:1096B0002E0090000000E800200798002E00900087
:1096C0009E0F5000F4FF39001AFF37000040EB00F6
:1096D0000C7102000000000016FF370060B9200086
:1096E00090407800F0C0B30080C0600060B92000F6
:1096F0000148780060B92000104078008040E80000
:1097000060B920000148780010C0B3000C7102005D
:10971000000000008040EB0040B9200001487800C4
:109720000D00370022C2BF00614060000004E0006D
:10973000FCFF320030118000ACFD07000C7102000C
:109740000000000040B92000104078008040E80090
:1097500040B920000148780040B9200090407800CE
:1097600060B920001040780080CF5000EDFF390034
:10977000F0FE370060B9200010407800A69C02007F
:109780000000000010C0B3000C71020000000000D7
:10979000E8FE370060B920009040780070C0B30048
:1097A00080C0600060B920000148780060B92000E6
:1097B0009040780060B720000148780060B7200032
:1097C000104078008080FB00208220000080400054
:1097D000104078001DFD070010C0B3000C7102009E
:1097E00000000000D3FE370080B920001040780050
:1097F0000000A10081B920008048780080B92000D5
:10980000104078000010A10081B920008048780045
:1098100080B92000104078000020A10081B920000C
:109820008048780070B72000104078000030A10018
:1098300071B720008048780060B92000104078009F
:109840000080FB004200DE00610060000004E000D8
:109850000500320080B92000104078000000A00010
:1098600081B920008048780060B92000104078005D
:109870000080FB000000D100610060000004E000F7
:109880000500320080B92000104078000010A000D0
:1098900081B920008048780060B92000104078002D
:1098A0000080FB00610060000004E0000500320061
:1098B00080B92000104078000020A00081B920006D
:1098C0008048780060B92000104078000080FB00DC
:1098D0004300DE000000A200610060000004E00020
:1098E0000500320070B72000104078000030A00062
:1098F00071B720008048780060B7200010407800E1
:109900008080FB0020822000008040001040780012
:10991000CEFC070010C0B3000C7102000000000074
:1099200084FE37000040EB000C71020000000000D4
:1099300080FE37004F0478000080FA000000060027
:109940000400FA00049C0200000000000004E00093
:109950002200320032C2BF00684060000004E00014
:10996000040032003100200010CF2000C499020012
:109970000000000032C2BF00644060000004E0004C
:10998000040032003100200040CF2000C4990200C2
:1099900000000000F29B020000000000004F780071
:1099A00032C2BF00624060000004E00008003200E4
:1099B000F100200070CF2000C499020000000000D8
:1099C00090118000D1FF2F000100600090118800ED
:1099D0001E80FB001007980006003700F1002000F1
:1099E00060D02000C4990200000000000000EB00DD
:1099F000100798001E0090000080FA00000006008A
:109A00000200FA00000F78001E007800DE9B0200C2
:109A100000000000001020000080FA000000060096
:109A20000000FA0001022000C0DB2000C4990200FF
:109A30000000000060B7200010407800486F02006E
:109A40000000000000C2B3000C7102000000000022
:109A500060B7200010407800E94F500007003A003E
:109A6000C0118000EA6E02000000000000C2B300D6
:109A70000C710200000000000C00370060B72000ED
:109A8000104078000080FB0080004000A0B0200063
:109A90000080400010007800EA6E02000000000024
:109AA00000C2B3000C71020000000000A0DD200025
:109AB0001040780063406000486F02000000000022
:109AC00000C2B3000C71020000000000A0DD200005
:109AD000104078000080FB004200DE006140600022
:109AE000486F02000000000000C2B3000C710200C9
:109AF00000000000A0DD2000104078000080FB0086
:109B00004300DE0061406000486F0200000000007A
:109B100000C2B3000C7102000000000070B720000A
:109B2000104078000080FB004300DE0061406000D0
:109B3000486F02000000000000C2B3000C71020078
:109B40000000000031002000F0AD2000C4990200A8
:109B5000000000000080FA00000006000C00FA007F
:109B60001A1A020000000000441602000000000063
:109B7000500798005E009000EA0F500005003A0080
:109B80001A1A020000000000441602000000000043
:109B9000000F78001A1A02000000000044160200AC
:109BA00000000000400798001A1A020000000000A0
:109BB0004416020000000000300798001A1A020044
:109BC000000000004416020000000000200798007A
:109BD0001A1A0200000000004416020000000000F3
:109BE000100798005E0090000000E00009003400BB
:109BF0005E009000EA0F500006003C005E009000FE
:109C00000040E9008040780060B7200001487800FB
:109C1000020037000000EB00500798004E00900053
:109C20000000E0000F0034004E009000E40F5000F0
:109C30000C003C004E0090000040E900E340600052
:109C4000A0DD20001040780063C16000C1CFB300E8
:109C50000140600002407000A1DD200080487800D3
:109C6000020037000000EB00500798003E00900013
:109C70000000E000100034003E009000E20F5000B1
:109C80000D003C003E0090000040E9006141600092
:109C9000A0DD200090407800614061004201DD00BD
:109CA000B0CFB30080C0600082C07000A0DD200093
:109CB00001487800020037000000EB0050079800D0
:109CC0002E0090000000E000100034002E009000F4
:109CD000E20F50000D003C002E0090000040E90013
:109CE00061416000A0DD200090407800614061008B
:109CF0004301DD0070CFB30080C0600082C07000FF
:109D0000A0DD200001487800020037000000EB00D1
:109D1000500798001E0090000000E0001000340082
:109D20001E009000E20F50000D003C001E0090004D
:109D30000040EA006141600070B720009040780068
:109D4000614061004301DD0070CFB30080C060005E
:109D500082C0700070B72000014878000200370010
:109D60000000EB00500798005E0090000000E0004B
:109D700073003A000000EB0060698800D108200001
:109D8000308720004E9A0200000000008001EB00A6
:109D9000A20020001100200010002000901C0200F2
:109DA000000000000040E9008040780060B720001B
:109DB0000148780060B7200010407800E94F50005B
:109DC0000B003A00C1012000001B21004E9A020046
:109DD000000000008001EB00F2FF270011002000CE
:109DE00020022000901C020000000000000F7800FC
:109DF0004105200050D12000C4990200000000005D
:109E00008001EB0042002000110020001000200023
:109E1000901C0200000000000040E900E3406000E8
:109E2000A0DD20001040780063C16000C1CFB30006
:109E30000140600002407000A1DD200080487800F1
:109E40001102200090D62000C499020000000000FA
:109E50008001EB00220020001100200010002000F3
:109E6000901C0200000000000040E9006141600019
:109E7000A0DD200090407800614061004201DD00DB
:109E8000B0CFB30080C0600082C07000A0DD2000B1
:109E90000148780021032000A0D82000C4990200C6
:109EA000000000008001EB002200200011002000D3
:109EB00010002000901C0200000000000040E9009B
:109EC00061416000A0DD20009040780061406100A9
:109ED0004301DD0070CFB30080C0600082C070001D
:109EE000A0DD200001487800F1042000B09320009C
:109EF0004E9A0200000000008001EB0022002000CA
:109F00001100200010002000901C02000000000042
:109F10000040EA006141600070B720009040780086
:109F2000614061004301DD0070CFB30080C060007C
:109F300082C0700070B7200001487800010037002F
:109F4000B7FE070060B7200010407800E94F5000CE
:109F50001C003A00A0DD2000104078000080FB00CB
:109F60004200DE006140600080417800A0DD2000FA
:109F7000104078006340600080427800A0DD20003F
:109F8000104078000080FB004300DE00614060006C
:109F90000041780070B72000104078000080FB007E
:109FA0004300DE0061406000804078001E007800C1
:109FB0000342780085417800329B020000000000D7
:109FC00022003700A0DD2000104078000080FB0058
:109FD0004200DE006140600000417800A0DD20000A
:109FE000104078006340600080417800A0DD2000D0
:109FF000104078000080FB004300DE0061406000FC
:10A000008042780070B72000104078000080FB008C
:10A010004300DE00614060000043780060B720002C
:10A02000104078000080FB0080004000A0B02000BD
:10A03000008040001000780002427800054178005E
:10A0400086407800329B020000000000B69B0200B0
:10A0500000000000C111800040118000808F50007E
:10A060000400310001022000C01C21004E9A0200B1
:10A07000000000000080FA00000006000000FA0066
:10A08000C29B0200000000000080FA0000000600F1
:10A090000400FA00000F78001E00780010079800F6
:10A0A0001E009000E10F50000C0032001E009000D6
:10A0B000E10F5000040039001E009000E20F500034
:10A0C0003D0032005900370031052000C0DD20007E
:10A0D000C49902000000000058003700B1002000C1
:10A0E000F0E220004E9A020000000000D1002000A3
:10A0F000A0E320004E9A020000000000F49A020043
:10A10000000000000000E0004C00320090118000D0
:10A11000D1FF2F000100600090118800000037007F
:10A1200032C2BF00614060000004E000060032005F
:10A1300023C2BF00624060000004E00002003A0059
:10A14000B01180002011880022C2BF006140600071
:10A150000004E0000600320033C2BF00624060002D
:10A160000004E00002003A0030118000A0118800D5
:10A1700032C2BF00624060000004E00004003A0008
:10A1800022C2BF00624060000004E000E4FF320031
:10A1900091118000D0FF2F00008060009011880096
:10A1A00011118000D0FF2F00008060001011880086
:10A1B000CA82A900DAFF3700E100200070E4200025
:10A1C0004E9A020000000000F1002000C01E210095
:10A1D0004E9A02000000000090118000D1FF2F0075
:10A1E000010060009011880032C2BF006140600031
:10A1F0000004E0000600320023C2BF00624060009D
:10A200000004E00002003A00B01180002011880034
:10A2100022C2BF00614060000004E000F2FF320093
:10A2200030118000000F7800040037004102200048
:10A23000C02020004E9A0200000000000080FA00BA
:10A24000000006000000FA0091118000D0FF2F00EE
:10A250000080600090118800A0DD20001040780090
:10A260000040A000A1DD20008048780070B72000E9
:10A27000104078000010A00071B7200080487800DE
:10A28000C101200050E520004E9A020000000000AD
:10A290000080FA00000006000000FA00A0DD2000A7
:10A2A000104078000040A100A1DD20008048780027
:10A2B00070B72000104078000010A10071B7200096
:10A2C000804878004101200010E720004E9A0200EB
:10A2D000000000000080FA00000006000200FA0002
:10A2E0000000EB00000F780035003700A0DD2000F3
:10A2F00010407800704060000004E0002C00320044
:10A3000080A32800DC6C0200000000006100200037
:10A3100060692000C49902000000000032C2BF0042
:10A32000684060000004E0000400320031002000BA
:10A3300010CF2000C49902000000000032C2BF000C
:10A34000644060000004E00004003200310020009E
:10A3500040CF2000C499020000000000F29B0200E0
:10A36000000000000080FB009C960200000000003E
:10A3700032C2BF00624060000004E000080032000A
:10A38000F100200070CF2000C499020000000000FE
:10A3900090118000D1FF2F00010060009011880013
:10A3A00080A32800DC6C02000000000002003700DF
:10A3B000F29B02000000000010002000000F780057
:10A3C000049C0200000000000004E000C7FF3A0007
:10A3D0001E0078000080FA00000006000000FA006D
:10A3E000B1002000100921004E9A02000000000078
:10A3F0000080FA00000006000000FA0090A3280088
:10A40000B06C0200000000000080FA0000000600AE
:10A410000400FA00A0DD2000104078000000A10038
:10A420000010A100A1DD200080487800A0DD200000
:10A43000104078000020A100A1DD200080487800B5
:10A44000A0DD2000104078000030A100A1DD200038
:10A450008048780070B72000104078000030A000DD
:10A4600071B7200080487800F0588000A06E880006
:10A47000A0DD2000104078000040A100A1DD2000F8
:10A4800080487800A0DD2000104078000080FB00AC
:10A490004200DE006140600080417800A0DD2000C5
:10A4A000104078006340600080427800A0DD20000A
:10A4B000104078000080FB004300DE006140600037
:10A4C0000041780070B72000104078000080FB0049
:10A4D0004300DE006140600080407800A06E800094
:10A4E0000342780085417800329B020000000000A2
:10A4F000B69B020000000000BFFF0700000037000D
:10A50000049C0200000000000004E0000C00320087
:10A51000A0DD200010407800704060000004E000E2
:10A5200005003200F29B0200000000000C710200E6
:10A530000000000002003700F29B02000000000053
:10A5400032C2BF00624060000004E000040032003C
:10A5500090118000D1FF2F00010060009011880051
:10A5600022C2BF00614060000004E000E4FF32004E
:10A57000301180008040780080DD200001487800A4
:10A5800080DD2000104078000080FB004400DE00E9
:10A590008040780070DD20000148780070DD2000E8
:10A5A000104078000080FB00100798001E0090000B
:10A5B000E40F5000D00032009E009000E48F500065
:10A5C00007003C001E0090000000E0000F00320079
:10A5D0009E009000E18F50009F0032008A013700FA
:10A5E0001E009000E60F5000CB0032009E0090004D
:10A5F000E68F5000840135009E0090006880500076
:10A60000E10F500080013E00FB00370080DD20009C
:10A61000104078000080FB00000F78001E007800DA
:10A62000E20F5000190032009E007800E28F5000C7
:10A6300007003C001E0078000000E0000E00320021
:10A640009E007800E18F50000E0032007E0037003F
:10A650001E007800E70F5000260032009E007800B0
:10A66000EF8F50005B0032001E007800E30F5000B7
:10A670001700320074003700C29B02000000000087
:10A68000650137005CFF07009DFF370010C0B30075
:10A690000C7102000000000032C2BF006240600086
:10A6A0000004E0000400320090118000D1FF2F0070
:10A6B0000100600090118800A0DD200010407800AB
:10A6C0000040A000A1DD2000804878008CFF37000A
:10A6D000A0DD2000104078000040A100A1DD200096
:10A6E0008048780010C0B3000C7102000000000028
:10A6F00083FF370010C0B3000C710200000000009F
:10A70000C29B02000000000022C2BF006140600046
:10A710000004E000FCFF3200301180004800DD0042
:10A72000A06E880010C0B3000C7102000000000091
:10A7300022C2BF00614060000004E000FCFF320064
:10A74000A16E80003011800000807000A06E880033
:10A75000A0DD2000104078000080FB004200DE00F9
:10A760006140600080417800A0DD2000104078004A
:10A770006340600080427800A0DD20001040780037
:10A780000080FB004300DE00614060000041780073
:10A7900070B72000104078000080FB004300DE000E
:10A7A0006140600080407800A06E80000342780025
:10A7B00085417800329B020000000000B69B020039
:10A7C0000000000010C0B3000C7102000000000087
:10A7D0004BFF370010C0B3000C71020000000000F6
:10A7E00090118000D1FF2F000100600090118800BF
:10A7F0000000370032C2BF00614060000004E0008A
:10A800000600320023C2BF00624060000004E00086
:10A8100002003A00B01180002011880022C2BF005F
:10A82000614060000004E000F2FF320033C2BF006C
:10A83000624060000004E000EEFF3A00301180004A
:10A84000A0118800EBFF37000040EB000C71020004
:10A85000000000002AFF370080DD200090407800D3
:10A86000F0C0B30080C0600080DD200001487800A7
:10A8700080DD2000104078008040E80080DD20006E
:10A880000148780010C0B3000C7102000000000005
:10A890008040EB0060DD2000014878000F003700A9
:10A8A00022C2BF00614060000004E000FCFF3200F3
:10A8B00030118000DE9B02000000000010C0B300D9
:10A8C0000C7102000000000060DD200010407800E4
:10A8D0008040E80060DD20000148780060DD200055
:10A8E0009040780080DD20001040780080CF50003C
:10A8F000EBFF390002FF370080DD200010407800B8
:10A90000A69C02000000000010C0B3000C71020001
:10A9100000000000FAFE370080DD20009040780043
:10A92000F0C0B30080C0600080DD200001487800E6
:10A9300080DD200010407800EA4F50000300360010
:10A94000A1C0B30080DD20000148780080DD200038
:10A95000104078000080FB0080004000E0B1200043
:10A960000080400010007800A06E8800C29B0200AA
:10A9700000000000A0DD2000104078000080FB00F7
:10A980004200DE006140600080417800A0DD2000D0
:10A99000104078006340600080427800A0DD200015
:10A9A000104078000080FB004300DE006140600042
:10A9B0000041780070B72000104078000080FB0054
:10A9C0004300DE006140600080407800A06E80009F
:10A9D0000342780085417800329B020000000000AD
:10A9E000B69B02000000000010C0B3000C71020012
:10A9F00000000000C2FE3700A0DD200010407800FB
:10AA00000000A1000010A100A1DD20008048780016
:10AA1000A0DD2000104078000020A100A1DD200072
:10AA200080487800A0DD2000104078000030A100B0
:10AA3000A1DD20008048780070B720001040780029
:10AA40000030A10071B720008048780080DD200030
:10AA5000104078000080FB004300DE0061006000D1
:10AA60000004E0000D003200A0DD2000104078005E
:10AA7000634060000014A000E3406000A0DD2000FF
:10AA80001040780063C16000C1CFB3000140600096
:10AA900002407000A1DD20008048780080DD2000A9
:10AAA000104078000080FB004200DE006100600082
:10AAB0000004E0000D003200A0DD2000104078000E
:10AAC000634060000004A000E3406000A0DD2000BF
:10AAD0001040780063C16000C1CFB3000140600046
:10AAE00002407000A1DD20008048780080DD200059
:10AAF000104078000080FB000000D1006100600081
:10AB00000004E00005003200A0DD200010407800C5
:10AB10000020A000A1DD20008048780080DD20001A
:10AB2000104078000080FB00610060000004E0003D
:10AB300005003200A0DD2000104078000030A000A9
:10AB4000A1DD20008048780080DD200010407800E2
:10AB50000080FB004400DE000000A20061006000F5
:10AB60000004E0000500320070B7200010407800BB
:10AB70000030A00071B7200080487800C29B02001E
:10AB800000000000A0DD2000104078000080FB00E5
:10AB90004200DE006140600080417800A0DD2000BE
:10ABA000104078006340600080427800A0DD200003
:10ABB000104078000080FB004300DE006140600030
:10ABC0000041780070B72000104078000080FB0042
:10ABD0004300DE006140600080407800A06E80008D
:10ABE0000342780085417800329B0200000000009B
:10ABF000B69B02000000000010C0B3000C71020000
:10AC0000000000003EFE37000040EB000C71020027
:10AC1000000000003AFE37000080FA000000060045
:10AC20000000FA00EE980200000000000080FB0027
:10AC30000080FA00000006000200FA00000F780011
:10AC40001E0078005698020000000000001020004E
:10AC50000080FA00000006000000FA00549902008B
:10AC6000000000000080FB000080FA0000000600E9
:10AC70000000FA0060BA200010407800B49802008A
:10AC8000000000000080FA00000006000000FA004A
:10AC900060BA2000104078000080FB000080FA00BD
:10ACA000000006000000FA008040EB0060BA2000BF
:10ACB0000148780041022000B00020004E9A0200B6
:10ACC000000000000080FA00000006000000FA000A
:10ACD00011C0B30060BA2000014878004102200092
:10ACE000B00020004E9A0200000000000080FA0030
:10ACF000000006000000FA0070B720001040780045
:10AD00000030A00071B72000804878008040EB0040
:10AD100080BB200001487800C922A800CB22A900EE
:10AD2000E1022000F00220004E9A02000000000024
:10AD30000080FA00000006000400FA00881F780076
:10AD4000000F78001E00E0004400320020032000C5
:10AD50009E0F100041003E001E0FE90080BB200046
:10AD6000104078000080FB009E0F500005003E0060
:10AD700091022000D00520004E9A02000000000041
:10AD800063013700E100200060082000C499020040
:10AD9000000000001E0078000040E800486F02003C
:10ADA00000000000E0A12800B06C020000000000DC
:10ADB0008040EB0020BB2000014878001F003700D6
:10ADC0001E01780020BB2000104078008080FB002E
:10ADD0004310DD008100400090BB20000080400057
:10ADE000104078000080FB009C96020000000000EC
:10ADF00000C2B3000C710200000000001E017800C8
:10AE000020BB2000104078008080FB004310DD0054
:10AE10008100400090BB200000804000104078007E
:10AE2000569802000000000020BB2000104078006F
:10AE30008040E80020BB20000148780020BB2000B3
:10AE400010407800E74F5000DDFF360010A22800C8
:10AE5000DC6C0200000000002D0137001E007800AD
:10AE600010079800500520009E009000808F500031
:10AE700011013200500520009E009000808F50008C
:10AE800008003E001E0090000000E00012003200AA
:10AE9000300320009E009000808F5000DD003200C3
:10AEA00017013700C00E20009E009000808F5000D8
:10AEB00063003200000F20009E009000808F500041
:10AEC0005F003200C00C20009E009000808F500078
:10AED000020132000A013700D100200040092000A1
:10AEE0004E9A02000000000071012000100A2000AC
:10AEF0004E9A02000000000080BB20001040780045
:10AF00000004E00005003A0091022000D005200076
:10AF10004E9A020000000000440037008040EB0021
:10AF200030BB2000014878003A00370000C2B3006F
:10AF30000C7102000000000030BB200010407800BF
:10AF40000040E800486F02000000000020A2280036
:10AF5000B06C0200000000008040EB0020BB20002D
:10AF6000014878001600370030BB20001040780000
:10AF70000081FB0020BB2000104078008080FB0097
:10AF80004310DD008100400090BB200000804000A5
:10AF9000104078000080FB009C960200000000003A
:10AFA00000C2B3000C7102000000000020BB2000B2
:10AFB000104078008040E80020BB20000148780065
:10AFC00020BB200010407800E74F5000E6FF36001D
:10AFD00061002000800B2000C499020000000000E6
:10AFE00030BB2000104078000080FB00C300DD0073
:10AFF00090BB20000080400010407800F700070060
:10B0000030BB2000104078008040E80030BB2000BA
:10B010000148780080BB20009040780030BB2000C1
:10B020001040780080CF5000C0FF3E00310D20005E
:10B03000E00B20004E9A020000000000B400370030
:10B040001E00780080407800C0832000014878000E
:10B05000C00E20009E0F100005003A0031012000B4
:10B06000101920004E9A0200000000000400370072
:10B07000D1002000401A20004E9A0200000000007B
:10B0800071012000100A20004E9A0200000000000A
:10B090008040EB0020BB2000014878000A01070037
:10B0A0008040780030BB2000014878008040EB00F1
:10B0B00080BB2000014878004D00370000C2B3007B
:10B0C0000C7102000000000020BB2000104078003E
:10B0D0000040E800486F02000000000020A22800A5
:10B0E000B06C0200000000000000EB00805D8800F2
:10B0F0000D003700815D800090C02000008040007E
:10B10000104078000080FB009C96020000000000C8
:10B1100000C2B3000C71020000000000805D8000DE
:10B120000000E800805D8800805D8000E70F50002F
:10B13000F0FF360061002000800B2000C49902005F
:10B140000000000090C0200010407800A30007001D
:10B1500020BB200010407800E94F50001B003E004B
:10B160000000EB00805D88001000370080BB2000ED
:10B17000104078008081FB00845D8000815D80004C
:10B1800090C0200000804000104178004318DD008E
:10B190008400400090BB20000080400002487800FE
:10B1A000805D80000000E800805D8800805D800098
:10B1B000E70F5000EDFF360080BB20001040780004
:10B1C0008040E80080BB20000148780020BB2000C0
:10B1D000104078008040E80020BB20000148780043
:10B1E000C70007008040780030BB2000014878008D
:10B1F00030BB2000104078000004E000AFFF3A00B0
:10B20000B1022000101B20004E9A02000000000036
:10B210003F0037004800070011012000C01D20003A
:10B22000C49902000000000030C3B3005698020029
:10B23000000000000000EB00805D88001400370073
:10B24000885D8000EE9802000000000080407800D9
:10B2500070BA20000000440001487800815D800041
:10B2600070BA200000804000104078000080FB0091
:10B270009C9602000000000000C2B3000C710200A6
:10B2800000000000805D80000000E800805D880014
:10B29000805D8000E70F5000E9FF360010A2280013
:10B2A000DC6C02000000000070BA20001040780042
:10B2B0004A000700160037001F00070001012000A8
:10B2C000D01E20004E9A02000000000050C5B300BE
:10B2D00056980200000000000D003700160007001D
:10B2E000F1002000D01F20004E9A02000000000054
:10B2F000C0CCB300569802000000000004003700E4
:10B3000041022000C02020004E9A020000000000F0
:10B310004F0478000080FA00000006000000FA00E8
:10B3200091002000800821004E9A020000000000D9
:10B330000080FA00000006000200FA00D097020028
:10B3400000000000004F7800A10020000023200032
:10B35000C4990200000000001E04E00005003A004D
:10B360003100200050BB20004E9A02000000000077
:10B370001800370091002000A0232000C49902008B
:10B38000000000001E80FB00610060000004E0007F
:10B39000040032005101200030242000C499020032
:10B3A000000000001E80FB000000D1006100600072
:10B3B0000004E0000400320041012000802520004C
:10B3C000C49902000000000010A22800DC6C0200FA
:10B3D000000000000080FA00000006000400FA00EF
:10B3E000004F78001E80FB0010079800200220000C
:10B3F0009E009000808F50001E003200200220002E
:10B400009E009000808F500007003C001E009000BE
:10B41000E40F50001C0032009E009000F08F50009E
:10B420000A00320022003700800220009E009000B7
:10B43000808F50000A003200D00220009E00900051
:10B44000808F50001500320019003700B101200034
:10B45000C02620004E9A02000000000018003700AD
:10B46000A1012000702820004E9A02000000000078
:10B470001300370051012000102A20004E9A0200CC
:10B48000000000000E00370081012000602B20002A
:10B490004E9A020000000000090037000101200060
:10B4A000E02C20004E9A020000000000040037004B
:10B4B000E1002000E02D2000C499020000000000FF
:10B4C0000080FA00000006000000FA008040EB0057
:10B4D00010C12000014878008040EB0030C12000FE
:10B4E000014878008040EB0020C12000014878002E
:10B4F000080007000080FB000080FA000000060042
:10B500000000FA00030007000080FB000080FA0042
:10B51000000006000A00FA0010C0B300704798004F
:10B520000040EB00604798000040EB005047980057
:10B5300010C0B300104798000040EB00404798004F
:10B540008040EB0040C120000148780030C120005D
:10B55000104078000004E0009C003A00D097020000
:10B56000000000000004E0000C0032008040EB000E
:10B5700010C12000014878008040EB0030C120005D
:10B58000014878008040EB0020C12000014878008D
:10B590000000EB0040079800A1003700C0832000A6
:10B5A00010407800569802000000000054990200F4
:10B5B000000000003047980054990200000000008D
:10B5C000204798003E409000E14F500003003A00B1
:10B5D0002E409000E14F500068003200BE409000C5
:10B5E0002E40900080CF500003003200BE409000FB
:10B5F000014F78002600370010C1200090407800ED
:10B600007E409000814F50000E0031005E4090005F
:10B610008080FB0090C020000080400090407800B7
:10B620001E40900080C060000040EB00004F78009A
:10B630000104E0000C00320010C0B300004F78009D
:10B640000900370010C12000904078000040EB0056
:10B65000004F78007E409000814F500002003A0079
:10B6600010C0B300004F78001E04E00008003A004C
:10B670007E409000604798006E409000E84F500078
:10B6800003003E0020C12000EE40900001487800F9
:10B6900010C0B3009E4F10000D003A005E409000B5
:10B6A0000081FB005E4090008080FB0090C0200085
:10B6B00000804000904078001E40900080C07000E4
:10B6C00090C02000000041000148780011003700C0
:10B6D0005E4090000082FB005E4090008080FB0096
:10B6E00090C0200000804000104078008041780029
:10B6F0001E419000024078000080EA008180EA004C
:10B7000000C061008040780090C02000000042002E
:10B71000014878001E407800B49802000000000044
:10B720007E4090000040E800704798001E40900066
:10B7300000404000104798001E4090000004E000C8
:10B740000B003A005E4090008080FB0090C020001B
:10B750000080400010407800920007005E4090009A
:10B760000040E8005047980010C0B3001047980010
:10B770005E409000E74F50008CFF3600FE40900086
:10B7800000C4B30080CF50001000360040C120003C
:10B79000104078000004E0000C003A0010C12000C6
:10B7A000EE4090000148780010C120001040780061
:10B7B0000004E00003003A0011C0B30030C12000D3
:10B7C0000148780010C0B300404798004E409000F8
:10B7D0000004E0000400320090C020001040780017
:10B7E0000004E0000B003A008040EB0010C1200094
:10B7F000014878008040EB0030C12000014878000B
:10B800008040EB0020C12000014878000040EB00A0
:10B81000404798004E4090000080FB004007980091
:10B820004E0090000080FA00000006000E00FA00B2
:10B830000040EB00404798000C0037004E4090005D
:10B840000081FB004E4090008080FB0090C02000F3
:10B85000008040009040780065004700017178004A
:10B860004E4090000040E800404798004E40900055
:10B87000E74F5000F1FF360010C1200090407800E3
:10B880002147980030C1200090407800114798006F
:10B8900020C12000104F780001C4B30010C1200067
:10B8A000014878008040EB0030C12000014878005A
:10B8B00018FF07000004E0001A00320010C0B300B7
:10B8C000304798000040EB004047980011003700D7
:10B8D0004E4090008080FB00650047006141780089
:10B8E0004E4090008080FB0090C02000008040000F
:10B8F00010407800804F5100030032000040EB0000
:10B9000030479800090037004E4090000040E800A2
:10B91000404798004E409000E74F5000ECFF360043
:10B92000020037000040EB00304798000040EB0079
:10B93000404798000C0037004E4090000081FB000B
:10B940004E4090008080FB0065004700E140780099
:10B9500090C0200000004100014878004E40900057
:10B960000040E800404798004E409000E74F5000EC
:10B97000F1FF360010C12000AE4090000148780071
:10B9800030C120009E4090000148780020C1200076
:10B990001E4878003E4090000080FB000080FA00C6
:10B9A000000006000200FA00004F780040C12000AD
:10B9B000104078001E4068008080FB00D08320008B
:10B9C000008040009040780040C12000014878008D
:10B9D00040C12000104078000080FB000080FA0089
:10B9E000000006000000FA0040A22800B06C02002F
:10B9F000000000000080FA00000006000400FA00C9
:10BA0000C922A800CB22A900C8C2A90070B7200093
:10BA1000104078000030A00071B720008048780006
:10BA200070B72000104078000020A10071B72000FE
:10BA300080487800EBFF07000000370022C2BF00FB
:10BA4000614060000004E000FCFF32003011800023
:10BA50008040780070BB20000148780070BB200057
:10BA6000104078000080FB004400DE008040780039
:10BA700060BB20000148780060BB200010407800C7
:10BA80000080FB00100798001E009000E10F50009E
:10BA9000780032009E009000E48F50009D0032003C
:10BAA0001E0090000000E00001003200A1003700FD
:10BAB00070BB2000104078000080FB00000F780071
:10BAC0009E007800E28F5000170032001E007800C0
:10BAD000E20F500007003C009E0078000100E000EB
:10BAE000980032001E007800E10F50000C00320078
:10BAF0005C0037009E007800E48F50001300320095
:10BB00001E007800E40F5000560035009E007800BB
:10BB100068805000E10F500052003E0010003700D6
:10BB2000B0FF0700C5FF3700D097020000000000FB
:10BB30008040780040BB20000148780010C0B3006E
:10BB40000C71020000000000BCFF3700EE980200FC
:10BB5000000000000C71020000000000B7FF370079
:10BB600010C0B3000C7102000000000070BB200088
:10BB700010407800E94F500004003A00C1CEB300F5
:10BB8000C0832000014878000300370001CFB300D4
:10BB9000C0832000014878004BFE070080407800F9
:10BBA00040BB200001487800190037008040EB00BE
:10BBB00050BB2000014878000D00370050BB20002A
:10BBC000104078008080FB0090C020000080400082
:10BBD000104078000C7102000000000050BB2000F3
:10BBE000104078008040E80050BB200001487800F9
:10BBF00050BB200010407800E74F5000EFFF3600A8
:10BC00003FFE07008040780040BB200001487800DC
:10BC100040BB2000104078000004E000E3FF3A0041
:10BC20008040EB0050BB200001487800080037003E
:10BC300000C0EB000C7102000000000050BB2000AF
:10BC4000104078008040E80050BB20000148780098
:10BC500050BB200010407800E74F5000F4FF360042
:10BC600076FF37000040EB000C710200000000007E
:10BC700072FF370070BB200090407800F0C0B30026
:10BC800080C0600070BB20000148780070BB2000BD
:10BC9000104078008040E80070BB20000148780028
:10BCA00010C0B3000C710200000000008040EB00E7
:10BCB00050BB2000014878000F00370022C2BF00AF
:10BCC000614060000004E000FCFF320030118000A1
:10BCD000569802000000000010C0B3000C71020072
:10BCE0000000000050BB2000104078008040E800B9
:10BCF00050BB20000148780050BB200090407800E5
:10BD000070BB20001040780080CF5000EBFF39005E
:10BD10004AFF370070BB200010407800A69C02004C
:10BD20000000000010C0B3000C7102000000000011
:10BD300042FF37000040EB000C71020000000000E1
:10BD40003EFF37000080FA00000006000000FA0005
:10BD500040A42800B06C0200000000000080FA003F
:10BD6000000006000000FA000040EB0084810200A1
:10BD7000000000000040EB00848102000000000091
:10BD80000040EB0084810200000000000040EB0056
:10BD900084810200000000000000EB00C08002006F
:10BDA000000000000000EB00C08002000000000066
:10BDB0000000EB00C0800200000000000080FA00DC
:10BDC000000006000C00FA0070B720001040780058
:10BDD0000030A00071B720008048780070B72000C4
:10BDE000104078000020A10071B720008048780042
:10BDF00011C0B30060B720000148780081C0B300D3
:10BE000080B720000148780021C0B30010DF200077
:10BE10000148780080C0EB0020C0B300607F0200C2
:10BE200000000000C922A900C902A900C8E2A800B8
:10BE300010C0B300F081020000000000C3FF070043
:10BE40000000370022C2BF00614060000004E00033
:10BE5000FCFF3200301180008040780050DF20006D
:10BE60000148780050DF2000104078000080FB007F
:10BE70004400DE008040780040DF20000148780068
:10BE800040DF2000104078000080FB003007980061
:10BE90003E009000E30F500014013200BE009000FD
:10BEA000E38F50000A003C003E019000E10F51007A
:10BEB000A4003200BE019000E18F5100F8003C0068
:10BEC0003E0090000000E00012003200E502370062
:10BED000BE009000E68F50008E0232003E019000BE
:10BEE000E60F510004003C00BE019000E48F5100B9
:10BEF00080023200DB0237003E009000E80F500065
:10BF00009B023200BE009000EA8F500031013200E7
:10BF1000D402370050DF2000104078000080FB0082
:10BF20006101B9004207980053079800D000200033
:10BF3000010020004E019000DE019000800F5100B2
:10BF4000818F59007B003E004E009000DE00900083
:10BF500000600100C70237000C0037000D003700F9
:10BF600012003700170037001D003700230037008C
:10BF700043003700470037004B00370051003700BF
:10BF8000570037005D003700630037006FFF070080
:10BF9000ACFF3700EE7F02000000000010C0B300CD
:10BFA0000C71020000000000A6FF37002E80020086
:10BFB0000000000010C0B3000C710200000000007F
:10BFC000A0FF37000040EB00F081020000000000FD
:10BFD00010C0B3000C7102000000000099FF370090
:10BFE00010C0B300F08102000000000010C0B300D8
:10BFF0000C7102000000000092FF370010DF2000EB
:10C0000010407800E24F500006003A001481020010
:10C01000000000008040780030DF200001487800F8
:10C0200006003700F00F20004E80020000000000E4
:10C030008040780030DF20000148780070B7200091
:10C0400010407800644060000004E0000700320007
:10C0500030DF2000104078008497020000000000CC
:10C060008040780030DF20000148780030DF200079
:10C07000104078000C7102000000000071FF3700D2
:10C0800062810200000000000C710200000000004C
:10C090006CFF370002820200000000000C710200F9
:10C0A0000000000067FF370010C0B300A681020047
:10C0B0000000000010C0B3000C710200000000007E
:10C0C00060FF37000040EB00DE810200000000004E
:10C0D00010C0B3000C7102000000000059FF3700CF
:10C0E00010C0B300DE8102000000000010C0B300E9
:10C0F0000C7102000000000052FF37000040EB000E
:10C10000CC8102000000000010C0B3000C710200DE
:10C11000000000004BFF370010C0B300CC810200CC
:10C120000000000010C0B3000C710200000000000D
:10C1300044FF37000040EB000C71020000000000DB
:10C1400040FF370050DF200090407800F0C0B3007F
:10C1500080C0600050DF20000148780050DF2000E0
:10C16000104078008040E80050DF2000014878004F
:10C1700010C0B3000C710200000000008040EB0012
:10C1800030DF2000014878003E00370022C2BF00A7
:10C19000614060000004E000FCFF320030118000CC
:10C1A0008040780020DF20000148780070B7200030
:10C1B00010407800644060000004E0000700320096
:10C1C00020DF20001040780084970200000000006B
:10C1D0008040780020DF20000148780010DF200038
:10C1E00010407800E24F500009003A0020DF2000A4
:10C1F000104078000080FB00C080020000000000BA
:10C2000010C0B3000C7102000000000018003700DD
:10C2100020DF2000104078000080FB004E800200EC
:10C22000000000008040780020DF200001487800F6
:10C2300070B7200010407800644060000004E00007
:10C240000700320020DF20001040780084970200B1
:10C25000000000008040780020DF200001487800C6
:10C2600020DF2000104078000C7102000000000068
:10C2700030DF2000104078008040E80030DF2000F0
:10C280000148780030DF20009040780050DF200027
:10C290001040780080CF5000BCFF3900E9FE370025
:10C2A00050DF200090407800F0C0B30080C06000F4
:10C2B00050DF20000148780050DF20001040780057
:10C2C0008040E80050DF20000148780050DF200067
:10C2D00010407800A68102000000000010C0B300EA
:10C2E0000C71020000000000D6FE370050DF200075
:10C2F00090407800F0C0B30080C0600050DF2000A4
:10C300000148780050DF2000104078008040E800AD
:10C3100050DF20000148780010C0B3000C7102000B
:10C320000000000022C2BF00614060000004E00085
:10C33000FCFF3200301180008040780040DF200098
:10C34000014878008040EB0030DF20000148780091
:10C350001600370040DF2000104078000004E000A5
:10C3600004003D0010C0B300848102000000000002
:10C37000030037000040EB00848102000000000051
:10C3800040DF2000104078000040400080407800EE
:10C3900040DF20000148780030DF200010407800A6
:10C3A0008040E80030DF20000148780030DF2000C6
:10C3B0009040780050DF20001040780080CF50007F
:10C3C000E4FF390010C0B3000C710200000000004F
:10C3D0009CFE370050DF2000104078000080FB00FA
:10C3E00020079800400A2000AE009000808F500087
:10C3F00015003200500A20002E019000800F5100DD
:10C40000C5003200000A2000AE019000808F51006C
:10C41000010032003301370022C2BF0061406000DA
:10C420000004E000FCFF3200301180008040780002
:10C43000C0DE20000148780010C0B3000C7102007B
:10C44000000000007FFE3700C0DE200010407800B2
:10C450000080FB00100798001E009000E10F5000C4
:10C46000040032009E009000E28F50003B0032003A
:10C47000A500370022C2BF00614060000004E00058
:10C48000FCFF320030118000506F8800506F800038
:10C490006300B900506F88000000EB00406F880017
:10C4A0000C00370022C2BF00614060000004E000C1
:10C4B000FCFF320071408000406F800080804000AF
:10C4C0003011800080487800406F80000000E80054
:10C4D000406F8800416F8000506F8000808F500057
:10C4E000F0FF39000000EB00406F880013003700B8
:10C4F00071408000406F8000008040000080E800B4
:10C500001041780071408000406F80000080400042
:10C510000000E8009041780071408000406F80008A
:10C5200000804000104078008340780053010700ED
:10C53000406F800063004000406F8800416F8000C2
:10C54000506F8000808F5000E9FF390010C0B300A9
:10C550000C710200000000003AFE370022C2BF004A
:10C56000614060000004E000FCFF320030118000F8
:10C57000506F8800506F80004200DD00506F8800CF
:10C580000000EB00406F88000C00370022C2BF00A3
:10C59000614060000004E000FCFF32007140800058
:10C5A000406F80008080400030118000804878001B
:10C5B000406F80000000E800406F8800416F8000FD
:10C5C000506F8000808F5000F0FF39000000EB00BA
:10C5D000406F8800440037000040EB008481020077
:10C5E000000000000040EB00848102000000000019
:10C5F0000040EB0084810200000000000040EB00DE
:10C60000848102000000000071408000406F8000C3
:10C6100000804000104078000080FB00C0800200D5
:10C620000000000071408000406F800000804000EA
:10C630000000E800104078000080FB00C08002008D
:10C640000000000071408000406F800000804000CA
:10C650000080E800104078000080FB00C0800200ED
:10C660000000000071408000406F800000804000AA
:10C670006301400071408000406F800000804000F6
:10C6800063004000104078006F406000004978006F
:10C690008040EB0030DF20000148780006003700C2
:10C6A000B0FD070030DF2000104078008040E80037
:10C6B00030DF20000148780071408000406F80002A
:10C6C00000804000630040009040780030DF200090
:10C6D0001040780080CF5000F1FF3E00406F800096
:10C6E00064004000406F8800416F8000506F800000
:10C6F000808F5000B8FF390010C0B3000C710200E9
:10C7000000000000CFFD37000040EB000C7102007C
:10C7100000000000CBFD3700C0DE20001040780094
:10C720000080FB00000F78001E017800E10F51002F
:10C73000040032009E017800E28F51004500320073
:10C74000C0FD370022C2BF00614060000004E0006D
:10C75000FCFF320030118000506F880022C2BF0001
:10C76000614060000004E000FCFF320030118000F6
:10C770008040780040DF2000014878000000EB0096
:10C78000406F88002E00370040DF20009040780086
:10C7900020DF2000014878008040EB0030DF2000DF
:10C7A000014878001900370020DF20001040780091
:10C7B0000080FB00610060000004E0000400320023
:10C7C00010C0B300848102000000000003003700A5
:10C7D0000040EB00848102000000000020DF200008
:10C7E000104078000080FB000000D10080407800FD
:10C7F00020DF20000148780030DF20001040780062
:10C800008040E80030DF20000148780030DF200061
:10C8100010407800E34F5000E3FF3600148102001F
:10C820000000000014810200000000000C710200F2
:10C8300000000000406F80000000E800406F8800AA
:10C84000416F8000506F8000808F5000CEFF390014
:10C850007CFD370022C2BF00614060000004E000A0
:10C86000FCFF320030118000506F88000000EB00A8
:10C87000406F88001600370022C0B30060B9200066
:10C88000A10B2000B7000700ED00070022C0B30095
:10C8900060BB2D00A10B2000B200070022C0B30036
:10C8A000603D2D00A10B2000AE000700E400070052
:10C8B00022C0B30060BB2000A10B2000A90007002C
:10C8C000DF000700406F80000000E800406F880034
:10C8D000416F8000506F8000808F5000E6FF39006C
:10C8E00058FD37000040EB000C7102000000000012
:10C8F00054FD370050DF200010407800A69C020055
:10C900000000000010C0B3000C7102000000000025
:10C910004CFD370050DF20009040780030C0B3005D
:10C9200080C0600050DF20000148780050DF200008
:10C930009040780060B720000148780060B7200080
:10C940009040780010DF200010407800607F0200E7
:10C950000000000010C0B300F081020000000000E1
:10C9600010C0B3000C7102000000000035FD37005C
:10C9700070B72000104078000030A10071B720008F
:10C980008048780050DF2000104078000080FB00D5
:10C990004300DE000000A200610060000004E0002F
:10C9A0000500320070B72000104078000030A00071
:10C9B00071B720008048780021C0B30010DF20004C
:10C9C0000148780050DF2000104078000080FB0014
:10C9D0004200DE00610060000004E000030032005D
:10C9E00031C0B30010DF20000148780070B720008C
:10C9F000104078000020A10071B720008048780026
:10CA000050DF2000104078000080FB000000D100C3
:10CA1000610060000004E0000500320070B72000F3
:10CA2000104078000020A00071B7200080487800F6
:10CA300060B720009040780010DF200010407800A0
:10CA4000607F02000000000010C0B300F08102000F
:10CA50000000000010C0B3000C71020000000000D4
:10CA6000F8FC37000040EB000C71020000000000F1
:10CA7000F4FC37000080FA00000006000600FA000F
:10CA80002047980031479800424798002E40900078
:10CA90000080FB004600DE00004F78000040EB0005
:10CAA00010479800220037001E409000E34F5000CE
:10CAB0000C003A001E04E0000A00320010C0B3006F
:10CAC000DE810200000000001E80FB0022970200B1
:10CAD000000000000040EB00DE81020000000000CA
:10CAE000100037002E4090000080FB0061006000C5
:10CAF0000004E0000400320010C0B3008481020092
:10CB000000000000030037000040EB0084810200B9
:10CB1000000000002E4090000080FB000000D100CB
:10CB2000204798001E4090000040E8001047980001
:10CB30001E409000E34F5000DBFF36003E40900067
:10CB40000080FB00C0800200000000004E4090000A
:10CB50000080FB00C0800200000000000080FA009E
:10CB6000000006000800FA0010079800210798004E
:10CB7000624798000040EB00848102000000000042
:10CB80000040EB0084810200000000000040EB0048
:10CB900084810200000000000040EB00848102005C
:10CBA000000000001E0090008497020000000000BA
:10CBB0000080FB00C0800200000000001E0090000A
:10CBC000AE0090004809DD004800DE000000710062
:10CBD000C808DE0084970200000000000080FB000F
:10CBE000C0800200000000001E009000AE00900017
:10CBF0004008DE00010020008497020000000000D1
:10CC00000080FB00C0800200000000006E40900029
:10CC10006F406000604798000040EB00004F7800D4
:10CC2000020037004FFC07001E4FE8006E409000E6
:10CC30009E4F1000FBFF39000080FA000000060044
:10CC40000000FA0010C0B300848102000000000060
:10CC50000040EB0084810200000000000040EB0077
:10CC600084810200000000000040EB00848102008B
:10CC7000000000000000EB00C08002000000000087
:10CC800014810200000000000C710200000000008E
:10CC900014810200000000000C710200000000007E
:10CCA00030FC07002FFC07000080FA00000006009F
:10CCB0000200FA00005D80000000E0001200320077
:10CCC00000C2B3000C71020000000000310020001F
:10CCD00010442000C49902000000000000C2B3000C
:10CCE0000C71020000000000F05C80000000E00019
:10CCF00003003A000040EB008481020000000000C5
:10CD00000000EB00005D8800F05C80000000E000A7
:10CD100003003A001481020000000000004F780078
:10CD200010002000005D88001E80FB000080FA00DB
:10CD3000000006000400FA00000F7800005D80008B
:10CD40000000E0001200320000C2B3000C710200CB
:10CD5000000000003100200010442000C4990200AF
:10CD60000000000000C2B3000C71020000000000CF
:10CD7000F05C80000000E00003003A000040EB009F
:10CD800084810200000000000000EB00005D8800CC
:10CD9000F05C80000000E00007003A001E00780010
:10CDA000C08002000000000062810200000000005C
:10CDB0000080FB00000F780000C2B3000C7102007D
:10CDC000000000001E00E00007003A0031002000D3
:10CDD00010442000C4990200000000000030200030
:10CDE0001007980006003700410020004044200052
:10CDF000C4990200000000000010200010079800F5
:10CE00001E0090000080FA00000006000000FA00FA
:10CE1000005D80000000E0000F00320041002000B3
:10CE200040442000C49902000000000000A1280036
:10CE3000DC6C020000000000F05C80000000E000FC
:10CE400003003A0010C0B30084810200000000001B
:10CE50000000EB00005D8800F05C80000000E00056
:10CE60000F003A00EE7F0200000000000000E0002A
:10CE70000B00320091002000A0232000C499020082
:10CE8000000000005101200030242000C49902005D
:10CE90000000000000A12800DC6C0200000000007F
:10CEA000D1002000804420004E9A020000000000C3
:10CEB0000080FA00000006000000FA00005D80001B
:10CEC0000000E0000F00320041002000404420003C
:10CED000C49902000000000000A12800DC6C0200E0
:10CEE00000000000F05C80000000E00003003A0059
:10CEF00010C0B30084810200000000000000EB00BD
:10CF0000005D8800F05C80000000E00002003A0054
:10CF10002E80020000000000C100200050452000CB
:10CF20004E9A0200000000000080FA000000060097
:10CF30000000FA000101200020522000C4990200E4
:10CF4000000000000040EB00486F020000000000FD
:10CF500000C2B3000C7102000000000060B72000A6
:10CF600010407800486F02000000000000C2B300CB
:10CF70000C7102000000000010A12800DC6C02000F
:10CF8000000000000080FA00000006000400FA0023
:10CF90000000EB00100798000000EB00F05C880038
:10CFA0001A1A0200000000004416020000000000EF
:10CFB000000F78001E00E00009003400400020004F
:10CFC0009E0F100006003C001E0078000040E900A3
:10CFD0008040780060B720000148780002003700E8
:10CFE0000000EB00000F78001E00E0002D003A006A
:10CFF0000000EB00606988000000EB00F05C880036
:10D00000F05C80000000E0000F003A00B103200057
:10D01000604820004E9A0200000000008001EB00F2
:10D02000420020001100200010002000901C02008F
:10D03000000000000040E9008040780060B7200058
:10D040000148780022003700C140800030002300F2
:10D05000808F500004003E0051032000104C20003F
:10D06000C499020000000000C1022000604F2000AF
:10D07000C4990200000000008001EB003200200093
:10D080001100200010002000901C02000000000091
:10D090000040E9008040780060B720000148780037
:10D0A0000B003700C140800030002300808F50000B
:10D0B00004003E0051032000104C2000C4990200DF
:10D0C000000000009AFF07000000EB00005D8800F0
:10D0D00070B72000104078000030A00071B7200029
:10D0E00080487800F05C80000000E00009003A0011
:10D0F000C922A800C902A800CB02A900CB22A9001E
:10D1000060B720009040780020C0B300607F02002C
:10D11000000000000080FA00000006000000FA0095
:10D120000000EB00005D8800F05C8000E10F500023
:10D1300001003A0007E2A9000080FA0000000600A2
:10D140000600FA00100798001E00900020079800C3
:10D150002E009000E10F50000C0032002E009000D5
:10D16000E10F5000040039002E009000E20F500043
:10D170006500320073003700510320002053200067
:10D18000C499020000000000720037008040EB00EC
:10D19000003020000E82020000000000E1022000AA
:10D1A000705620004E9A020000000000CBC2BF0063
:10D1B000614060000004E00004003200CBC2BF0008
:10D1C000624060000004E0000C003A009100200082
:10D1D000A0232000C499020000000000510120009B
:10D1E00030242000C49902000000000000A12800A3
:10D1F000DC6C020000000000560037000000EB006D
:10D20000000F780039003700F05C80000000E0007B
:10D2100009003A00EE7F0200000000001E007800C6
:10D22000C0800200000000006281020000000000D7
:10D230000080FB00100798001E0090000000E00036
:10D2400024003A001E0078009C96020000000000B6
:10D2500080C2B3000C710200000000001E007800C4
:10D260000080D1009C960200000000001E007800A3
:10D270000000A200610060000004E0000400320031
:10D2800030A12800B06C0200000000000B00370045
:10D29000F05C80000000E00005003A00148102000C
:10D2A0000000000010C0B3008481020000000000F4
:10D2B00060A12800B06C02000000000010A128004E
:10D2C000B06C02000000000000C2B3000C7102004C
:10D2D00000000000F05C80000000E00002003A0066
:10D2E0002E800200000000001E0FE800F00F20005A
:10D2F0009E0F1000C4FF340000A12800DC6C020067
:10D300000000000013003700F05C8000E10F5000C7
:10D3100001003A0007E2A9007100200050592000E6
:10D320004E9A020000000000F1002000C01E210003
:10D330004E9A02000000000010C0B3000E0007006B
:10D340000400370041022000C02020004E9A020055
:10D35000000000000080FA00000006000000FA0053
:10D36000B1002000C00921004E9A02000000000018
:10D370000080FA00000006000A00FA00004F980042
:10D380000040EB00204798000040EB001047980059
:10D390000040EB00004F7800B47102000000000074
:10D3A000C922A800C902A800CB02A900CB22A9006B
:10D3B00062A0A80062C0A8008660A900CBC2BF001E
:10D3C0000080FB000000D1006140600060479800D1
:10D3D0006E40900050479800CBC2BF006140600093
:10D3E000604798006E40900030479800000037007A
:10D3F00086C0BF00684060000004E00012003A00F0
:10D4000023C2BF00624060000004E0000E003A004A
:10D41000F27102000000000022C2BF006140600003
:10D420000004E000F2FF320030118000004F78006D
:10D4300062A0A90062C0A9000E4890000004E000AC
:10D4400061003A00630037008660A900CBC2BF00CC
:10D450000080FB000000D100614060006047980040
:10D46000CBC2BF0061406000404798002E40900052
:10D470000004E0002E0032003E4090000004E00076
:10D480002B003A004E4090000004E00028003200DB
:10D490001E409000E74F50000B003E001E407800F9
:10D4A00000404000004F78006E4090000004E00013
:10D4B000010032001E04A0001E4090000040E80061
:10D4C000104798003B0037000E4890000004E00031
:10D4D000040032001E80FB00D46F02000000000038
:10D4E00006003700C0C5B300C27102000000000092
:10D4F0001E407800C2710200000000006E409000E3
:10D500000004E00004003200D0C2B300C271020087
:10D510000000000003003700B0C2B300C271020077
:10D52000000000000040EB00104798002100370089
:10D530003E4090000004E0001E0032004E4090008B
:10D540000004E0001B0032005E4090000004E00098
:10D550000B0032006E4090000004E00008003A002A
:10D5600010C0B300204798000040EB00104798001F
:10D57000B0C5B300C2710200000000000D0037000A
:10D580005E4090000004E0000A003A006E40900007
:10D590000004E000070032000040EB002047980044
:10D5A0000040EB0010479800D0C5B300C2710200E4
:10D5B000000000006E409000504798004E409000E0
:10D5C000304798008AFF370000A12800DC6C020079
:10D5D000000000000080FA00000006000000FA00D1
:10D5E00090A12800B06C0200000000000080FA004A
:10D5F000000006000400FA00C922A800C902A80021
:10D60000CB02A900CB22A900C8C2A90070B7200094
:10D61000104078000030A00071B7200080487800EA
:10D6200070B72000104078000020A10071B72000E2
:10D630008048780080C0EB0020C0B300607F02000B
:10D6400000000000E5FF07000000370022C2BF0015
:10D65000614060000004E000FCFF320030118000F7
:10D6600080407800C0B9200001487800C0B920008F
:10D67000104078000080FB004400DE00804078000D
:10D68000B0B9200001487800B0B9200010407800FF
:10D690000080FB00100798001E009000E10F500072
:10D6A0005E0032001E009000E10F500004003C00BC
:10D6B0001E0090000000E0000800320097003700D4
:10D6C0001E009000E40F50008C0032001E009000FD
:10D6D000E60F50007A00320090003700C0B92000F9
:10D6E000104078000080FB00000F78001E007800DA
:10D6F000E30F5000260032001E007800E30F5000B8
:10D700000A003C001E007800E10F500018003200B3
:10D710001E007800E10F500017003C001E0078004A
:10D720000000E00081003200380037001E00780061
:10D73000E60F5000210032001E007800E60F500076
:10D7400004003C001E007800E40F50001600320078
:10D750002E0037001E007800E70F50001E00320038
:10D760001E007800EF0F5000220032002700370023
:10D770009AFF0700B5FF3700EE7F020000000000AF
:10D7800010C0B3000C71020000000000AFFF3700B2
:10D790002E8002000000000010C0B3000C710200D7
:10D7A00000000000A9FF3700148102000000000003
:10D7B0000C71020000000000A4FF37000040EB00E5
:10D7C000848102000000000010C0B3000C71020050
:10D7D000000000009DFF370010C0B30084810200EC
:10D7E0000000000010C0B3000C7102000000000037
:10D7F00096FF37000040EB00DFFE070010C0B300CB
:10D800000C7102000000000090FF37000040EB00A8
:10D810000C710200000000008CFF3700C0B920002E
:10D8200090407800F0C0B30080C06000C0B9200014
:10D8300001487800C0B92000104078008040E8001E
:10D84000C0B920000148780010C0B3000C7102007C
:10D85000000000008040EB00A0B9200001487800E3
:10D860001000370022C2BF00614060000004E000E9
:10D87000FCFF320030118000C08002000000000078
:10D8800062810200000000000C7102000000000034
:10D89000A0B92000104078008040E800A0B9200026
:10D8A00001487800A0B9200090407800C0B920005D
:10D8B0001040780080CF5000EAFF390063FF370046
:10D8C000C0B920009040780030C0B30080C0600034
:10D8D000C0B9200001487800C0B92000904078000D
:10D8E00020C0B300607F02000000000010C0B30041
:10D8F0000C7102000000000054FF3700C0B9200086
:10D9000010407800A69C02000000000010C0B30088
:10D910000C710200000000004CFF37000040EB00DB
:10D920000C7102000000000048FF37000080FA0080
:10D93000000006000200FA00000F78001E00E00060
:10D940000300320010C3B3003302070002003700A7
:10D9500000C3B300300207000080FA000000060098
:10D960000600FA0010079800020037001E407800F9
:10D97000290207001E009000104F78001E4078001A
:10D98000404798004E4090000004E0000200320042
:10D9900010C0B300404798004E4090009E00900099
:10D9A0008100E800110798000004E000EFFF3A0052
:10D9B0000080FA00000006000600FA001007980038
:10D9C000020037001E407800130207001E0090007E
:10D9D000104F78001E407800404798004E4090005D
:10D9E0000004E0000200320010C0B300404798007D
:10D9F0004E4090009E0090008100E80011079800C2
:10DA00000004E000EFFF3A00D0C0B30002020700BC
:10DA1000A0C0B300000207000080FA00000006006A
:10DA20000400FA002047980000C8B300004F7800B7
:10DA3000A09D2800CAFF07000040EB001047980097
:10DA40000F0037002E4090001E4060000004E000F0
:10DA50000300320010C3B300EF01070002003700DB
:10DA600000C3B300EC0107001E80FB000000D100E2
:10DA7000004F78001E4090000040E80010479800DA
:10DA80001E409000E74F5000EEFF36000080FA0085
:10DA9000000006000E00FA00500798006107980089
:10DAA0000040EB00004F780000102E00515F200076
:10DAB00030079800410798000040EB00104798009D
:10DAC000320037003E019000CE0190005E009000D1
:10DAD000EE009000300602000000000010079800E1
:10DAE000210798001E04E00005003A001E00900087
:10DAF000AE009000E00F5000E08F58001800320098
:10DB00001E0090000043B000C30107009E0090007B
:10DB10003E009000000AB8009E0090004E00900069
:10DB20000088B9000501780000014100BE009000A6
:10DB30002E0090000088B9000001410082027800A8
:10DB40005E009000EE0090000400500085805800B8
:10DB5000500798006107980010C0B300004F78008C
:10DB60003E009000CE009000A200200003002000A4
:10DB700030060200000000003007980041079800BE
:10DB80001E4090000040E800104798001E409000A2
:10DB9000E74F5000CBFF36005E0090000043B0001E
:10DBA0009D0107000080FA00000006000C00FA004A
:10DBB00040079800510798000000EB0010079800FC
:10DBC0000000EB00000F78006000B800200798000C
:10DBD000310798004E019000DE019000F0232400F0
:10DBE000F1002000800F5100818F59002100360084
:10DBF0004E009000DE00900002242400F30020007C
:10DC0000300602000000000020079800310798004D
:10DC10002E0090006F000700C0C2B3007E01070015
:10DC20004E009000DE00900002242400F30020004B
:10DC300050060200000000004007980051079800BD
:10DC40004E019000DE019000703E20000100200097
:10DC5000800F5100818F590002003E00D09D2800A6
:10DC60003FFF070010002000100798001000200060
:10DC7000000F78004E019000DE019000703E200001
:10DC800001002000800F5100818F590032003600C2
:10DC90004E009000DE009000823E20000300200035
:10DCA00030060200000000002007980031079800AD
:10DCB0002E019000BE0190004006200001002000CF
:10DCC000800F5100818F5900030036002E00900014
:10DCD00040000700140037001E0090000000E00024
:10DCE0000F0032002E019000BE019000A000200025
:10DCF00001002000800F5100818F59000300360081
:10DD000000C3B3004401070002003700209E280032
:10DD100013FF07002E0090002E00070002003700BE
:10DD20002E0090002B000700C0C2B3003A0107008C
:10DD30004E009000DE009000823E20000300200094
:10DD400050060200000000004007980051079800AC
:10DD500010002000000F78004E019000DE019000BE
:10DD60004006200001002000800F5100818F5900E3
:10DD7000030036004E009000160007001300370025
:10DD80001E00E0000F0032004E019000DE01900006
:10DD9000A000200001002000800F5100818F590059
:10DDA0000300360000C3B3001B0107000200370068
:10DDB000209E2800EAFE07004E00900005000700A4
:10DDC000020037004E009000020007000080FA00B9
:10DDD000000006000800FA00300798000040EB0041
:10DDE000004F780000712200200798000040EB00EF
:10DDF000104798001E0037003E0090002E01900052
:10DE0000110009000280D800100798001E04E000ED
:10DE100003003A001E0090000000E0000C003200F9
:10DE20001E0090000043B000FB0007009E00900021
:10DE30002E0090000088B900800078003E0090001D
:10DE4000010050003007980010C0B300004F780068
:10DE50002E009000A2002000110009000280D800CE
:10DE6000200798001E4090000040E80010479800EE
:10DE70001E409000E34F5000DFFF36003E00900050
:10DE80000043B000E40007000080FA000000060034
:10DE90000600FA00404798000040EB00004F780071
:10DEA00040C6B300304798000040EB002047980080
:10DEB000200037004E4090008080FB003E409000E4
:10DEC0000081FB00110009008280D80010479800F3
:10DED0001E04E00003003A001E4090000004E00031
:10DEE0000B0032001E4090000043B000CA00070043
:10DEF0004E4190009E4090003E4090000088B90046
:10DF0000004051004047980010C0B300004F780017
:10DF10003E4090000080FB00A2002000110009009C
:10DF20000280D800304798002E4090000040E80062
:10DF3000204798002E409000E14F5000DDFF360052
:10DF40004E4090000043B000B30007000080FA008C
:10DF5000000006000400FA0010079800509F2800F7
:10DF60007FFE07001E0090004400DE006F0F60007F
:10DF70009E007800509E28000080400010407800ED
:10DF8000A50007001E0090006F0F60009E00780043
:10DF9000509E280000804000104078009E0007003E
:10DFA0000080FA00000006000400FA001007980044
:10DFB00000C3B300F300070080C7B300F1000700FF
:10DFC0001E0090004400DE006F0F60009E0078008D
:10DFD000509E28000080400010407800E9000700B3
:10DFE0001E0090006F0F60009E007800509E280079
:10DFF0000080400010407800E20007000080FA0036
:10E00000000006000400FA0010079800509F280046
:10E0100053FE07001E0090004C00DE006F0F6000F2
:10E020009E007800509E280000804000104078003C
:10E03000790007001E0090004800DE006F0F6000AE
:10E040009E007800509E280000804000104078001C
:10E05000710007001E0090004400DE006F0F60009A
:10E060009E007800509E28000080400010407800FC
:10E07000690007001E0090006F0F60009E0078008E
:10E08000509E280000804000104078006200070089
:10E090000080FA00000006000800FA00300798002F
:10E0A0003E009000CF80DE00F4030200000000007C
:10E0B000926C2200B33124005204020000000000E0
:10E0C00010079800210798001E009000AE009000F5
:10E0D0005606020000000000004F78001E40780045
:10E0E0006BFF0700E0C2B3004B0007001E0090006A
:10E0F000AE0090005606020000000000CF80DE0057
:10E10000F4030200000000000001BE001E009000A9
:10E11000AE009000D6040200000000001007980036
:10E120002107980002002000031224001E00900026
:10E13000AE00900092050200000000001007980059
:10E14000210798001E009000AE00900056060200C5
:10E1500000000000004F78001E4078004CFF0700D0
:10E160001E009000AE009000560602000000000065
:10E17000CF80DE00F4030200000000000001BE00BA
:10E180001E009000AE009000D604020000000000C7
:10E1900010079800210798000200200003122400B5
:10E1A0001E009000AE0090009205020000000000EA
:10E1B00010079800210798001E009000AE00900004
:10E1C0005606020000000000004F78001E40780054
:10E1D0002FFF07000080FA00000006000000FA0090
:10E1E00022C2BF00614060000080FB000080FA0096
:10E1F000000006000000FA0022C2BF00614060007B
:10E200000004E000FCFF3200301180000080FB00C1
:10E210000080FA00000006000200FA00004F7800BB
:10E22000D040800001102000010060000000E000EC
:10E2300006003A0023C2BF00624060000004E00014
:10E24000FCFF3A001E00FB00201188000080FA004D
:10E25000000006000200FA00004F78001E80FB005C
:10E26000401188000080FA00000006000000FA005B
:10E2700095C0BF00704060000004E00010003A004C
:10E280005140800040408000808F50000C003200E0
:10E2900023C2BF00624060000004E000FCFF3A00BF
:10E2A0008580A9009580A800314080004040800012
:10E2B00000804000104078000080FB0020118800A2
:10E2C0000080FA0000000600809FBE000000FA00F7
:10E2D000014080002040800080804000301180009C
:10E2E00080487800204080000000E800204088003E
:10E2F0002140800010408000808F500001003A00D3
:10E300009560A9008560A9000080FA004F00BE005A
:10E3100000400600809FBE000000FA0040408000E0
:10E320000000E800404088004140800050408000EC
:10E33000808F500002003A009580A9000600370047
:10E340003140800040408000008040001040780054
:10E350000080FB00201188008580A9000080FA0061
:10E360004F00BE00004006000000FA000000EB0075
:10E37000906E880010002000806E88000080FA00F7
:10E38000000006000200FA00004F7800816E800055
:10E39000906E8000808F500002003A00CA82A9006F
:10E3A0000E00370071408000806E80008080400049
:10E3B0001E40780080487800806E80000000E800F1
:10E3C000806E8800816E800000002100808F5000E8
:10E3D00002003A000000EB00806E88000080FA0026
:10E3E000000006000200FA00906E8000000FE800B6
:10E3F000000021009E0F100002003A000000EB0018
:10E40000000F7800806E80009E0F10000C0032001C
:10E4100023C2BF00624060000004E00008003A0030
:10E420001E007800906E880071408000906E800021
:10E4300000804000104078000080FB002011880020
:10E440000080FA00000006000400FA00000F7800C7
:10E45000110798001E007800900188001E009000AF
:10E460001080BA00C800DD001E0090001000BA0045
:10E47000008070000080FA00000006000600FA002C
:10E480000000EB00800888000000EB00F008880026
:10E490000000EB00E00C8800206180000000E0003C
:10E4A00008003A00A16C20009140780000CEB30033
:10E4B00000C06000CAE6B7000000EB00B060880052
:10E4C0003D00370020618000E30F500005003C0054
:10E4D000E0032000000F780010A1A8001081A80020
:10E4E0001500370020618000FE0F500005003C0041
:10E4F000A00F2000000F780010A1A8001081A90033
:10E500000D00370021618000400F2000808F5000F7
:10E5100005003C00007D2000000F780010A1A9003C
:10E520001081A8000400370000E82300000F7800E5
:10E5300010A1A9001081A9002061800000017800CD
:10E540001E007800110009000280D8000000E900D8
:10E55000200798002E00900060088800306180003D
:10E56000800078002E0090000088B900420620004C
:10E57000110009000280D80010079800A16C20004B
:10E580009140780000CEB30000C060006041B3004D
:10E59000CAE6B7001E009000D00C88001E00900054
:10E5A000C00C880060002000E00C880011E1A80089
:10E5B00020002000B06088000080FA000000060003
:10E5C0001200FA000000EB00800888000000EB0059
:10E5D000F00888000000EB00E00C8800B0608000CC
:10E5E000E20F500014003A00A16C20009140780026
:10E5F00000CEB30000C06000CAE6B700C100200032
:10E60000C02E20004E9A0200000000000000EB0027
:10E61000B0608800506980008000E800F00F2000A2
:10E620008080600080C220000080400010407800A0
:10E630000004E000AE0032000000EB00200798006C
:10E64000506980000000E80050698800516980002E
:10E65000F00F200000806000506988001A1A020044
:10E66000000000004416020000000000400798006F
:10E670001A1A020000000000441602000000000008
:10E68000CF80DE00F403020000000000008FBE0017
:10E690004E0090000000E00007003200CE00900025
:10E6A000F0F92000808F500003003E002E00900003
:10E6B0000000E800200798006011B8001E00BE00AE
:10E6C0004A040200000000000000E00001003C00DD
:10E6D0000B00370002002000832C24001E00BE0027
:10E6E0004E040200000000000000E00001003500C0
:10E6F000030037002E0090000000E800200798007B
:10E700002E009000E20F5000110032000000EB00DC
:10E710006069880011012000802F20004E9A0200BD
:10E72000000000001101200090302000C499020078
:10E73000000000008001EB0002FA20001100200020
:10E7400020032000901C02000000000040079800F9
:10E750004E009000E30F500005003E00E003200053
:10E760003007980010A1A8001081A80015003700FC
:10E770004E009000FE0F500005003E00A00F20004C
:10E780003007980010A1A8001081A9000D003700E3
:10E79000CE009000400F2000808F500005003E000A
:10E7A000007D20003007980010A1A9001081A8006A
:10E7B0000400370000E823003007980010A1A900EA
:10E7C0001081A9003E0090004E0190001100090048
:10E7D0000280D8000000E900600798002E00900039
:10E7E000E20F50000E0032000101200070322000C4
:10E7F000C4990200000000008001EB0032062000F6
:10E800008000EB0020032000901C020000000000AC
:10E81000CF80DE00F403020000000000008FBE0085
:10E8200002002000832C24001E00BE0052040200BF
:10E8300000000000008FBE006E009000CF80DE0060
:10E84000F40302000000000070079800010F980018
:10E850006E0090000000E00008003D000200200073
:10E86000037824007E0090008E089000D8040200F7
:10E870000000000070079800010F98001E01BE0004
:10E880007E0090008E0890009205020000000000BB
:10E89000FA0502000000000050079800A16C20005B
:10E8A0009140780000CEB30000C060006041B3002A
:10E8B000CAE6B7005E009000D00C88005E009000B1
:10E8C000C00C880060002000E00C88006E00900002
:10E8D0006008880011E1A800A1002000703320002A
:10E8E0004E9A02000000000020002000B060880066
:10E8F0000080FA00000006000000FA00B06080000E
:10E90000E20F500005003A00F10120001034200011
:10E910004E9A0200000000003E003700F100200087
:10E9200000362000C4990200000000000000EB0047
:10E93000F00888000000EB0080088800C942A800A9
:10E94000616820009140780000CEB30000C06000F4
:10E95000A040B30086E6B700A0032000800888002E
:10E960002E000700C0608800D1608800C26080006F
:10E97000D3608000F00F200001002000800F5100C4
:10E98000818F590009003600C0608000D16080008E
:10E99000C808DD000080FD00804078000040EB00EA
:10E9A000C0608800D160880009003700B1002000F5
:10E9B000B0192100C499020000000000A00020004E
:10E9C0008008880015000700C0608800D1608800BA
:10E9D000C0608000D1608000D66D020000000000A1
:10E9E00020A32800B06C02000000000060A32800F3
:10E9F000DC6C02000000000086C6BF00F041B300DE
:10EA000086E6B7000000EB00F00888000000EB008D
:10EA1000800888000080FA00000006000000FA006C
:10EA20000080EB00700888000080EB006008880020
:10EA30000000EB00400888000000EB003008880070
:10EA40000000EB00B00888000000EB00A008880080
:10EA500080002000F0088800400F2000E0088800B7
:10EA600000402200D00888008780A9001FE1A8008C
:10EA700011E1A80087C0BF00704060000004E00002
:10EA8000FCFF320011E1A9001FE1A900300880005D
:10EA900010618800400880000061880000618000EB
:10EAA00001002000E0608800F1608800E0608000E4
:10EAB000F1608000C000DD0000002000E060880000
:10EAC000F1608800106180006101B800E0608000A2
:10EAD000F16080000200400083804800E060880010
:10EAE000F1608800E0608000F16080000080FA0042
:10EAF000000006000000FA0070B720001040780007
:10EB0000614060000004E00002003A00C942A80031
:10EB100001003700C8C2A800E1002000F036200044
:10EB2000C4990200000000000080FA000000060006
:10EB30000000FA0070B720001040780061406000CB
:10EB40000004E00003003A00C942A900CB42A8003B
:10EB500002003700C8C2A900CAC2A8008100200074
:10EB6000D03720004E9A0200000000000080FA001A
:10EB7000000006000000FA0070B720001040780086
:10EB8000614060000004E00003003A00C942A900AF
:10EB9000CB42A90002003700C8C2A900CAC2A9001E
:10EBA00071002000503820004E9A02000000000042
:10EBB0000080FA00000006000200FA0070B7200092
:10EBC00010407800614060000004E00009003A0055
:10EBD000C942A8000000000000000000CBC2BF0036
:10EBE0000080FB004200DE0061406000004F7800C2
:10EBF00008003700C8C2A8000000000000000000A4
:10EC0000CAC2BF000080FB004600DE006140600019
:10EC1000004F78001E80FB000080FA000000060014
:10EC20000E00FA000040EB00404798000000EB00A7
:10EC3000800888000000EB00F00888000000EB006E
:10EC4000E00C8800B0608000E20F500014003A0031
:10EC5000A16C20009140780000CEB30000C060009D
:10EC6000CAE6B700C1002000C02E20004E9A020064
:10EC7000000000000000EB00B060880050698000D8
:10EC80008000E800F00F20008080600080C220003B
:10EC900000804000104078000004E000670032006F
:10ECA000506980000000E8005069880051698000C8
:10ECB000F00F200000806000506988001A1A0200DE
:10ECC000000000004416020000000000CF80DE00BB
:10ECD000F403020000000000008FBE0002002000CC
:10ECE000533324001E00BE004E040200000000004A
:10ECF0000000E00001003500030037004E409000A6
:10ED00000040E8004047980010A1A8001081A8002A
:10ED1000204E2000400798004E409000E14F5000E8
:10ED20000E0032000101200070322000C499020060
:10ED3000000000008001EB00420B20008000EB008F
:10ED4000A0052000901C020000000000CF80DE0023
:10ED5000F403020000000000008FBE0002002C003F
:10ED6000A35524001E00BE00520402000000000053
:10ED7000008FBE004E009000CF80DE00F403020042
:10ED80000000000050079800610798004E009000B6
:10ED90000000E00008003D0002002000037824008D
:10EDA0005E009000EE009000D80402000000000019
:10EDB00050079800610798001E01BE005E00900099
:10EDC000EE0090009205020000000000020020000A
:10EDD00083272400D804020000000000FA05020086
:10EDE0000000000030079800A16C200091407800DE
:10EDF00000CEB30000C060006041B300CAE6B700B7
:10EE00003E009000D00C88003E009000C00C8800AE
:10EE100060002000E00C88004E0090006008880030
:10EE200011E1A800A1002000703320004E9A0200DA
:10EE30000000000020002000B06088000080FA0080
:10EE4000000006000000FA00E0A32800B06C0200F9
:10EE5000000000000080FA00000006000200FA0036
:10EE6000CA82A800E0000700F6FF07000000370094
:10EE7000D40007008040780060DE20000148780060
:10EE800060DE2000104078000004E000C70035007C
:10EE900060DE2000104078000004E00002003A002C
:10EEA000E8FF0700F2FF370060DE20001040780026
:10EEB000E14F500006003A00CB000700564902001F
:10EEC00000000000C8000700DEFF0700E8FF370071
:10EED00060DE200010407800E24F500006003A004B
:10EEE000C1000700FA6A020000000000BE0007002F
:10EEF000D4FF0700DEFF370060DE200010407800FE
:10EF0000E34F500006003A00B70007000852020025
:10EF100000000000B4000700CAFF0700D4FF37005C
:10EF200060DE200010407800E44F500006003A00F8
:10EF3000AD000700FE5C020000000000AA00070010
:10EF4000C0FF0700CAFF370060DE200010407800D5
:10EF5000E54F500006003A00A3000700E25E020001
:10EF600000000000A0000700B6FF0700C0FF370048
:10EF700060DE200010407800E64F500006003A00A6
:10EF800099000700BE8C02000000000096000700F8
:10EF9000ACFF0700B6FF370060DE200010407800AD
:10EFA000E74F500004003A008F0007008E00070072
:10EFB000A4FF0700AEFF370060DE2000104078009D
:10EFC000EF4F50000A003A0010C0B3000C7102006D
:10EFD00000000000CA82A90023C2BF006140600097
:10EFE0000004E000FCFF32000000FE00A0FF37003C
:10EFF00060DE200010407800F24F500035003A00EB
:10F000000000EB00800888000000EB00F00888009A
:10F010000000EB00E00C8800A16C2000914078001B
:10F0200000CEB30000C060006041B300CAE6B70084
:10F03000640007000080FB00000F78001E007800CD
:10F040000000D100610060000004E0000100320017
:10F0500010A1A8009E007800618060000004E0001C
:10F06000010032001081A800560007000080FB005C
:10F070004800DD00000F7800520007000080FB0010
:10F080001E0F70001E007800D00C88009E007800D3
:10F09000C10C880060002000E00C880049000700D7
:10F0A0000080FB004800DD00000F780045000700ED
:10F0B0000080FB001E0F70001E00780060088800B2
:10F0C00011E1A80010C0B3000C71020000000000A4
:10F0D00067FF370060DE200010407800F34F5000DB
:10F0E0000D003A000000EB00800888000000EB00F3
:10F0F000E00C8800A16C20009140780000CEB300A5
:10F1000000C06000CAE6B70010C0B3000C71020076
:10F110000000000056FF370060DE2000104078003D
:10F12000F44F50000E003A0021E3A800C0C0B30025
:10F13000E495020000000000000F780021E3A90020
:10F140001E0078004800DE000C7102000000000084
:10F150001E0078000C7102000000000044FF370020
:10F1600060DE2000104078000080FB004500DE00DB
:10F170000080FB000000D100610060000004E0009E
:10F180000600320060DE2000104078001F000700FB
:10F190000C7102000000000035FF37000040EB005A
:10F1A0000C7102000000000031FF370060DE20001B
:10F1B00010407800A50007000C710200000000005C
:10F1C0002BFF37000000FA0022C2BF006140600040
:10F1D0000004E000FCFF3200301180000080FB00E2
:10F1E0000080FA00000006000000FA0000C0EB00FA
:10F1F000060007000040EB0094000700C962A90068
:10F20000CB62A9000080FA00000006000400FA00AA
:10F21000204798000040EB00004F78002E409000FF
:10F220000080FB004400DE00610060000004E0009C
:10F230000200320010C0B300004F78009E407800FA
:10F2400061C06000614060004201DD00912C20003F
:10F2500091407800B0CFB30000C060000240700061
:10F26000C9E2B7000040EB00004F78002E4090004C
:10F270000080FB004300DE00610060000004E0004D
:10F280000200320010C0B300004F78009E407800AA
:10F2900061C060006140600000414000912C20008E
:10F2A00091407800D0CFB30000C0600002407000F1
:10F2B000C9E2B7000040EB00004F78002E409000FC
:10F2C0000080FB004200DE00610060000004E000FE
:10F2D0000200320010C0B300004F78009E4078005A
:10F2E00061C0600061416000912C20009140780075
:10F2F000E0CFB30000C0600002407000C9E2B70078
:10F300000040EB00004F78002E4090000080FB0092
:10F310000000D100610060000004E0000200320043
:10F3200010C0B300004F78009E40780061C06000BC
:10F33000C700DD00C8C2BF000074A100014070001A
:10F34000C8E2B7000040EB00004F78002E4090006C
:10F350000080FB00610060000004E0000200320059
:10F3600010C0B300004F78009E40780061C060007C
:10F37000614060004601DD00812C20009140780052
:10F38000F0CBB30000C0600002407000C8E2B700DC
:10F39000500020004E97020000000000AE40900098
:10F3A00000CEB30000C0600020479800CBC2BF0071
:10F3B000644060000004E000030032002E40900032
:10F3C0000044A00020479800CBC2BF00624060000C
:10F3D0000004E000030032002E4090000034A00042
:10F3E00020479800CBC2BF00614060000004E000ED
:10F3F000030032002E4090000024A0002047980017
:10F40000CAC2BF0001C8B300014060000004E000B0
:10F41000030032002E4090000014A0002047980006
:10F42000CAC2BF000044B2000004E0000300320082
:10F430002E4090000004A000204798002E4090002D
:10F440000080FB000080FA00000006000400FA00C3
:10F45000204798002E4090000080FB004600DE0010
:10F46000610060000004E00005003200C082A900D5
:10F47000C282A800C8A2A900CAA2A800040037003E
:10F48000C082A900C282A900C8A2A900CAA2A9007C
:10F490000040EB00004F78002E4090000080FB0001
:10F4A0004400DE00610060000004E0000200320061
:10F4B00010C0B300004F78009E40780061C060002B
:10F4C000614060004201DD00B12C200091407800D5
:10F4D000B0CFB30000C0600002407000CBE2B700C4
:10F4E0000040EB00004F78002E4090000080FB00B1
:10F4F0004300DE00610060000004E0000200320012
:10F5000010C0B300004F78009E40780061C06000DA
:10F510006140600000414000B12C20009140780023
:10F52000D0CFB30000C0600002407000CBE2B70053
:10F530000040EB00004F78002E4090000080FB0060
:10F540004200DE00610060000004E00002003200C2
:10F5500010C0B300004F78009E40780061C060008A
:10F5600061416000B12C200091407800E0CFB300F1
:10F5700000C0600002407000CBE2B7000040EB002A
:10F58000004F78002E4090000080FB000000D1006A
:10F59000610060000004E0000200320010C0B3000F
:10F5A000004F78009E40780061C06000C700DD0019
:10F5B000CAC2BF000074A10001407000CAE2B700D7
:10F5C0000040EB00004F78002E4090000080FB00D0
:10F5D000610060000004E0000200320010C0B300CF
:10F5E000004F78009E40780061C06000614060007C
:10F5F0004601DD00A12C200091407800F0CBB30043
:10F6000000C0600002407000CAE2B7005000200055
:10F610004E97020000000000AE40900000CEB30004
:10F6200000C0600020479800CBC2BF00644060006B
:10F630000004E000030032002E4090000044A000CF
:10F6400020479800CBC2BF00624060000004E00089
:10F65000030032002E4090000034A00020479800A4
:10F66000CBC2BF00614060000004E0000300320034
:10F670002E4090000024A00020479800CAC2BF007E
:10F6800001C8B300014060000004E0000300320044
:10F690002E4090000014A00020479800CAC2BF006E
:10F6A0000044B2000004E000030032002E4090004D
:10F6B0000004A000204798002E4090000080FB002E
:10F6C0000080FA00000006000000FA0070B7200079
:10F6D000104078000030A00071B72000804878000A
:10F6E000960007000080FA00000006000000FA0003
:10F6F0003C010700530007007027210010407800EC
:10F700000080FB000080FA00000006000400FA0000
:10F71000100798001E00900071010700004F78004C
:10F720001E04E00005003A003100200010442000D3
:10F73000C4990200000000000C00370010C0B300A4
:10F740009E4F100005003A00410020004044200078
:10F75000C49902000000000004003700810020006E
:10F7600000122100C49902000000000000102000D7
:10F770000080FA00000006000400FA00000F780084
:10F780001E007800100798001E0090000000E000A6
:10F79000040032001E009000E10F5000060032000D
:10F7A0002200370061022000801221004E9A0200E0
:10F7B0000000000021003700D1002000E0142100EB
:10F7C0004E9A020000000000F1002000C01E21003F
:10F7D0004E9A020000000000020107000004E00051
:10F7E00008003A0070272100104078000080FB00DC
:10F7F0009C9602000000000000C2B3000C710200E1
:10F800000000000022C2BF00614060000004E00070
:10F81000F1FF320030118000000F780000A62800B0
:10F82000DC6C0200000000000400370041022000F0
:10F83000C02020004E9A0200000000000080FA0064
:10F84000000006000400FA00004F78001E80FB0054
:10F85000100798009E009000E28F50001A003200BE
:10F860001E009000E20F500007003C009E00900038
:10F870000100E0002F0032001E009000E10F500058
:10F880000C003200270037009E009000E48F5000EB
:10F89000170032001E009000E40F50000F003500EA
:10F8A000F00F20009E009000808F50001800320062
:10F8B0001C00370001012000B01521004E9A020003
:10F8C000000000001B003700E1002000B0162100FE
:10F8D0004E9A02000000000016003700F1002000E0
:10F8E000901721004E9A020000000000110037001E
:10F8F00000C2B3000C710200000000008100200073
:10F9000000122100C4990200000000000900370025
:10F9100051002000801821004E9A020000000000D3
:10F9200004003700E1002000D01821004E9A0200A8
:10F93000000000000080FA00000006000000FA004D
:10F94000C922A800C902A900CB02A900CB22A900A4
:10F950000080FA00000006000400FA000040EB00FE
:10F96000410107000004E0000300320020002000F5
:10F97000100798000E003700CBC2BF000080FB00CC
:10F980000000D10061406000004F780010C0B3005B
:10F99000350107000004E0000300320020002000D1
:10F9A00010079800020037001E80FB001007980027
:10F9B0001E0090000080FA00000006000600FA0019
:10F9C0000040EB00204798000040EB0010479800F3
:10F9D000CBC2BF000080FB000000D100E14060000E
:10F9E000602721001040780061C16000E1CFB300C2
:10F9F00001406000024070006127210080487800CB
:10FA00006027210010407800614060000004E000A1
:10FA10000300320010002000200798006E0037001D
:10FA200010C0B300100107000004E0000300320022
:10FA30004100200021079800670037000040EB00DC
:10FA400030479800190037001E4090000080FB00EE
:10FA50000000D10010479800BFFF0700004F78005A
:10FA600020C0B3009E4F100003003A004100200068
:10FA7000210798005800370010C0B3009E4F1000B7
:10FA800007003A009E40900000C8B30000C040004C
:10FA9000104798002E4090000004A20020479800D4
:10FAA0003E4090000040E800304798003E40900003
:10FAB000E74F5000E4FF3600702721009E40900081
:10FAC00001487800A4FF0700004F780020C0B30071
:10FAD0009E4F100003003A004100200021079800CB
:10FAE0003D0037001E407800E14060008027210083
:10FAF0001040780061C16000E1CFB30001406000B8
:10FB00000240700081272100804878008027210072
:10FB100010407800614060008080FB002E40900023
:10FB20000080FB00808F500008003A0080272100F1
:10FB3000104078000020A000812721008048780034
:10FB40002100200021079800230037008027210092
:10FB5000104078000020A100812721008048780013
:10FB60007DFF0700004F780020C0B3009E4F1000BB
:10FB700003003A00410020002107980016003700DA
:10FB80001E4078006141600080272100904078008D
:10FB90006140610000414000D0CFB30080C06000F0
:10FBA00082C070008027210001487800C902A900A6
:10FBB0008027210010407800624060000004E000CF
:10FBC00003003A00310020002107980002003700AE
:10FBD0000000EB00200798002E0090000080FA0043
:10FBE000000006000200FA0000C0EB00004F7800A1
:10FBF000C922A800C902A8000040EB0010479800E5
:10FC000011003700CBC2BF00614060000004E0007B
:10FC100007003A0069FF0700004F78001E04E0006B
:10FC20000C00320040C0B3009E4F100009003200AB
:10FC3000500020004E970200000000001E4090007F
:10FC40000040E800104798001E409000E14F40003F
:10FC5000ECFF3A00C902A9001E80FB000080FA00F8
:10FC6000000006000400FA00004F780010C0B30046
:10FC70007D0007000004E0000300320020002000A7
:10FC800010079800130037009E40780061C06000A4
:10FC90006140600000414000912C200091407800BC
:10FCA000D0CFB30000C0600002407000C9E2B700CE
:10FCB0000040EB006C0007000004E000030032008D
:10FCC0002000200010079800020037008000EB00A1
:10FCD000110798001E0090000080FA000000060046
:10FCE0000800FA00404798000040EB0020479800C9
:10FCF000C902A900CB02A900C00320004E97020050
:10FD000000000000CB22A900C922A900C902A80056
:10FD1000100020004E970200000000000040EB00A1
:10FD2000510007000004E000030032004000200002
:10FD300030079800490037000000EB00000F780002
:10FD40001C0037004E4090000080FB006100600006
:10FD50000004E0000B00320010C0B300C1FF070038
:10FD60000004E0000300320040002000300798004B
:10FD70003A0037002E4090000004A200204798006F
:10FD8000070037000040EB00B6FF07000004E0006A
:10FD90000300320040002000300798002F00370099
:10FDA0004E4090000080FB000000D10040479800CA
:10FDB0001E0FE800700020009E0F1000E1FF3600CB
:10FDC0002E4090000004A200204798002E40900092
:10FDD000A4FF07000004E000030032004000200000
:10FDE000300798001D003700C922A800CB22A900C7
:10FDF00010C0B3001C0007000004E0000300320044
:10FE0000400020003007980014003700D2FE0700A1
:10FE1000E24F500003003A004000200030079800F5
:10FE20000E003700CCFE07000080FB00000F7800BA
:10FE3000200020009E0F100003003A004000200028
:10FE40003007980005003700C902A900CB02A900BD
:10FE50001E0078000080FB00300798003E009000F4
:10FE60000080FA00000006000600FA002047980013
:10FE70000080EB00000F7800CBC2BF006140600043
:10FE80008080FB002E4090000080FB00808F50009F
:10FE900003003A000000EB0020079800050037003F
:10FEA0001E0FE9001E00E000F3FF3A0010002000E2
:10FEB000200798002E0090000080FA000000060045
:10FEC0000400FA00004F780011479800C0DD2000C0
:10FED0001E48780030C0B3009E4F100005003A0065
:10FEE00000202000F06E880000082000006F8800CD
:10FEF0000400370000202000F06E88000020200061
:10FF0000006F88001E4090000080FB0010079800E2
:10FF10001E009000E10F5000110032001E00900002
:10FF2000E20F5000180032001E0090000000E000B8
:10FF3000010032001E00370041C1B30020DE200066
:10FF40000148780041C6B30030DE20000148780047
:10FF500021C3B30040DE2000014878001D003700B7
:10FF600021C0B30020DE200001487800A1C0B3000A
:10FF700030DE20000148780051C0B30040DE200090
:10FF8000014878001300370011C0B30020DE2000C4
:10FF90000148780051C0B30030DE200001487800ED
:10FFA00021C0B30040DE200001487800090037007E
:10FFB0008040EB0020DE2000014878008040EB000C
:10FFC00030DE2000014878008040EB0040DE200059
:10FFD000014878000080FA00000006000200FA00E4
:10FFE0000000EB00000F780030DE20009040780029
:10FFF0000030200009010700CBC2BF006140600053
:020000040001F9
:100000000004E00004003200CBC2BF006240600088
:100010000004E00002003A0010002000000F780009
:1000200030DE2000904078000020200017010700FB
:1000300030DE2000904078000010200013010700FF
:1000400030DE20009040780000202000F300070000
:100050001E0078000080FA00000006000000FA0090
:1000600030DE2000904078000030200007010700BB
:1000700030DE20009040780000102000E7000700EC
:1000800030DE20009040780000202000E3000700D0
:100090000000EB000080FA00000006000C00FA00EF
:1000A000500798000000EB00000F780080B7200098
:1000B000104078000080FB008000E9001000200064
:1000C0000100DD00300798005E00900020079800D6
:1000D0000000EB00400798002000370020DE2000E1
:1000E00010417800AE0090003E009000008060005B
:1000F00001202000FC00070030DE20009040780046
:1001000000102000C500070000082000260107009D
:100110000080FB001007980030DE2000904078003F
:1001200000102000D90007002E00900000004000C1
:10013000200798001E00780000004000000F7800A3
:100140001E0090000000E000010032001E0FE800D9
:100150004E0090000000E8004007980080B72000A3
:10016000104078008080FB004E009000808F50008F
:10017000DAFF3E001E0078000080FA000000060052
:100180000800FA003007980080B72000104078007F
:100190000080FB008000E900100020000100DD006D
:1001A000100798003E009000000F78000000EB0060
:1001B000200798001400370020DE2000104178004E
:1001C0001E0090001E00600001202000C6000700F5
:1001D00030DE200090407800001020008F000700E3
:1001E00030DE20009040780000102000A7000700BB
:1001F0001E00780000004000000F78002E009000E4
:100200000000E8002007980080B720001040780028
:100210008080FB002E009000808F5000E6FF3E00A3
:100220000080FA00000006000600FA000000EB0063
:10023000000F780000202000DB0007000000EB002A
:10024000200798001600370030DE2000904078002C
:10025000001020007100070000202000D2000700DD
:100260000080FB001007980030DE200090407800EE
:1002700000102000850007001E00780000004000EC
:10028000000F78001E0090000000E0000100320026
:100290001E0FE8002E0090000000E80020079800E4
:1002A00080B72000104078008080FB002E00900076
:1002B000808F5000E4FF3E001E0078000080FA00AE
:1002C000000006000200FA00006F8000B600070080
:1002D00030DE200090407800001020004F00070022
:1002E000006F8000B0000700004F780030DE200073
:1002F0009040780000102000640007001E80FB0082
:100300000080FA00000006000200FA00004F7800AA
:1003100020DE200010417800F16E80001E80FB007E
:100320007100070030DE20009040780000102000AF
:100330003A00070030DE20009040780000102000D6
:10034000520007000080FA00000006000400FA00D6
:10035000204798000040EB00004F7800090037006C
:1003600030DE200090407800001020002B000700B5
:1003700030DE20009040780000102000430007008D
:100380001E4FE8002E4090009E4F1000F4FF3900F1
:100390000080FA00000006000200FA00004F78001A
:1003A00020DE200010417800F16E80001E80FB00EE
:1003B0004D0007000080FA00000006000200FA006D
:1003C000004F780020DE2000104178001E80FB00E6
:1003D00001102000440007000080FA000000060021
:1003E0000200FA00004F780020DE20001041780063
:1003F0001E80FB00010420003B0007000080FA0083
:10040000000006000000FA00006F80006600070090
:100410000080FB000080FA00000006000400FA00E3
:10042000000F78002147980070B720001040780036
:10043000684060000004E0000B003A006016800095
:100440001E007000601688001E0078000080EA0020
:100450008180EA0080007800401680000080600003
:100460004016880003003700401680001E00700010
:10047000401688002E4090000080FB004E9702003E
:10048000000000000080FA00000006000400FA00EE
:10049000000F7800214798001E0078000080EA00D5
:1004A0008180EA0080007800601680000080600093
:1004B000601688001E0078000080EA008180EA0053
:1004C00080007800401680000080600040168800A0
:1004D0002E4090000080FB004E97020000000000BC
:1004E0000080FA00000006000600FA00000F780005
:1004F00011079800424798001E00E0000F003A00E4
:100500001E0090000080EA008180EA0080007800F0
:100510006016800000806000601688001E00900059
:100520000080EA008180EA008000780040168000A8
:1005300000806000401688001500370070B720006A
:1005400010407800684060000004E0000C003A00B1
:10055000611680001E009000008070006016880008
:100560001E0090000080EA008180EA008000780090
:1005700040168000008060004016880004003700AC
:10058000401680009E009000010070004016880018
:100590004E4090000080FB004E97020000000000DB
:1005A0000080FA00000006000400FA00000F780046
:1005B000401680001E0070004016880000000000F9
:1005C0000000000000000000501680001E006000C7
:1005D0000000E00003003200100020001007980027
:1005E000020037000000EB00100798001E0090008A
:1005F0000080FA00000006000000FA0014810200EA
:10060000000000000080FA00000006000200FA006E
:10061000000F78001E007800C0800200000000007B
:10062000001020000080FA00000006000000FA0020
:10063000EE7F02000000000081002000D092200028
:10064000C499020000000000D10020008044200076
:100650004E9A0200000000000080FA000000060030
:100660000000FA002E80020000000000610020005F
:1006700050932000C499020000000000C100200037
:10068000504520004E9A0200000000000080FA0051
:10069000000006000000FA00628102000000000075
:1006A0000080FB000080FA00000006000000FA0055
:1006B00002820200000000000080FB000080FA00BF
:1006C000000006000000FA000040EB00DE8102009E
:1006D000000000000080FA00000006000000FA00A0
:1006E00010C0B300DE810200000000000080FA00AC
:1006F000000006000000FA0010C0B300A68102004E
:10070000000000000080FA00000006000000FA006F
:100710000040EB00CC810200000000000080FA00E5
:10072000000006000000FA0010C0B300CC810200F7
:10073000000000000080FA00000006000000FA003F
:1007400001012000A0982000C499020000000000D0
:1007500060B7200010407800486F020000000000E1
:1007600000C2B3000C7102000000000070B720004E
:10077000104078000080FB004300DE006140600014
:10078000486F02000000000000C2B3000C710200BC
:100790000000000031002000F0AD2000C4990200EC
:1007A000000000000080FA00000006000400FA00CB
:1007B0001A1A0200000000004416020000000000A7
:1007C000100798001A1A02000000000044160200E8
:1007D00000000000000F78001E0090000000E00004
:1007E000090034001E009000E40F500006003C0099
:1007F0001E0090000040E9008040780060B72000B3
:1008000001487800020037000000EB001007980054
:100810001E00E00010003400200020009E0F100099
:100820000D003C001E0078000040EA0061416000BD
:1008300070B7200090407800614061004301DD0006
:1008400070CFB30080C0600082C0700070B720001D
:1008500001487800020037000000EB001007980004
:100860001E0090000000E00026003A000000EB00AF
:1008700060698800B1032000604820004E9A0200A1
:10088000000000008001EB00420020001100200069
:1008900010002000901C0200000000000040E90051
:1008A0008040780060B7200001487800F104200003
:1008B000B09320004E9A0200000000008001EB007F
:1008C000220020001100200010002000901C0200D7
:1008D000000000000040EA006141600070B72000A5
:1008E00090407800614061004301DD0070CFB300AB
:1008F00080C0600082C0700070B72000014878009E
:10090000010037008DFF0700CB02A900CB22A90010
:10091000C922A800C902A90060B720009040780051
:1009200020C0B300607F0200000000000080FA00D9
:10093000000006000400FA00000F78001E00780096
:10094000100798001E009000E10F50000C003200CC
:100950001E009000E10F5000040039001E009000BE
:10096000E20F50000700320008003700810320002A
:10097000A0992000C4990200000000000700370081
:100980001000070025000700040037004102200086
:10099000C02020004E9A0200000000000080FA00F3
:1009A000000006000200FA00000F7800B1002000ED
:1009B000C00921004E9A0200000000000080FA00E9
:1009C000000006000000FA00F1032000209D200036
:1009D0004E9A0200000000000040EB00F08102008F
:1009E00000000000F00F20004E9702000000000001
:1009F00010C0B300F08102000000000010C0B3007E
:100A0000A6810200000000000040EB00F08102001F
:100A1000000000000080FA00000006000A00FA0052
:100A2000881F7800D102200010A12000C499020084
:100A3000000000000000EB00000F780010003700FD
:100A40001E0478001481020000000000804078003D
:100A500063004700017478009E007800630047003F
:100A6000614078000080FB00AA6F020000000000D7
:100A700000C2B3000C710200000000001E0FE8006D
:100A8000300020009E0F1000EDFF360080A52800EA
:100A9000DC6C020000000000A1002000E0A32000A8
:100AA000C499020000000000630047001040780075
:100AB0000080FB004400DE000080FB00400798003F
:100AC0004E009000E90F5000130032004E009000DD
:100AD000E90F500004003C004E009000E80F500069
:100AE000080032001B0037004E009000EA0F500053
:100AF0000E0032004E009000EF0F50001000320048
:100B0000140037006100200080A42000C499020076
:100B1000000000001300370061002000E0A4200066
:100B2000C4990200000000000E00370061002000A0
:100B300040A52000C4990200000000000900370011
:100B400031002000A0A52000C49902000000000090
:100B50000400370071002000D0A52000C4990200D5
:100B60000000000080A52800DC6C020000000000EE
:100B7000B100200040A62000C4990200000000003F
:100B800063004700104090000080FB004700DE003B
:100B90000004E00005003A0061002000F0A62000FB
:100BA000C49902000000000004003700F10020009A
:100BB00050A72000C49902000000000080A5280072
:100BC000DC6C020000000000C100200040A82000F2
:100BD000C49902000000000063004700104090002C
:100BE0008080FB0080F72F00008060004380DE00E3
:100BF000204798002E4090000004E00005003A00D5
:100C0000D100200000A92000C499020000000000CB
:100C10001E0037002E409000EF4F500005003A00B4
:100C200031002000A0A52000C499020000000000AF
:100C30001600370000042000000F7800E300470092
:100C40000040EB0080487800080037001E00780064
:100C500000004000000F780063004700104078005B
:100C60008040E800630047000148780063004700C7
:100C7000904078002E40900080CF5000F3FF390064
:100C80001E007800EA6E02000000000080A5280027
:100C9000DC6C02000000000091012000D0A92000BF
:100CA000C4990200000000006300470090409000DB
:100CB00070C0B30000C06000204798001000200002
:100CC000000F7800E30047000040EB008048780008
:100CD000080037001E00780000004000000F780078
:100CE00063004700104078008040E8006300470040
:100CF0000148780063004700904078002E40900043
:100D000080CF5000F3FF39001E007800486F0200CA
:100D10000000000080A52800DC6C0200000000003C
:100D20004F0478000080FA00000006000000FA007E
:100D300040168000017C20000100700040168800F1
:100D40001100070020C0B3002D000700EE70020064
:100D5000000000000004E00005003200FA7002000C
:100D600000000000260007000004E00004003A0034
:100D7000360107000004E00001003A00F3FF3700ED
:100D80000080FA00000006000000FA00CA82A900F4
:100D90000000EB00400388000000EB0050038800D7
:100DA0000000EB00000388000000EB001003880047
:100DB0000000EB00F0088800D10A20009140780084
:100DC000F0C8B30000C06000ADE0B7000000EB0069
:100DD000E008880000642000D0088800000021009E
:100DE000507088008040EB0080E0200001487800CF
:100DF0000000EB00B06F88000080FA0000000600E1
:100E00000A00FA00004F7800007080004007980048
:100E1000CE009000E18F5000440032004E0190005F
:100E2000E10F5100040039004E009000E20F500025
:100E30004F003200000137009E80FB003107980010
:100E40003E019000E20F5100150032003E0090007C
:100E5000E20F500007003C00BE0090000100E000DF
:100E60000B0032003E019000E10F510010003200F3
:100E7000230037003E009000F10F5000EE003200DA
:100E8000BE009000F38F5000EB0032001C003700D2
:100E9000BDFF07001200200022079800E80037007D
:100EA000A0A42800B06C020000000000E20037009F
:100EB000CA82A8000000EB00F00888000000EB00E8
:100EC000B00888000000EB00A00888008000200027
:100ED000F00888008660A9009660A900D10A200069
:100EE00091407800F0C8B30000C060000044A0004A
:100EF000ADE0B70010002000B06F8800CE003700D2
:100F000080DF20001E48780041C0B300D0DF200001
:100F1000014878008040EB00E0DF200001487800C5
:100F20001000200000708800C3003700E0DF2000C0
:100F3000104078008040E800E0DF200001487800A1
:100F4000E0DF2000104078008080FB0080DF200080
:100F5000008040001E487800E0DF200090407800CC
:100F6000D0DF20001040780080CF5000B200390060
:100F700080DF2000104078000080FB001007980000
:100F8000100820009E009000808F50003E0032002C
:100F9000000C20001E019000800F5100050032005F
:100FA000000820009E009000808F50004E0032000C
:100FB0009F00370090DF2000104078000080FB0089
:100FC0004400DE00610060000004E0000300320025
:100FD000100380000000A0001003880090DF2000B4
:100FE000104078000080FB004300DE0061006000DC
:100FF0000004E00004003200100380000102200021
:10100000010070001003880090DF2000104078007D
:101010000080FB004200DE00610060000004E00090
:101020000400320010038000010420000100700061
:101030001003880090DF2000104078000080FB0043
:101040000000D100610060000004E00004003200F4
:1010500010038000010820000100700010038800C8
:1010600090DF2000104078000080FB0061006000ED
:101070000004E00004003200100380000110200092
:101080000100700010038800A0DF200010407800ED
:101090000080FB0050708800507080004800DD0028
:1010A0005070880090DF2000104078008080FB00A6
:1010B0005070800000807000507088005070800078
:1010C0004200DD00640040005070880051708000D4
:1010D00000002100808F50005500360000002100E4
:1010E0005070880052003700B0DF200010407800B8
:1010F0000080FB0001002000107088002170880033
:101100001070800021708000C808DD000080FD00A4
:10111000804078000040EB0010708800217088004B
:10112000A0DF2000104078000081FB0003002000B9
:1011300010708000217080000000710081807100BB
:10114000107088002170880010708000217080006D
:10115000C808DD000080FD00804078000040EB0002
:10116000107088002170880090DF20001040780007
:101170000081FB00030020001070800021708000BF
:10118000000071008180710010708800217088005B
:1011900010708000217080004209DD00CE00DE006A
:1011A000810071004200DD0064004000E0804800E2
:1011B0009201200003002000300602000000000021
:1011C00010708800217088001270800023708000E9
:1011D0000001200001002000800F5100818F590084
:1011E00007003600107080002170800070005000F1
:1011F000E0805800107088002170880004003700DB
:10120000100020000100200010708800217088006C
:1012100010708000217080004008DE000100200076
:10122000E00888001070800021708000D0088800DD
:101230000000EB00007088000000EB002007980021
:101240002E0090000080FA00000006000200FA0064
:10125000B06F8000E10F500001003200360037000F
:1012600086C0BF00684060000004E00003003A0050
:10127000100380000000E0002F003A001FE1A800EA
:101280008780A9000000EB00307088000E00370056
:1012900071408000307080008080400050168000D7
:1012A0004600DE008048780087C0BF0070406000C4
:1012B0000004E000FCFF32008780A900307080004D
:1012C0000000E800307088003170800050708000AD
:1012D000808F5000EEFF39000000EB001003880003
:1012E0000000EB00F008880050708000307088002B
:1012F0000A0037007140800030708000008040009C
:101300000000E900104078000C71020000000000AD
:10131000307080000000E90030708800307080007C
:101320000000E000F3FF3A0097FE070010002000E5
:10133000000F7800020037000000EB00000F78007B
:101340001E0078000080FA00000006000200FA008B
:10135000000F78001E0078008040780040272100B0
:10136000104078000080FB000000D1006140600068
:1013700046010700001020000080FA00000006006F
:101380000000FA0040272100104078000010A10062
:10139000412721008048780041012000B0EC200066
:1013A0004E9A0200000000000080FA0000000600D3
:1013B0000000FA0040272100104078000010A00033
:1013C000412721008048780021012000F0ED200015
:1013D0004E9A0200000000000080FA0000000600A3
:1013E0000000FA0070B72000104078000030A00024
:1013F00071B7200080487800402721001040780015
:101400000010A0004127210080487800816A200058
:101410009140780000CEB30000C060007040B3007F
:10142000A8E6B700916C20009140780000CEB30090
:1014300000C060007040B300C9E6B700816C2000B6
:101440009140780000CEB30000C060000034A000DE
:10145000C8E6B700CAC2A900C8C2A900C902A9004B
:10146000C8E2A800C922A900D013200010128800E9
:101470000000EB00201288000000EB000012880042
:1014800041E2A800D101200040F020004E9A020065
:10149000000000000080FA00000006000800FA00CA
:1014A00020079800506980000000E800506988001B
:1014B00051698000F00F20000080600050698800B2
:1014C0001A1A02000000000044160200000000008A
:1014D000100798000000EB00606988002E00900063
:1014E000300798003E009000E30F50003C003200AF
:1014F0003E009000E30F500004003E003E009000CC
:101500000000E0000B0032000F0037003E009000AA
:10151000E60F5000480032003E009000E70F5000F8
:101520006A0032003E009000E40F500037003200A5
:101530008B0037008109200060F620004E9A0200DF
:10154000000000008A0037005100200030632000B6
:101550004E9A020000000000AC0007002E00900030
:10156000E10F5000820032001E0090000000E000F9
:10157000030034001E009000E20F500013003400FE
:1015800041022000E0FF20004E9A0200000000000F
:101590008001EB002200200011002000200020002C
:1015A000901C020000000000100798001E00900030
:1015B000E10F500003003A000040EB007500070007
:1015C0000200370080C0B300720007004100200015
:1015D000200221004E9A0200000000006400370043
:1015E00011C0B3000040EB00A8000700F00020008D
:1015F000229702000000000051002000600221003C
:101600004E9A020000000000590037001E009000B2
:101610008040780000C8B30080C070000040EB003C
:101620009A000700A1002000B00221004E9A02009B
:10163000000000004E00370011C0B3000040EB0076
:1016400092000700F0002000229702000000000036
:1016500000032000200798001E0090000000E0001A
:1016600002003A0000052000100798000000EB007F
:10167000000F780011003700AE00900090032000AA
:10168000808F5000020036000003200020079800E1
:101690002E0090008040780010C0B3007B0007004F
:1016A0002E0090000C710200000000002E0090003F
:1016B0000000E800200798001E0FE8001E009000C0
:1016C0009E0F1000ECFF35002900370011C0B30059
:1016D0000040EB006D000700F000200022970200A0
:1016E0000000000010022000200798001E0090005B
:1016F0000000E00002003A000005200010079800FA
:101700000000EB00000F780011003700AE009000E1
:10171000F0072000808F50000200360010022000E9
:10172000200798002E0090008040780010C0B30081
:10173000560007002E0090000C710200000000000F
:101740002E0090000000E800200798001E0FE8001F
:101750001E0090009E0F1000ECFF350004003700C3
:1017600041022000C02020004E9A0200000000002C
:101770000080FA00000006000000FA00B10020001E
:10178000C00921004E9A0200000000000080FA000B
:10179000000006000200FA00004F78001E407800AA
:1017A0000042B000804078000040EB0037000700A6
:1017B000F0002000229702000000000081C0B3006A
:1017C0000040EB0031000700F000200022970200EB
:1017D0000000000011C0B3000040EB002B00070028
:1017E000F00020002297020000000000E1C0B300DA
:1017F0000040EB0025000700F000200022970200C7
:10180000000000000080FA00000006000000FA005E
:101810000040EB004A000700F00020002297020081
:101820000000000031C0B3000040EB0026000700BC
:1018300050002000229702000000000031C0B300D9
:101840000040EB0020000700000A20004E97020035
:101850000000000031C0B3000040EB001A00070098
:10186000000A20004E9702000000000021C0B300D3
:101870000040EB0014000700000A20004E97020011
:10188000000000000080FA00000006000200FA00DC
:10189000004F7800114798001E4090000080FB0028
:1018A0004400DE00804078001E40780006000700FB
:1018B0001E409000EF4060001E40780002000700CC
:1018C0000080FA00000006000200FA00004F7800D5
:1018D000114798001E4090004400DD00104798001A
:1018E0001E4090000004A0001047980010C0B300F4
:1018F0009E4F100003003A001E4090000014A0000C
:10190000104798001E4090000D0007001E409000F8
:101910000034A000104798001E4090000800070007
:101920009E40900070CFB30000C060001047980048
:101930001E409000020007000080FA000000060030
:101940000200FA00004F78001E407800F6460200C0
:1019500000000000CAC2A800CAC2A9000080FA00A4
:10196000000006000000FA0000A52800B06C02008C
:10197000000000000080FA00000006000A00FA00E3
:10198000704080003007980010002000D09388003D
:10199000F4FF070000003700FA70020000000000AA
:1019A000104798001E4090000080FB004007980000
:1019B000CE009000E38F5000200032004E009000D7
:1019C000E30F50000A003C00CE009000E18F500071
:1019D0005B0032004E009000E10F50005E003C00C2
:1019E000CE0090000100E000E7003200DB0037008D
:1019F0004E009000E60F50000E003200CE00900026
:101A0000E68F500004003C004E009000E50F5000AF
:101A100095003200D1003700CE009000E78F5000D3
:101A2000640032004E009000E80F50005400320075
:101A3000CA003700CBFF0700D7FF3700BE00900079
:101A400030C0B300804878003E0090008000E8007D
:101A500080C0B3008048780021E3A800C0C0B30074
:101A6000E495020000000000200798003E0090006E
:101A70008080E8002E0090004800DE00804878005A
:101A80003E009000E30040002E0090008048780067
:101A9000B0C0B300E49502000000000020079800E9
:101AA0003E009000E40040002E0090004800DE0060
:101AB000804878003E009000E50040002E00900035
:101AC00080487800A0C0B300E49502000000000048
:101AD000200798003E009000E60040002E00900095
:101AE0004800DE00804878003E009000E70040009B
:101AF0002E0090008048780090C0B300E49502006A
:101B000000000000200798003E009000E800400020
:101B10002E0090004800DE00804878003E009000D3
:101B2000E90040002E0090008048780021E3A900E1
:101B3000A10020003E009000BA00070096FF370089
:101B4000FA70020000000000104798001E4090004C
:101B50008F00070090FF3700FA70020000000000BD
:101B600010479800FA70020000000000004F780053
:101B70009E4078001E409000BC00070086FF3700A2
:101B8000FA7002000000000010479800FA7002008E
:101B900000000000004F78001E4090000080FB0015
:101BA000C800DD001E80FB0000807000D09388001C
:101BB00079FF3700FA70020000000000104798001B
:101BC0001E4090000080FB00200798001E409000FF
:101BD000E14F500004003A0030C0B3002A71020007
:101BE000000000000300370020C2B3002A71020089
:101BF00000000000FA70020000000000104798008A
:101C0000FA70020000000000004F78009E40900033
:101C1000A0CAB30080CF500003003A0050C5B30003
:101C20009E4F1000050032000000EB0020079800D6
:101C300020C2B3002A71020000000000BE00900024
:101C400070C0B300804878003E0090008000E8003B
:101C50002E00900080487800210020003E00900077
:101C6000700007004CFF3700FA700200000000000F
:101C700010479800FA70020000000000004F780042
:101C80008560A9001E4090000080FB00C800DD00B8
:101C90001E80FB0000807000100798009E009000DE
:101CA00000002200808F5000020036000000220059
:101CB000100798001E009000670040004300DE00FF
:101CC00020079800BE00900050C0B3008048780004
:101CD0003E0090000000E8009E409000014878001F
:101CE0003E0090000080E8001E487800310020008F
:101CF0003E0090004B0007007040800000408800CC
:101D00002E00900000004000104088000000EB0012
:101D10002040880071408000408320000080400007
:101D2000304088000000EB00404088000000EB00DD
:101D3000504088009560A800D0938000314080001A
:101D400004408000800178001E01900004007800AB
:101D5000309D0200000000000FFF3700BE00900021
:101D60000040EB00804878003E0090008000E800D2
:101D70000040EB0080487800110020003E009000F9
:101D80002800070004FF37000080FA00000006006A
:101D90000200FA00004F7800CAC2A900CB22A900B5
:101DA000CB02A900CB42A90020C0B3009E4F100077
:101DB00005003A00CAC2A800CB02A800CB22A800A6
:101DC000CB42A80004003700CAC2A900CB02A90078
:101DD000CB22A900CB42A90010C0B3009E4F100037
:101DE0000300320020C0B3009E4F100006003A00EE
:101DF000C8C2A900C922A900C902A900C942A900F4
:101E0000C8E2A80005003700C8C2A800C922A8007F
:101E1000C902A800C942A800C8E2A8000080FA00D0
:101E2000000006000600FA0010079800210798003D
:101E30000000EB00000F7800070037009E007800DC
:101E40001E00900000804000104078000C710200DD
:101E5000000000001E0FE8002E0090009E0F1000F2
:101E6000F6FF39000080FA00000006000400FA00C6
:101E7000004F7800114798001E80FB001007980063
